:020000022000DC
:106000000000042091860200856707007F6D07006D
:1060100085670700856707008567070000000000A7
:10602000000000000000000000000000856707007D
:106030008567070000000000856707008567070087
:106040008585020085670700E5890200C188020096
:10605000D188020085670700ED810200856707008F
:1060600085670700C5890200D589020061860200A4
:106070008567070085670700856707008567070054
:10608000358E02007186020085670700856707006C
:10609000856707008567070031890200856707006B
:1060A0008567070085670700856707008567070024
:1060B00085670700856707000000000000000000FA
:1060C000856707008567070085670700E18802008C
:1060D000818602008567070085670700058A020040
:1060E000F5890200856707008567070009890200B6
:0860F0000000000085670700B5
:1070000040F8044B40F8045B40F8046B40F8047B04
:1070100040F8048B40F8049B40F804AB40F804BBF4
:1070200040F804CB40F804DB6846704781F000412B
:1070300002E000BF83F0004330B54FEA41044FEA5D
:10704000430594EA050F08BF90EA020F1FBF54EAF8
:10705000000C55EA020C7FEA645C7FEA655C00F094
:10706000E2804FEA5454D4EB5555B8BF6D420CDD65
:107070002C4480EA020281EA030382EA000083EAE8
:10708000010180EA020281EA0303362D88BF30BD88
:1070900011F0004F4FEA01314FF4801C4CEA1131DE
:1070A00002D0404261EB410113F0004F4FEA03333D
:1070B0004CEA133302D0524263EB430394EA050FC8
:1070C00000F0A780A4F10104D5F1200E0DDB02FA37
:1070D0000EFC22FA05F2801841F1000103FA0EF2CB
:1070E000801843FA05F359410EE0A5F120050EF191
:1070F000200E012A03FA0EFC28BF4CF0020C43FAC2
:1071000005F3C01851EBE37101F0004507D54FF0CE
:10711000000EDCF1000C7EEB00006EEB0101B1F51E
:10712000801F1BD3B1F5001F0CD349085FEA300064
:107130004FEA3C0C04F101044FEA445212F5800F6F
:1071400080F09A80BCF1004F08BF5FEA500C50F10C
:10715000000041EB045141EA050130BD5FEA4C0CEF
:10716000404141EB0101013C28BFB1F5801FE9D24C
:1071700091F0000F04BF01460020B1FA81F308BF6F
:107180002033A3F10B03B3F120020CDA0C3208DD3B
:1071900002F1140CC2F10C0201FA0CF021FA02F116
:1071A0000CE002F11402D8BFC2F1200C01FA02F186
:1071B00020FA0CFCDCBF41EA0C019040E41AA2BFAB
:1071C00001EB0451294330BD6FEA04041F3C1CDA73
:1071D0000C340EDC04F11404C4F1200220FA04F093
:1071E00001FA02F340EA030021FA04F345EA03013D
:1071F00030BDC4F10C04C4F1200220FA02F001FAFF
:1072000004F340EA0300294630BD21FA04F0294680
:1072100030BD94F0000F83F4801306BF81F4801119
:107220000134013D4EE77FEA645C18BF7FEA655C8C
:1072300029D094EA050F08BF90EA020F05D054EA5E
:10724000000C04BF1946104630BD91EA030F1EBF63
:107250000021002030BD5FEA545C05D14000494167
:1072600028BF41F0004130BD14F580043CBF01F55A
:10727000801130BD01F0004545F0FE4141F4700140
:107280004FF0000030BD7FEA645C1ABF194610461B
:107290007FEA655C1CBF0B46024650EA013406BF1C
:1072A00052EA033591EA030F41F4002130BD00BFDB
:1072B00090F0000F04BF0021704730B54FF4806498
:1072C00004F132044FF000054FF0000150E700BF19
:1072D00090F0000F04BF0021704730B54FF4806478
:1072E00004F1320410F0004548BF40424FF0000165
:1072F0003EE700BF42004FEAE2014FEA31014FEAA8
:1073000002701FBF12F07F4393F07F4F81F06051F6
:10731000704732F07F4208BF704793F07F4F04BF41
:1073200041F40021704730B54FF4607401F000451E
:1073300021F000411CE700BF50EA010208BF70477E
:1073400030B54FF000050AE050EA010208BF70476F
:1073500030B511F0004502D5404261EB41014FF4D8
:10736000806404F132045FEA915C3FF4D8AE4FF0E0
:1073700003025FEADC0C18BF03325FEADC0C18BFC3
:10738000033202EBDC02C2F1200300FA03FC20FA14
:1073900002F001FA03FE40EA0E0021FA02F1144461
:1073A000BDE600BF4FEA4102B2F1E04324BFB3F5AE
:1073B000001CDCF1FE5C0DD901F0004C4FEAC0026C
:1073C0004CEA5070B2F1004F40EB830008BF20F050
:1073D0000100704711F0804F21D113F13872BCBF0A
:1073E00001F00040704741F480114FEA5252C2F15F
:1073F0001802C2F1200C10FA0CF320FA02F018BFA8
:1074000040F001004FEAC1234FEAD32303FA0CFCFA
:1074100040EA0C0023FA02F34FEA4303CCE77FEA89
:10742000625307D150EA01331EBF4FF0FE4040F4D3
:107430004000704701F0004040F0FE4040F4000082
:10744000704700BF80F0004002E000BF81F00041C3
:1074500042001FBF5FEA410392EA030F7FEA226CFA
:107460007FEA236C6AD04FEA1262D2EB1363C1BF8A
:10747000D218414048404140B8BF5B42192B88BFF9
:10748000704710F0004F40F4000020F07F4018BF1C
:10749000404211F0004F41F4000121F07F4118BF3C
:1074A000494292EA030F3FD0A2F1010241FA03FCE4
:1074B00010EB0C00C3F1200301FA03F100F00043CC
:1074C00002D5494260EB4000B0F5000F13D3B0F194
:1074D000807F06D340084FEA310102F10102FE2A03
:1074E00051D2B1F1004F40EBC25008BF20F0010073
:1074F00040EA03007047490040EB0000013A28BF12
:10750000B0F5000FEDD2B0FA80FCACF1080CB2EB94
:107510000C0200FA0CF0AABF00EBC2505242184312
:10752000BCBFD0401843704792F0000F81F40001B7
:1075300006BF80F400000132013BB5E74FEA41038A
:107540007FEA226C18BF7FEA236C21D092EA030FF6
:1075500004D092F0000F08BF0846704790EA010F70
:107560001CBF0020704712F07F4F04D1400028BF9D
:1075700040F00040704712F100723CBF00F500007F
:10758000704700F0004343F0FE4040F400007047B5
:107590007FEA226216BF08467FEA23630146420261
:1075A00006BF5FEA412390EA010F40F48000704774
:1075B0004FF0000304E000BF10F0004348BF40421A
:1075C0005FEA000C08BF704743F0964301464FF056
:1075D00000001CE050EA010208BF70474FF00003B2
:1075E0000AE000BF50EA010208BF704711F00043F3
:1075F00002D5404261EB41015FEA010C02BF8446C3
:107600000146002043F0B64308BFA3F18053A3F521
:107610000003BCFA8CF2083AA3EBC25310DB01FA68
:1076200002FC634400FA02FCC2F12002BCF1004FEC
:1076300020FA02F243EB020008BF20F0010070477D
:1076400002F1200201FA02FCC2F1200250EA4C00D1
:1076500021FA02F243EB020008BF20EADC70704717
:107660007BB972B90029BEBF00204FF0004106E08F
:1076700008BF00281CBF6FF000414FF0FF3000F042
:1076800081B9ADF1080C6DE904CE002909DB002BAE
:107690001ADB02F04FFDDDF804E0DDE9022304B05F
:1076A0007047404261EB4101002B1BDB02F042FDC1
:1076B000DDF804E0DDE9022304B0404261EB410162
:1076C000524263EB43037047524263EB430302F0C1
:1076D00031FDDDF804E0DDE9022304B0404261EB56
:1076E00041017047524263EB430302F023FDDDF892
:1076F00004E0DDE9022304B0524263EB4303704728
:1077000053B94AB9002908BF00281CBF4FF0FF3108
:107710004FF0FF3000F036B9ADF1080C6DE904CE42
:1077200002F008FDDDF804E0DDE9022304B0704753
:1077300070B54FF0FF0C4CF4E06C1CEA11541DBF07
:107740001CEA135594EA0C0F95EA0C0F00F0DEF8D2
:107750002C4481EA030621EA4C5123EA4C5350EAB7
:10776000013518BF52EA033541F4801143F4801308
:1077700038D0A0FB02CE4FF00005E1FB02E506F099
:107780000042E0FB03E54FF00006E1FB03569CF0EE
:10779000000F18BF4EF0010EA4F1FF04B6F5007FF4
:1077A00064F5407404D25FEA4E0E6D4146EB060666
:1077B00042EAC62141EA55514FEAC52040EA5E50EF
:1077C0004FEACE2EB4F1FD0C88BFBCF5E06F1ED899
:1077D000BEF1004F08BF5FEA500E50F1000041EBD0
:1077E000045170BD06F0004646EA010140EA02007D
:1077F00081EA0301B4EB5C04C2BFD4EB0C0541EA9F
:10780000045170BD41F480114FF0000E013C00F3B3
:10781000AB8014F1360FDEBF002001F0004170BDD7
:10782000C4F10004203C35DA0C341BDC04F11404F0
:10783000C4F1200500FA05F320FA04F001FA05F27C
:1078400040EA020001F0004221F0004110EBD37049
:1078500021FA04F642EB06015EEA430E08BF20EA75
:10786000D37070BDC4F10C04C4F1200500FA04F318
:1078700020FA05F001FA04F240EA020001F00041AA
:1078800010EBD37041F100015EEA430E08BF20EA1D
:10789000D37070BDC4F1200500FA05F24EEA020E65
:1078A00020FA04F301FA05F243EA020321FA04F094
:1078B00001F0004121FA04F220EA020000EBD3704B
:1078C0005EEA430E08BF20EAD37070BD94F0000F4B
:1078D0000FD101F00046400041EB010111F4801F7F
:1078E00008BF013CF7D041EA060195F0000F18BF30
:1078F000704703F00046520043EB030313F4801F6C
:1079000008BF013DF7D043EA0603704794EA0C0F25
:107910000CEA135518BF95EA0C0F0CD050EA41063B
:1079200018BF52EA4306D1D181EA030101F00041B8
:107930004FF0000070BD50EA410606BF10461946E0
:1079400052EA430619D094EA0C0F02D150EA0136EC
:1079500013D195EA0C0F05D152EA03361CBF10462D
:1079600019460AD181EA030101F0004141F0FE41CC
:1079700041F470014FF0000070BD41F0FE4141F450
:10798000780170BD704700BF4A0011D212F5001295
:1079900011D20DD56FF47873B3EB62520ED44FEA67
:1079A000C12343F0004343EA505323FA02F07047E7
:1079B0004FF00000704750EA013002D14FF0FF3025
:1079C00070474FF00000704730B5144685B017A3DC
:1079D000D3E90023FFF744FE054601A9284647F0F6
:1079E0003DFC9DF807309DF806200F491B0443EA33
:1079F00042539DF8082043EAC2239DF8092043EA38
:107A000042139DF80A2043EA5203BDF8042025F0F2
:107A10000105A2F2BC7243EA4263A5FB01012360A7
:107A200005B030BDAFF3008000CA9A3B00CA9A3B54
:107A300000000000182A2DE9F74F054621D0202A22
:107A400022D00A200423C5F8002185F8040185F816
:107A50000531284600F0AAFC0022034695F80541AE
:107A6000A24214D3DFF8DCC0DFF8DCE000EB8403D3
:107A700095F804210132B4EB820F1AD303B0BDE8AC
:107A8000F08F0C200623DEE70E200823DBE711F839
:107A9000044B03F8044B11F8034C03F8034C11F8A2
:107AA000024C03F8024C11F8014C03F8014C01326E
:107AB000D4E795F80521B4FBF2FA02FB1A4913F852
:107AC000041C13F8038C13F8027C13F8016C019268
:107AD000B9F1000F0BD11CF808B01CF807801CF896
:107AE00006701CF801601EF80A108BEA0101D5F837
:107AF0000021202A0CD1B9F1040F09D1DFF84490FC
:107B000019F8011019F8088019F8077019F80660BB
:107B1000019AA21A043310F8229000EB820281EA43
:107B2000090103F8041C517888EA010803F8038C62
:107B300091784F4003F8027CD278564003F8016CEC
:107B4000013495E73F3D0A00343D0A002DE9F04F2E
:107B5000044685B0084600F029FC89460246804666
:107B6000214600204EF0EBFD231D019304F110038C
:107B70000125029322462146002311F82300324EAC
:107B8000305C01F823000133042BF6D1019B013155
:107B90008B42F1D1617963786170617A6171617B47
:107BA0006172A17A6373A378A170A17BA372A37998
:107BB000A171E17BA373E378E170E17AE173E1798C
:107BC000E172E37199F80431AB4234D092F800B01D
:107BD0005678917892F803A08BEA060081EA0A03AE
:107BE00080EA0307039366F0B6F98BEA0000784059
:107BF000107086EA010066F0AEF946407E4056708D
:107C0000039866F0A8F94140794091708BEA0A0028
:107C100066F0A1F98AEA000A029B87EA0A07D77090
:107C200004329342D2D128464246214601354EF0D5
:107C300086FDEDB29EE742462146284605B0BDE8E6
:107C4000F04F4EF07CBD00BF3F3D0A002DE9F04FE4
:107C5000504C904603F003029B101F2B04EB821440
:107C600089469E464C49A8BF4FF01F0E1C2B1D464F
:107C7000A8BF1C2551F822206168033587B025EA8A
:107C8000E575294101920391E268A1688446294182
:107C900000202A410290049105925CF8045B3F4A5F
:107CA000154225F0004111D106AA02EB810151F8DD
:107CB000102C002D40EA0200B8BF5242B8F1010872
:107CC00049F8042BE9D107B0BDE8F08F344A1542DA
:107CD00009D154F82120002BBABFCEF100018A400F
:107CE00042FA0EF2E5E72F4A154214D110392E4A16
:107CF000019E52F8212082FB0616AEF10302002AF3
:107D000044DA51426FF0004242FA01F7B742D0DB49
:107D100006FA01F2CDE74A04B2F1006FB6BF4A0598
:107D200000210421B2F1005FB8BF92001F4EB8BF1E
:107D30000231B2F1804FBCBF52000131B242C7BF25
:107D40001B4F1C4E1C4F1D4E924687FB0ABA77688C
:107D50005744924687FB0ABAB7685744924687FB56
:107D60000ABAF768BA448AFB027236691644144AA2
:107D700052F8212086FB0272019ED20082FB067619
:107D8000104A52F82120AEEB0202B8E746FA02F29E
:107D90008FE700BFA8760A0098760A00FCFFFF7FF5
:107DA000F0FFFF7FC0FFFF7FD8750A009979825AE4
:107DB0006321851070750A00A9BDA02984750A0089
:107DC000B8750A0098750A002DE9F74F00F5A0482C
:107DD0004FF0000A476D88F8B4AD88F8AEADB1F148
:107DE000000B816DC0F820A04FF0FF3304464362C2
:107DF0000CBFFF220C22CB1BD019013B04F5DA7615
:107E00008842C8BF1A46236C0092314604F15400E0
:107E10009847009A8242054613D1002F68D1A549A0
:107E20000522304659F062FA78B1A349052230465E
:107E300059F05CFA48B10823E361002003B0BDE8C3
:107E4000F08F0623F8E70123F6E7B4F8BA31236090
:107E5000A360B4F8BC316360E36094F8BE31C3F34F
:107E600002120132A261BBF1000F40F0BB8194F815
:107E7000BF2188F8B02D180688F8AFBD4BD503F0A8
:107E8000070B0BF1010B4FF0030A05F5DA710AFA43
:107E90000BFA236C5246214404F1540098470544E0
:107EA00098F8B50D01282DD804F58D520221123213
:107EB00001FA0BF1A44611449CF8C1319CF8C2E1CF
:107EC000DB084FEA9E0EDB0243EA4E139CF8C3E147
:107ED00043EADE0300B15BBA22F8023F91420CF1A3
:107EE000030CE9D14FF0030A0AFA0BFA0AF10D0A62
:107EF00016F80A302C2B00F0E3803B2B0ED1072321
:107F0000E3616FE104F58D50524604F2C111143063
:107F100059F000FAEAE74FF00D0AE9E7212B40F0AB
:107F20009B8006EB0A020AF102015378FE2B68D00F
:107F3000FF2B21D0012B5ED0F92B84D1735C042B55
:107F400013D1D17888F8AF1D5079137903EB002352
:107F50000A204343012BD8BF64232362C90744BFCF
:107F6000937988F8B13D0AF108018A46C0E70AEB27
:107F70000301BAF1000FF8D016F801A04B1CA5EBD5
:107F8000030B0AF11F025A4515DB01F2B5115A46DF
:107F900021443046009359F0E8F9009B0BF5DA7163
:107FA0001F440AF12002236C214404F15400984735
:107FB00000230BEB0005BAF10B0FD8D106EB030B36
:107FC0003E4900935246584659F090F9009B03F100
:107FD0000B010028D0D19BF80B30032BCCD19BF8A0
:107FE0000C30012BC8D19BF80E209BF80D3003EB11
:107FF00002236362C0E7735C4A1C9918002BFAD114
:10800000B3E716F801A04B1CA5EB030B0AF11F0206
:108010005A4515DB01F2B5115A462144304600930A
:1080200059F0A3F9009B0BF5DA711F440AF1200205
:10803000236C214404F15400984700230BEB000506
:10804000A26B1AB9DA19A263A4F83CA00AEB0301E7
:10805000BAF1000FD5D188E7A36DDB1B202BB4BF8D
:1080600007230123E8E604F5A55006EB0B011430C5
:10807000009259F04FF9009A93447EE0009259F033
:1080800049F9009A616B236C114461635144ABEB75
:108090000202214404F1540000929847636B009A55
:1080A00029461A4494E0636C394404F1540098471B
:1080B00098E000BF272409002D240900262209008A
:1080C00006EB0A030AF10A0B99785A7802EB0122AF
:1080D00022611979DA7802EB0122626199795A7981
:1080E00002EB01222260197ADA7902EB0122626046
:1080F0005B7A88F8B33D1A0644D503F007030133D1
:1081000005F5DA7103229A4001932144236C009211
:1081100004F15400984798F8B51D009A01290544C8
:10812000A1D8019B04F5A5524FF0020C12324FF07A
:10813000010B0CFA03FC04EB0A000BFA03FB94445A
:1081400090F8BE3190F8BFE1DB084FEA9E0EDB02EB
:1081500043EA4E1390F8C0E143EADE0301B15BBA93
:1081600022F8023F944500F10300E9D10BF1FF3BF7
:108170000BEB4B0B0AF10D0AD34404F5A04301228B
:1081800083F8B42D16F80B30174A04F5A0480BF10C
:10819000010188F8B23DD35CA3610023636341F21F
:1081A000B47A8D421EDD16F801B0606B4B1CEA1AE2
:1081B00050449345204406EB03013FF75FAF5A4616
:1081C000009359F0A7F8626B009B5A440BEB030134
:1081D0006263BBF1000FE4D101238D4288F8AE3D0C
:1081E0003FF761AF012029E6B8720A002DE9F04F90
:1081F00000248BB0CDE90444664B674867490122EF
:1082000025461E6846B1D0F80463164204D01D60AE
:108210001E680296029E144304338B424FEA4202C8
:10822000EFD15D4BD3F87C218AB10022C3F87C21C9
:10823000D3F87C310393039B4FF0A04344F00044F8
:10824000D3F810350493564BD3F810350593E3B2A9
:10825000D3B1544F01260025344210D0AB0003F1B6
:10826000804303F5C043D3F81005D3F8101557F831
:10827000253023B1C1F30141C0F3052098470135F2
:10828000082D4FEA4606E7D1002C7FDA0DF1200BCE
:1082900000230893CBF80430DFF804914FF0FF334C
:1082A000069307930025404B0193A846019A12F9C3
:1082B000013F01925A1C50D0C3F3C20000F12802C2
:1082C0000DEB020C03F007011CF8102CCA40D70775
:1082D000DCB203F03F0640D5324A17463244A409C7
:1082E00092F9282057F822A0BAF1000F0AD1032CE6
:1082F00033D11BF800E001228A4042EA0E020BF85B
:10830000002001E0032CF4D01F2E8BBF03F01F03CD
:1083100033464A464FF0A04203F5E07352F823304B
:108320001CF8182CCA40D207C3F3014305D5022B11
:1083300013D1032C0BD1214604E0032B0DD1032CC8
:1083400005D10221304637F0C1FC0135EDB2BAF15A
:10835000000F02D021463046D04708F10103022B1E
:108360004FF00108A2D18DB14FF0A0430499D3F88A
:108370001025D9F81035914202D10599994205D0BE
:108380000492089ACDE90532099B8AE70BB0BDE853
:10839000F08F00BF0061004000600040206100409D
:1083A000000300501C61012073610120D0F80031EE
:1083B000103B102B07D8054A22FA03F313F0010FE4
:1083C00008BF002070470020704700BF0101010076
:1083D0002DE9F04F04468DB00846FFF7E7FF0D4644
:1083E00001900246214695F804014EF0A8F995F84F
:1083F0000461231D013E099304F11003F6B20A93B0
:10840000627A637B62736279627262786271A27A65
:108410006370A378A270A27BA372A379A271E279A0
:10842000A373E378E270E27AE271E27BE272E373D3
:1084300025462246002312F823105148415C02F8D9
:1084400023100133042BF6D1099B01329342F1D161
:10845000019A214630464EF072F9002E00F08C80D1
:1084600095F80080AB780093404665F074FD02906B
:1084700065F071FD039065F06EFD6F780B903846E6
:1084800065F069FD024665F066FD049065F063FDE8
:108490008246009895F803B065F05DFD059065F0A3
:1084A0005AFD069065F057FD8146584665F053FD2C
:1084B000079065F050FD089065F04DFDDDE9023153
:1084C00083EA010C0B9B069983EA0C0C82EA0C0CE4
:1084D0008AEA0C0C81EA0C0C89EA0C0C009980EAFF
:1084E0000C0C87EA0C0C81EA0C0C04995A404A40A7
:1084F00005998AEA02024A40089989EA02024A403A
:108500004240009988EA02024A408BEA02026A70FD
:10851000039A05995A408AEA02024A4006994A405B
:10852000079989EA02024A40424088EA02027A40F8
:108530008BEA0C0C8BEA020B85F800C085F802B0C0
:10854000029A5340049A53408AEA030A089A89EA35
:108550000A0981EA09035340584000990A9B88EAB6
:10856000000887EA08077940E9700435AB427FF4D8
:1085700077AF013EF6B243E70DB0BDE8F08F00BF24
:10858000343C0A0010B54FF08043D3F8044362072F
:1085900007D54FF4847060F0D2F810B11E4B1B6801
:1085A0009847A30608D54FF48A7060F0C8F818B150
:1085B0001A4B00201B689847600608D54FF48C7052
:1085C00060F0BDF818B1154B01201B6898472106D3
:1085D00008D54FF48E7060F0B2F818B1104B00203F
:1085E0001B689847E20508D54FF4907060F0A7F833
:1085F00018B10B4B01201B689847A3050AD54FF40F
:10860000927060F09CF828B1054BBDE810401B68E3
:108610000220184710BD00BFAC620120B0620120EB
:10862000B4620120DFED0A7A9FED0A7ADFED0A6A73
:10863000A0EE277ADFED097AE7EE007AB7EE007A4E
:10864000A0EE267A67EE807A87EE870A704700BF31
:108650006BD30DBCBA132FBDAEE534BF75AA2A3E4D
:1086600002480322002122F07BBE00BF00B0004080
:1086700002480422012122F073BE00BF0010014015
:1086800002480422022122F06BBE00BF00400240DB
:1086900008B57E4A7E4B7F498B42C0F0BF807E4B3F
:1086A0007E4A00219342C0F0BE804FF08053D3F841
:1086B0003021082A4ED14FF080420021C2F80C111F
:1086C000C2F81011C2F8381502F54042D3F804146C
:1086D000C2F82015D3F80814C2F82415D3F80C14E6
:1086E000C2F82815D3F81014C2F82C15D3F81414B6
:1086F000C2F83015D3F81814C2F83415D3F81C1486
:10870000C2F84015D3F82014C2F84415D3F8241445
:10871000C2F84815D3F82814C2F84C15D3F82C1415
:10872000C2F85015D3F83014C2F85415D3F83414E5
:10873000C2F86015D3F83814C2F86415D3F83C14A5
:10874000C2F86815D3F84014C2F86C15D3F8443455
:10875000C2F8703555F069FF18B1514B514AC3F852
:108760008C2655F062FF18B14F4BFB22C3F8182539
:1087700055F05BFF58B14FF080424FF08051D2F876
:10878000E43ED1F8581261F30303C2F8E43E55F019
:108790004CFF20B1454B4FF40072C3F840264FF018
:1087A0008053D3F83031082B09D14FF08043D3F8F0
:1087B0000024D10744BF6FF00102C3F800243C4AF3
:1087C000D2F8883043F47003C2F88830BFF34F8F7B
:1087D000BFF36F8F4FF01023D3F80C22D20725D5AB
:1087E000344B0122C3F80425D3F80024002AFBD01F
:1087F0004FF01022D2F80C3223F00103C2F80C32F1
:108800002C4BD3F80024002AFBD00022C3F8042507
:10881000D3F80024002AFBD000F0ACFC52F8040B83
:1088200043F8040B38E743F8041B3BE7D3F8002276
:10883000002A03DBD3F80432002B22DA1D4B01227D
:10884000C3F80425D3F80024002AFBD04FF01022EF
:108850001221C2F80012D3F80024002AFBD04FF0F6
:1088600010231222C3F80422124BD3F80024002A4A
:10887000FBD00022C3F80425D3F80024002AFBD043
:10888000CAE70D4B0D4A1A6041F030FADC800A004D
:108890000000012094050120C00501201C6F01206B
:1088A000005000404881030000F00040009002406A
:1088B00000ED00E000E00140000001200090D00346
:1088C0000149024847F0E6BDE06101200030004068
:1088D00002494FF0402047F0DDBD00BF1462012087
:1088E00008B50748D0F8183143B14FF48C715FF0E8
:1088F0001EFFBDE80840034857F04DBA08BD00BF51
:10890000003002408061012008B50748D0F81831D6
:1089100043B14FF48C715FF00AFFBDE80840034893
:1089200057F039BA08BD00BF00F00240A461012031
:1089300073B51F4C022501A861F0B9FC052812D1BE
:108940001C4D4FF40C741C48ADF802400DF10201AF
:1089500061F039FC08B30C2803D1184918485AF0C3
:10896000F0FB02B070BD019B032B14D004D8022B86
:10897000E1D100232370DEE7A3F10902022ADAD84D
:108980000A2B06D0092B14BF0120022047F048FC17
:10899000D1E70020FAE72570CDE7D5F8B430002BF9
:1089A000D1D01E680448D3E9011290473346F6E758
:1089B000FD6E0120BC620120EC5E01202420090034
:1089C000E86309000149024857F0DBBFC861012094
:1089D000009000400149024857F0D3BFD461012004
:1089E00000A000400149024864F0FFB9486201203C
:1089F000002000400149024864F0F7B96C62012090
:108A0000008002402DE9F04FBC4BBD4AD3F8001363
:108A1000002385B01C4601201D4621FA03F6F60707
:108A20000BD552F8236046B100FA03F6344342F8FE
:108A30002350BFF36F8FBFF34F8F0133192BECD14E
:108A4000E10738D5AD4B0122C3F81425C3F8102532
:108A500000221546930003F1804303F51C330132D5
:108A6000082A5D609D62F5D1A44BA6485D629D64B5
:108A7000C3F85851D3F80024D3F800140A43C3F8BC
:108A80000024D3F80023C3F808239F4AC3F8042323
:108A900000214FF4927258F07EFC9A4A8DF80850EB
:108AA00040231383138101214FF4807301A8ADF893
:108AB000043018F0DBF814F4006F924D07D08F4BA0
:108AC000D3F8A836A5F81631012385F81C31A20287
:108AD00004F4800635D5894AD2F8143513F480732E
:108AE00008D01EB1D2F80034DB0702D408204BF0C6
:108AF00061FD0123814AD2F81015CF0540F14A816A
:108B000095F81C318BB1002385F81C31B5F816316E
:108B10009BB24FF4E06203930121882301A8ADF8D2
:108B20000420ADF8083018F0A1F8744B4FF44072EF
:108B3000D3F820350293012101A8ADF8042018F0E4
:108B400095F87EB36D4BD3F8006440F20172324069
:108B5000F005C3F8002409D50121C3F82C1501A89C
:108B60004FF48063ADF8043018F080F871050FD52C
:108B7000624B0122C3F808259A65D3F8002312F44A
:108B8000001208BFC3F854214FF40012C3F80423A5
:108B9000B20507D54FF4A063012101A8ADF8043058
:108BA00018F064F823022ED5544BD3F88014D3F870
:108BB0008424D3F888E4D3F88CC4D3F89074D3F821
:108BC0009464D3F89804D3F89C3411F07F0FD2B298
:108BD00001D1052A17D04FF4C0688DF808108DF820
:108BE0000E00012101A8ADF804808DF809208DF850
:108BF0000AE08DF80BC08DF80C708DF80D608DF8C3
:108C00000F3018F033F8414B23403BB1BFF35B8F7B
:108C10003F4B4FF000021A70BFF35B8F394FDFF804
:108C2000DCB00026B8464FF0140AB14606F10C033A
:108C300024FA03F3D80726D50AFB06B305EB461141
:108C4000D3F80827D8F8003013FA82F3C8F80030B8
:108C5000B1F806C090B2082E1CFA82F24FEA461311
:108C6000CA8000F0A480B8F80820824240F09F80BB
:108C7000CA88B8F8041092B2914240F2988016B9AE
:108C800024481AF04FFE0136092E08F12008CDD1F4
:108C9000214B2340002B00F09480184BD3F86C84B8
:108CA000C3F86C84BFF36F8FBFF34F8F14F48064ED
:108CB0001CBFD3F88044D3F88064DFF848A01DBF00
:108CC000C6F3C016C4F3C01486F0010626464FF062
:108CD00000094FF4E06B28FA09F1CA0703D4B9F18F
:108CE000000F31D184B3054B142202FB09315FFA26
:108CF00089F0D1F80836DAF810100FE00070024061
:108D000000710240A82101200514C001FCFB1F00D6
:108D1000C82201204C7002400004000151FA83F186
:108D2000CAF8101005EB4911B1F816E05EFA83FCA1
:108D3000A1F816C0B1F816C0BAF814E01FFA8CFCFE
:108D4000E6455ED94BF016FC09F10109B9F1080FAF
:108D50000AF1200ABFD100244FF0010904F11003E9
:108D600028FA03F3DB0701D474B96EB105EB4412A2
:108D70006301D17A002955D0D288B98892B2914244
:108D800050D9E0B24BF016FC0134082C07F1200753
:108D9000E4D116E0002B7FF4C8AE95F82131002B0A
:108DA0007FF4C3AE4FF40013C2F80833BDE62B4482
:108DB000DA7A8AB94FF0E023D3F8F03DD90700D52D
:108DC00000BE1A4A1A4B136010460023536005B0C8
:108DD000BDE8F04F07F0E8BEDA88A8F8042083F871
:108DE0000B90DB888DF808609BB24FF4E0620121A4
:108DF00001A8ADF8042003938DF8099017F036FF11
:108E000041E7C98AADF804B089B260F07F000391F0
:108E100000218DF808008DF8091001A8012117F034
:108E200025FF91E72B4483F80A90ADE7C068012045
:108E300097D0080010B5074CD4F800314BB1064B61
:108E40005B68984720464FF48071BDE810405FF0A2
:108E50006EBC10BD0000014090620120022A2DE985
:108E6000F04159D13B4B826883FB02423A4D846901
:108E700085FB046422440A60DFF8F0C042688CFB82
:108E80000242364EC46986FB047422444A6002687A
:108E900083FB0242046A85FB046422448A60304EEC
:108EA000026886FB02422F4C056A84FB05752A4442
:108EB000CA604FF06045426885FB0272C76985FB56
:108EC00007E73A440A61826884FB0272876986FB7D
:108ED00007E73A444A61426983FB02728A61026988
:108EE0008CFB0272CA61C26883FB02720A62C368A9
:108EF00086FB03234B62036985FB03238B62436973
:108F000084FB0323CB620023C1E91033C1E90E3394
:108F1000C1E90C33BDE8F081134B902404FB02320D
:108F200002F1480E02F18C0501F14406683250F856
:108F3000043B55F804795EF804CB1C468CFB048492
:108F400041F8044B87FB0343AA4246F80439EED1AB
:108F5000E0E700BFD8E3CEB8281C3107CD3C410D77
:108F60009A615FC9669EA0F630730A0033C3BEB231
:108F70002DE9F8431C4E04468846914600254FF4DF
:108F8000004746F00106B4F85E20ABB29A4205D81D
:108F900094F83400BDE8F84336F0ACBE03F00F039C
:108FA00047FA03F313EA090F14BF012100212046F9
:108FB0004EF028FAB4F85E30AAB2A3EB08039A4246
:108FC00003DD94F8340036F0C3FE94F8610036F007
:108FD000BFFE4020B04794F8610036F08BFE402081
:108FE000B0470135CFE700BFD0230A00F8B590F8AD
:108FF0006530013B80F86B3090F866305A1E80F87F
:109000006C20012B88BF90F86C304FF000058CBFAE
:1090100003F1FF33012380F86D30044680F86E5071
:109020000127856540F2033694F86330EAB2934233
:109030003CD82368314A934257D002F5805293427C
:1090400055D002F58052934253D002F580329342BC
:1090500051D002F5805293421ED10423284850F883
:10906000332000EBC300002590F90430012151604A
:10907000002BC2F80455D160C2F80855C2F810554B
:109080004FF48035C2F8045306DB5A0903F01F037E
:1090900099401C4B43F82210236801224FF47A7147
:1090A0005A60DA60C3F840151A60F8BDA36C03EB90
:1090B00002131B7B1F2B86BF03F01F0312494FF0C7
:1090C000A04103F5E07341F82360A36C94F86D10A0
:1090D00003EB02133942187B04D036F039FE7F00CF
:1090E0000135A1E736F006FEF9E70023B6E70123D4
:1090F000B4E70223B2E70323B0E700BF00800040DB
:109100008C6D0A0000E100E00003005000280CDB39
:109110004309064900F01F0020330122824041F834
:109120002320BFF34F8FBFF36F8F704700E100E044
:109130004309064900F01F0020330122824041F814
:109140002320BFF34F8FBFF36F8F704700E100E024
:109150000028ABBF00F16040054B00F5614000F016
:109160000F004FEA4111B4BF195480F80013704743
:1091700014ED00E0BFF34F8F0549064BCA6802F4B7
:10918000E0621343CB60BFF34F8F00BFFDE700BF2A
:1091900000ED00E00400FA05014B1868704700BFBD
:1091A0005400012007EE900AF5EEC07AF1EE10FAB5
:1091B00001D400F009B808B580F0004000F004F8D0
:1091C000404261EB410108BD70B5FEF793F80C4BCE
:1091D000002204460D46FEF7ABFAFEF7D5FB064625
:1091E000FEF766F8074B0022FEF7A2FA02460B468E
:1091F00020462946FDF71EFFFEF7C6FB314670BD2F
:109200000000F03D0000F04170B510EE105A25F05E
:1092100000440123B4F1FF4FB0EE403A064603602C
:1092200004D320EE003AB0EE430A70BD34B9DFED4E
:10923000D07AB7EE007A87EE273AF4E7B4F1E45F2C
:109240000BD2002DBEBF4FF0FF330360B1EE400ADA
:1092500024F080FDB1EE403AE5E7002D80F2C682B1
:10926000B4F1964FE3D2B4F17A5F9FEDC25A78D24F
:10927000DFEDBF0A20EE050A002000F015FEF0EE3B
:10928000402AF5EE402AF1EE10FAD0D023EE220A61
:10929000B0EEC00A85EE000A24F05CFDF5EEC02AAF
:1092A000F1EE10FAB0EE402A40F1B9804FF0FF33F2
:1092B000B4F17E5F336000F09382B4F1804F00F030
:1092C0008F82B1EE433A6B0000F1DE81AA4B9C42E3
:1092D00000F2F580B0EE430A24F03CFDA74B9C421F
:1092E000B1EE400A40F29D80B7EE007A37EE437A45
:1092F00067EE077ADFEDA26A9FEDA26A9FEDA23AC0
:10930000A7EEA66ADFEDA16AE6EE276A9FEDA06AE6
:10931000A6EEA76ADFED9F6AE6EE276A9FED9E6ADA
:10932000A6EEA73ADFED9D6AE7EE866A9FED9C6A9E
:10933000A6EEA76ADFED9B6AE6EE276A9FED9A6AC2
:10934000A6EEA76ADFED996AE6EE276A23EE073AF2
:10935000A6EEA73AF6EE007AA7EE673A33EE003AA9
:10936000FFE0B1EE407AB0EE470A1DF0FBF9B4EE33
:10937000407AF1EE10FA19D0F6EE007A27EE277A4D
:10938000B0EE470A1DF0EEF937EE400A30EE000A63
:10939000F0EE407AFEEECF7A17EE903A062B39D8EF
:1093A000DFE803F02312121F1F2B2B00DFED807A62
:1093B00077EEC37A17EE903A03F0010307EE903A86
:1093C0009B00B8EEE70AE9E7F6EE007A37EEC00A4E
:1093D000DFED670A20EE050A00F036FBF1EE402AC9
:1093E0004FE7F7EE007A37EEC00ADFED610A20EEB4
:1093F000050A002000F058FDF0E7F7EE087A30EE9D
:10940000670ADFED5B0A20EE050A00F01DFBB1EEF6
:10941000400AE3E7F0EE007A30EE670AE5E7012361
:1094200046E7644B9C4264D99FED637A33EE477AFA
:1094300067EE074A9FED616ADFED616ADFED615A11
:109440009FED615A9FED613A64EE877AE7EE866A96
:109450009FED5F6AA6EEA76ADFED5E6AE6EE276A19
:109460009FED5D6AA6EEA76ADFED5C6AE7EEA65A9D
:10947000DFED5B6AE5EEA76ADFED5A5AE6EEA75A22
:10948000DFED596AE5EEA76ADFED585AA7EEA55A57
:10949000DFED575AE5EE275A9FED565AA5EEA75A2B
:1094A000DFED555AE5EE275AE5EE876AA6EEE73A74
:1094B000DFED527A94EE863A33EE673A4EE7504B40
:1094C0009C4206D9B0EE007A37EE437A9FED280A27
:1094D0000EE74C4B9C4206D99FED4B7A9FED240A38
:1094E00033EE477AA4E7F7EE007A33EE673A9FED62
:1094F000200A9FED467ADFED467ADFED466AE3EE1D
:10950000077A9FED457AA7EE837ADFED447AE7EE9E
:10951000037A9FED437AA7EE837ADFED4D7AE7EE8B
:10952000037A9FED407AE3EE076A9FED3F7AA6EE5D
:10953000837ADFED3E6AE7EE036A9FED3D7AA6EEA1
:10954000837AF7EE006AE7EE036A67EE837A87EEC6
:10955000A67AFEEE006AF0EE477AE3EE267A37EE60
:10956000803A002DBFF65FAE32EE433A5BE600BFB5
:1095700000000000DB0F49406666663F1F4A3B3F24
:10958000A283D337679767393F239E3DA1549C3A06
:109590007E02F23B01F0893D752C3C384584E2386F
:1095A00034B6053AC66E3D3B1599A83C661AA53EF1
:1095B0000000004B07336D3E0C5BEC3E6B7BA53926
:1095C00076F4B7BA67F8663A85300DBA521CE631C0
:1095D00007E7C73B474D06BD5EB9F73E27F9A3B97C
:1095E000FE7771BB3D37933C3C2117BEF7E9AF399D
:1095F0009916143BFEFC28BC155A843DCDCDF83D90
:1096000017A6DD3F1FA69D3FC316BB3F5E3C5B3CDC
:1096100078756A3EAF72D53DB24B7A3FE73ABA3FB2
:10962000F400223FDBD5523BDFEF443F2D390840A9
:10963000BE2E1D4067FF0538B435F13ABDD7F5366B
:10964000E440DA3CE6DC153E7ACCA63E5A245C3E89
:109650003F239EBDD6EE4B3A54BF983C6E0F303E32
:10966000C5D0383F3B2DB23FE8C4D5BAD23D5B3AB6
:109670005C061CBAFD0C503A610B36BBABAAAA3D86
:109680001D7FD63E00000000B4F1824FF7EE002AA5
:1096900075D2FDEEC35A1FED197A5FED196A1FED01
:1096A000196AF8EEE57A15EE903A73EE677A033BA5
:1096B000E7EE876A1FED1E7AA6EEA77A5FED1F6AB6
:1096C000E7EE276A1FED207AA6EEA77A5FED216A02
:1096D000E7EE276A1FED227AA6EEA77A5FED236AEE
:1096E000E7EE866A1FED246AA6EEA76A5FED256A9B
:1096F000E6EE276A1FED266AA6EEA76A5FED276AE7
:10970000E6EE276A27EE277AE6EEA72A87EE223AC8
:10971000B6EE007AA7EE873A042B3FF622AFDFE8D9
:1097200003F02B2825220300B1EE087A37EE877A62
:10973000F1EE046A77EEA66A66EE876AB1EE007A09
:1097400037EE877A27EE267AB0EE080A37EE800ADF
:1097500020EE070AB0EE007A77EE877A27EE800ACD
:1097600024F0F8FAFAE5B7EE007AE1E7F7EE006ADE
:10977000E4E7B7EE007AE7E7B7EE000AEAE7B0EE13
:10978000430A24F0E7FAB4F1B94F30EE620A24D26A
:10979000C2EE836A5FED4C5A1FED4C6A66EEA67A04
:1097A000B6EE007AA7EEA56A5FED4F5AE6EE275AAD
:1097B0001FED506AA5EEA76A5FED515AE6EE275AF3
:1097C0001FED526AA5EEA76A33EE477A1FED543AB1
:1097D000A6EE263AA7EE003AC3E623EE003AC0E62C
:1097E0001FED583AC0E61FED593A1CE5B4F17E5F13
:1097F000F9D0B4F1804FF6D01FED5E2A63E500BFCB
:109800007FB510EE105A834A25F000439342044678
:1098100005D8002380ED000A4360002022E07E4A44
:1098200093423AD825F00043002DDFED7C7A7C4A44
:1098300023F00F0318DD934230EE670A09BFDFED16
:10984000797A9FED797A9FED797A30EE670A70EE3A
:10985000477A30EE670AC0ED007A30EE470A80EDB5
:10986000010A012004B070BD934230EE270A09BFFF
:10987000DFED6C7A9FED6C7A9FED6C7A30EE270A03
:1098800070EE077A30EE670AC0ED007A30EE070A14
:1098900080ED010A4FF0FF30E4E7654A93426DD84E
:1098A0009FED647AB0EEC00AF6EE007AE0EE077A39
:1098B000FDEEE77AF8EEE76A17EE900ADFED577AE9
:1098C000A6EEE70A1F28DFED587A66EEA77A30EE9B
:1098D000677A09DC5849461E25F0004251F82610E7
:1098E00022F0FF028A4207D117EE102AC2F3C752B4
:1098F000C2EBD352082A02DC84ED007A1BE09FED14
:10990000497AB0EE406AA6EEC76A70EE467AE6EE95
:10991000C77A9FED467AD6EE877A36EE677A17EEEB
:10992000102AC2F3C752C2EBE353192B15DC84EDA6
:10993000007AB0EE460A30EE470A002D30EE670A94
:1099400084ED010A8EDAB1EE477AB1EE400A84ED79
:10995000007A84ED010A404284E79FED387AB0EE48
:10996000460AA6EEC70A76EE407AE6EEC77A9FED83
:10997000347AD6EE877A30EE677ABDE7B3F1FF4FDF
:1099800006D330EE400A80ED010A80ED000A44E77C
:10999000DA15863AA3EBC25307EE903ABDEEE77AAA
:1099A000DFED286AB8EEC77A77EEC77A8DED017AD7
:1099B00067EEA67ABDEEE77AB8EEC77A77EEC77A99
:1099C0008DED027A67EEA67AF5EE407AF1EE10FAA6
:1099D000CDED037A19D1B5EE407AF1EE10FA16D03A
:1099E0000223214601A800F089F8002DBFF63AAF06
:1099F000D4ED007AF1EE677AC4ED007AD4ED017A05
:109A0000F1EE677AC4ED017AA5E70323E9E70123C4
:109A1000E7E700BFD80F493FE3CB1640800FC93FAF
:109A2000D00FC93F004435374344353708A3852E4E
:109A3000800F494384F9223FC4670A0000A3852EA2
:109A400032318D240000804310EE103A23F00043A1
:109A5000B3F1485FB7EE007A04D2FDEEC07A17EE9C
:109A6000902ABAB360EE006ADFED1C5A9FED1C6AC3
:109A70001C4AA6EEA56A9342DFED1B5AE6EE265A73
:109A80009FED1A6AA5EEA66ADFED195AE6EE265A90
:109A90009FED186AA5EEA66A60EEC00A26EE266A59
:109AA000F6EE007AE6EE860A66EEA77A04D877EE3E
:109AB000E07A37EE670A70470F4A93429ABF03F184
:109AC0007F4306EE903AF5EE026A37EE667A77EE5D
:109AD000E67AECE7B0EE470A704700BF4ED747ADD5
:109AE000F6740F319999993E7CF293B4010DD037F9
:109AF000610BB6BAABAA2A3D0000483F2DE9F04FF2
:109B00009246033A48BF0AF10402D7B0D2109B46EE
:109B1000551C2DB202910BF1FF31EB0080460DF187
:109B20006809501A0BF1090CC24F0393AAEBC50543
:109B300000EB0C064C460028AABF3B5CDFEDC17A67
:109B400007EE903A00F10100A8BFF8EE677AB04244
:109B5000E4EC017AEFD142AF08EB8B0309EB8B0405
:109B60000193BE46DFEDB77A26464046F0EC016A27
:109B7000019B36ED017A9842E6EE877AF6D1013103
:109B80008C45EEEC017A04F10404EBD1A949DFED38
:109B9000AA6A9FEDAA6A531809240593A3000493A7
:109BA00056AB03EB840212ED140A07EB840006A9FE
:109BB0002246002A45DC28463EF02EF8B0EE407AD8
:109BC000B4EE000A27EE000A1CF0CCFDF2EE007A9B
:109BD000A0EE677A002DFDEEC77A17EE906AF8EED8
:109BE000E77A37EE677A3EDD06AA601EC5F1080EF9
:109BF00052F8203043FA0EF10E4401FA0EF1591AD0
:109C000042F82010C5F10702114100293ADD002277
:109C100001360DF1180E1346944255DC002D03DD7C
:109C2000012D62D0022D6AD002292BD1B7EE000A95
:109C300030EE477A33B328463DF0EEFF37EE407AF8
:109C400020E060EE267A013AFDEEE77AF8EEE77A58
:109C5000A7EEC60ABDEEC00AA1EC010A30ED010A6A
:109C600037EE800AA5E705D1621E06A951F8221039
:109C70000912CAE7F6EE007AB4EEE77AF1EE10FACE
:109C800020DA0021B5EE407AF1EE10FA40F084803F
:109C9000601E00230DF1180E082838DC002B56D169
:109CA0000FA9012251F8040DB0B3049B3E1D04EB33
:109CB0000B01601C1E4409EB8101224490422DDD02
:109CC00014466BE70221A2E7DEF8000053B920B189
:109CD000C0F58070CEF80000012001320EF1040EB4
:109CE000034699E7C0F1FF00F4E704F1FF3E06A840
:109CF00050F82E2002F07F0240F82E2094E704F165
:109D0000FF3E06A850F82E2002F03F02F4E75EF86E
:109D1000202001381343BFE70132C3E7059B1B5CDA
:109D200007EE903AF8EE677A4446E1EC017ADFED0F
:109D3000457A8C46F4EC015A019B3CED017A9C4239
:109D4000E5EE877AF6D1E6EC017A0130B6E7013C20
:109D5000083D06AA52F82430DBB12846B7EE000AC7
:109D60003DF05AFF9FED347A381D4FEA840800EB2E
:109D70008400234606AD002B3CDA2346002B63DB30
:109D8000DFF8BCE0DFED2F7A07EB830C0025E01A4B
:109D900047E0013C083DDDE7039BB0EE470AA3EB3B
:109DA0000A003DF039FF9FED257AB4EEC70AF1EEC7
:109DB00010FA19DBDFED207A60EE277A06AAFDEEB5
:109DC000E77A0835F8EEE77AA7EEC70AFDEEE77AFC
:109DD000BDEEC00A10EE103A42F8243017EE903A69
:109DE000013442F82430B8E7BDEEC00A06AA10EEEE
:109DF000103AF6E755F8232007EE902AF8EEE77AB6
:109E0000013B67EE807A20EE070A60ED017AB2E747
:109E1000FEEC016ABCEC017A01350A2DE6EE877A88
:109E200001D08542F4DD56AA02EB800040ED287A8D
:109E3000013BA3E744680A000000803B0000804328
:109E40000C690A00000000002FA81FED027A00EB49
:109E500008032246002A17DAE1B1F1EE477A029BA5
:109E6000C3ED007ADDED2E7A77EEC77A01239C42AE
:109E700013DA09B1F1EE677A029B06F00700C3ED31
:109E8000017A57B0BDE8F08F73ED017A013A37EEF1
:109E9000277ADFE7F0EE477AE1E7B0EC017A0133A9
:109EA00077EE877AE3E700BF10EE103A23F0004325
:109EB000B3F1485F04D2FDEEC07A17EE903A5BB37F
:109EC00020EE007ADFED157A9FED156AA7EE276A7E
:109ED000DFED147AE6EE077A9FED136AA7EE876A44
:109EE000DFED127A60EE076AE6EE077A30B99FED91
:109EF000106AA7EE276AA6EE260A704767EEE67A92
:109F0000B6EE006AE0EE867AD7EE870ADFED097AD0
:109F1000E6EEA70A30EE600A704700BFD3C92E2FC5
:109F2000342FD7B21BEF3836010D50B98988083C61
:109F3000ABAA2ABEABAA2A3E10EE103A23F000428A
:109F4000B2F1465FF0EE407A14D2BDEEC07A17EE61
:109F5000101A29BB431C134306D1F0EEC07AB7EEAA
:109F6000007A87EE270A7047012800F09B80BFEE39
:109F7000007AF6E74C498A4212D3002B9FED4B7AC8
:109F8000B8BFF1EE407A37EE677ADFED497AB8BFB5
:109F9000F1EE600A77EEE07ADFED460A77EE877A37
:109FA00067EEA76ADFED445A9FED446A9FED445A7D
:109FB0003D4926EEA67A67EEA64AA7EE256A8A42B2
:109FC000DFED405AE6EE075A9FED3F6AA5EE876A3D
:109FD000DFED3E5AE6EE075A9FED3D6AA5EE876A31
:109FE000DFED3C5AE7EE055A9FED3B5AA5EE875A46
:109FF000DFED3A5AE5EE075A9FED395AA5EE875A3A
:10A00000DFED385AE5EE075AB0EE467AA5EEA67AAD
:10A01000B0EE606AA7EE246A9FED337AE6EE260A78
:10A02000E4EE870A37EEA00A1DD307EE100AF8EE19
:10A03000C76A60EE005A30EE260A9B1785EE806AEA
:10A0400003F00203C3F1010307EE103A36EE606A33
:10A05000B8EEC77A77EEC67AB0EE006AE7EEC66A67
:10A0600026EE870A704701281CD010EE103A6FF3D5
:10A070000B0306EE903A76EEE77A70EEE70AFFEE13
:10A08000007A87EE807AF7EE007A17EE103A6FF3D7
:10A090000B0300EE103AE6EE807AE0EE807AA7EE4F
:10A0A000870A7047704700BF40A12C3FDA0F493F35
:10A0B00068212233000000005FAE9BB745F4A3384F
:10A0C0008453D937C8261A3A16696B3BA427B33C88
:10A0D0008988083E7AC09538B937813948DEBE3A5A
:10A0E0001F37113CD10D5D3DABAAAA3E42084B087B
:10A0F00002F0553203F05533801AC91A8A088308D2
:10A1000001F0333100F0333002F0333203F03333F7
:10A110000344881803EB131300EB101003F00F3304
:10A1200000F00F30184400EB002000EB0040000E60
:10A13000704700BF2DE9F04782B00646DDF828E001
:10A140000846B4460D46002B4ED18A4214466DD9BE
:10A15000B2FA82F242B1C2F12003954026FA03F32B
:10A1600094401D4306FA02FC260CA7B2B5FBF6F19B
:10A170004FEA1C4306FB115543EA054301FB07F078
:10A18000984209D9E31801F1FF3580F00381984224
:10A1900040F20081023923441B1A1FFA8CFCB3FBE6
:10A1A000F6F006FB10334CEA034C00FB07F3634563
:10A1B0000AD914EB0C0C00F1FF3580F0ED806345FB
:10A1C00040F2EA80A444023840EA0140ACEB030CC0
:10A1D0000021BEF1000F04D02CFA02F30022CEE9D8
:10A1E000003202B0BDE8F0878B4209D9BEF1000F02
:10A1F00001D0CEE900610021084602B0BDE8F08739
:10A20000B3FA83F1174600294DD1834202D3B242FB
:10A2100000F20F81B6EB070C60EB030301201D4633
:10A22000BEF1000FDDD0CEE900C5DAE7002A00F06C
:10A2300098801A46B4FA84F3002B40F0AF800B1BD1
:10A24000270CA6B20121B3FBF7F54FEA1C4007FB30
:10A25000153340EA034306FB05F8984507D9E31890
:10A2600005F1FF3002D2984500F2E8800546A3EBE5
:10A2700008031FFA8CFCB3FBF7F007FB10334CEA22
:10A28000034C06FB00F3634508D914EB0C0C00F1FA
:10A29000FF3602D2634500F2CE803046ACEB030CB1
:10A2A00040EA054095E7C1F120058B4022FA05FC04
:10A2B0004CEA030C00FA01F426FA05F3E84002FA2E
:10A2C00001F943EA04084FEA1C4206FA01FAB0FB1E
:10A2D000F2F71FFA8CF602FB17004FEA184444EA23
:10A2E000004407FB06F0A0420AD91CEB040407F166
:10A2F000FF3380F09C80A04240F29980023F64448A
:10A30000241A1FFA88F3B4FBF2F002FB104443EA6C
:10A31000044300FB06F69E4209D91CEB030300F13F
:10A32000FF3480F082809E427FD90238634440EA45
:10A330000740A0FB09749B1BA3423E46A04664D382
:10A3400061D0BEF1000F0AD0BAEB060263EB08033E
:10A3500003FA05F5CA401543CB40CEE9005300216E
:10A360003FE7730843EAC1734A08190C41EA024106
:10A370004FEAC67C9BB2B2FBF4F02646A0462746C5
:10A380001F2243EA0143B1FBF4F1A3EB080341EAC6
:10A39000004158E72946FFE6284615E71A46C3F16B
:10A3A00020019C4026FA01F320FA01F1904003437A
:10A3B000270C06FA02FCB1FBF7F0A6B207FB10155A
:10A3C000190C41EA054100FB06F58D423BD96118A5
:10A3D00001D28D4220D8491B0138B1FBF7F5019518
:10A3E00005FB06F8019D9BB207FB151143EA0143EB
:10A3F000434526D2E31805F1FF31C6D24345C4D206
:10A40000A91E2344C1E7BA459BD2B7EB090664EB0A
:10A410000C040138A04694E7651B29440238B1FBBF
:10A42000F7F5019505FB06F8DCE720467FE71F46B8
:10A4300066E70846F4E6A44402382FE7023D2344C9
:10A4400015E70199A1E7491BB1FBF7F5019505FB5C
:10A4500006F8C7E72DE9F0410D4606464FF0FFFA32
:10A46000294640F2175058F079FE06F108070446D5
:10A4700090B1436828469847A36801219B69054627
:10A48000984710B1294846F001FCA3683946284690
:10A490009B68BDE8F04118472549284657F098FFCA
:10A4A000044618B390F85030D906EBD443F01003AB
:10A4B00080F85030394653F0B2FE96F82A3003F057
:10A4C0000C03002B94F8513014BF0122002223F01A
:10A4D000060343EA420384F8513005D194F8503022
:10A4E00043F0020384F85030BDE8F081114928465A
:10A4F00057F06EFF0446B0B190F82A309A07C1D4E5
:10A5000043F00203394680F82A3053F02BFC96F8CA
:10A510002A1001F00C010039204618BF0121BDE8C6
:10A52000F04153F006BC0448ADE700BF184A0900EB
:10A53000F8C409005CC509000D4A09002DE9F7437C
:10A540000746002608466A4601A9019658F08AFB8C
:10A550000199022902D8234846F084FB7868012239
:10A5600089001DF04FFC7E6080463E81019BB4B2A5
:10A57000A34206D85B00C7F804803B8103B0BDE866
:10A58000F083009B184953F8245040F203522846A8
:10A5900025F0F6FD686840F20352022125F0AEFD79
:10A5A000A86840F2946125F019FE40F2946347F6E2
:10A5B000FF720E49814657F07AF8E86840F29A61D6
:10A5C00025F00CFE094940F29A6347F6FF720546F2
:10A5D00057F06DF828F8249008EB84040136658064
:10A5E000C4E700BFB4470900BC2809000080FFFF92
:10A5F0002DE9F04F2DED028B91468DB0C268BDF86C
:10A6000064B0DDF86880BDF86C701D9C06468A4613
:10A610001D46B0EE408A82B980F845204BEA070318
:10A620001F2B14D8BAF1000F40F08980002F00F0E2
:10A63000B28054464FF0040A13E043689A4200F097
:10A64000B380002380F845300FF0B6FBE6E7BAF19F
:10A65000000F40F09580002F00F0968054464FF098
:10A66000080AB9F1000F00F09C8040F20122ADF819
:10A670001820002D00F093806A1CADF81A200022EB
:10A68000079206A85FF0CBFD8146002851D1182221
:10A6900001460DEB020056F07EFEDFED457A9FEDA0
:10A6A000457A454B8DF818A028EE278A5D43C8EE01
:10A6B000077A42F210734F4508BFC846B5FBF3F561
:10A6C0004846189BADF82450012507948DF82D506D
:10A6D0000293ADF80CB0CDF81080ADF81470B6EE62
:10A6E000007A77EE877AFCEEE77ACDED087A4DF0C6
:10A6F00077FC8146E8B9314C06AA02A920465FF0F2
:10A7000068FD8146A8B92E49324606F128000AF0B4
:10A7100077FF9DF97020217828465FF08AFD8146F9
:10A7200038B9207829465FF056FD814608B9189B54
:10A73000F36048460DB0BDEC028BBDE8F08F3CB332
:10A74000F0EE0C7AB4EEE78AF1EE10FA6946204694
:10A7500010D807EE905A9FED1B7AF8EE677AF4EE68
:10A76000C77AF1EE10FA05D84DF0FEF86C464FF0BE
:10A77000020A76E74DF0F8F80C464FF0030A70E74E
:10A7800000244FF0060A6CE73C464FF00A0A68E7DF
:10A790004FF0010A65E73C464FF0050A61E72A469B
:10A7A0006BE7CDE906996CE74FF01109C1E700BFEF
:10A7B0000024744900401C4440420F0071050120F0
:10A7C000C58007006666A63F2DE9F84341609946BB
:10A7D0004B680B9F90469A790A9B80F82C20038542
:10A7E0008D7D044605F0300605F0060572B34B6812
:10A7F000D8684EF03DFCE0842DB10023C4E9028905
:10A80000C4E90433A361002384F82D3084F82A308E
:10A81000A384089BE361099B23621AB3EFB11B4930
:10A82000224638460AF0ECFE5DB115F0040118BF6F
:10A83000012160681ABF84F82B10002201220FF05A
:10A8400065FCDEB1B20616D4012315E04FF6FF73A6
:10A85000C3842B4635461E46CEE70C4821460AF0F7
:10A86000B3FEE1E767B10A49224638460AF0C8FE5E
:10A8700026B17307E8D4022384F82B30BDE8F883AF
:10A88000034821460AF0A0FEF2E700BFA38A0800B1
:10A890000D8B080037B504464FF6FF702361002387
:10A8A000A080A160E271A371E3608B88ADF80430F1
:10A8B000501C8B798DF80630221D01A9C0B25FF0C3
:10A8C000D6FC054678B9094AA18813888B4228BF6F
:10A8D0000B461380064A13888B4238BF0B46084646
:10A8E000138000F08BF8284603B030BD58050120D6
:10A8F000D46A01202DE9F04F89B081469DF8486067
:10A9000015465FFA81F81C46002B36D043681A7949
:10A910001B680621C3F800151D4B342101FB0233CF
:10A9200086F00106022283F82D207201194E4FF0A5
:10A93000000AB4F5806F274603A928BF4FF480674B
:10A940004846CDE9047ACDE9065A8DF80CA08DF879
:10A950000D80019200F0C2FDB042834603D1E41B9A
:10A96000019A3D44E5D1D9F8040035F02FFD584651
:10A9700009B0BDE8F04F45F06BBD41460FF0D6FE83
:10A98000A0420CBF6FF01200204609B0BDE8F08F66
:10A99000E06101200000AD0B074A002311688142ED
:10A9A00001D1184670470133082B02F10402F5D19A
:10A9B0004FF0FF30704700BFCC4601200C4B187899
:10A9C00001280DD10B4B1B78FF2B0BD10A4B1868BC
:10A9D000C20708D4C30308D4800C00F004007047F9
:10A9E0000228F3D17047052070470120FAE700BF25
:10A9F000446F01204C6F0120CC6601202DE9F0410D
:10AA0000094D0746884600244FF6FF7635F81400B6
:10AA1000B04203D0424639465FF02DFC4434B4F5D1
:10AA2000AA7FF3D1BDE8F08160090120034B53F800
:10AA3000203013B19A6801329A607047A420012037
:10AA400038B5144B53F82040ECB1207935F070F94B
:10AA50000546607935F06CF9A2790F49E37940EA4F
:10AA6000450000F0030040EA8202A0718A5C1344B2
:10AA700094F908205BB29342E37105DBE36801338C
:10AA8000E3600023E37138BD52429342FBDCE3688C
:10AA9000013BF5E7EC460120B4230A002DE9F04F15
:10AAA0000546A7B08A460146002058F057FB09AC7E
:10AAB000002841D1CDE913000CAA7E21284629F0B7
:10AAC0005DFEA94B0F9301224023CDE9102316AB65
:10AAD00012930FAB0E93A54B09940A9300260820FE
:10AAE000CDE9050656F027FB07902046CDE9036621
:10AAF0008DF8206055F0ACFFDFF880B23746354660
:10AB00009DF85490B9F1000F13D0204655F0A0FFE6
:10AB1000B9F15D0F00F092804AD8B9F13A0F3BD8F5
:10AB2000B9F11F0F14D8B9F10A0F31D8B9F1080FD4
:10AB3000E6D88F4846F0AAF80121284629F010F8F7
:10AB400043680A93002309950B938DF85430C5E7A9
:10AB5000A9F12002D2B20123934013EA0B0F40F077
:10AB60000F81844A1340CBD1B9F1220FE1D1069372
:10AB70009DF854100029DCD0222940F0A480204602
:10AB800055F066FFDDE906102CF0FAF981462CE05D
:10AB9000B9F10D0FB4D0CCE7B9F15B0FC9D10020EA
:10ABA00022F02AFE8146002D3AD04FF0010821E024
:10ABB000B9F1740F70D039D8B9F1660F4FD0B9F12F
:10ABC0006E0FB6D19DF85430752BB2D1204655F09A
:10ABD0003FFF6C28ADD1204655F03AFF6C28A8D134
:10ABE000204655F035FF4FF00E09002D00F00E8184
:10ABF0004FF00008604B9F4240F0F58049462846E0
:10AC000057F0FAFFB8F1000F3FF47AAF049B002B26
:10AC100040F0F780012101A82BF086FF049B1D6006
:10AC200048462BF099F84D46074669E7B9F17B0F86
:10AC300000F0D580B9F17D0F7FF47BAF002D3FF49C
:10AC400078AF039B002B00F00081013B049A039333
:10AC500052F8235028462BF07FF8074650E79DF81E
:10AC60005430612B7FF465AF204655F0F1FE6C281F
:10AC70007FF45FAF204655F0EBFE73287FF459AFA9
:10AC8000204655F0E5FE65287FF453AF204655F089
:10AC9000DFFE4FF01E09A8E79DF85430722B7FF4B9
:10ACA00048AF204655F0D4FE75287FF442AF2046C9
:10ACB00055F0CEFE65287FF43CAF204655F0C8FE27
:10ACC0004FF03E0991E75C290CD1204655F0C0FEBB
:10ACD0007528014606D86D2808D8622840D0662815
:10ACE00008BF0C2105A862F053FD35E0A0F16E030A
:10ACF000072BF7D801A252F823F000BF1DAD0200C8
:10AD0000E5AC0200E5AC0200E5AC020065AD020076
:10AD1000E5AC020021AD020025AD02000A21E1E709
:10AD20000921DFE74FF000084FF00409204655F0F5
:10AD30008FFE40F02000A0F130025738D2B2C0B2EE
:10AD4000092A88BF0246B9F1010942EA0818EDD183
:10AD5000414605A862F02EFD204655F079FE07E732
:10AD60000821BFE70D21BDE7CC5D0900030A0800FB
:10AD70000B35090001100004385D09000020FF03B5
:10AD8000002306939846494605A862F001FD9DF808
:10AD90005490B9F12E0F17D009F0DF03452B13D0D3
:10ADA000B9F12B0F12D0B9F12D0F0FD0484645F055
:10ADB000A5FE024650B9DDE90610B8F1000F09D032
:10ADC000134658F039F9E1E64FF00108204655F0F6
:10ADD0003FFED8E743460A222DF088FFD6E6002042
:10ADE0002BF074FFDEE62EB9B8F1000F7FF4A1AEB0
:10ADF0004E4685E631464A46284657F042FB002635
:10AE000000E7294601A857F0F7FE09E7BAF1000F5D
:10AE100011D0B9F1000F3FF48CAE039B002B7FF4EF
:10AE200088AE05A862F02BFD484627B0BDE8F08F3C
:10AE3000204655F00DFE9DF85450284645F072FE10
:10AE40000028F5D1002DE4D073E6A946BAF1000F31
:10AE5000F1D0E2E7C20713B5044603D5C0F34700BB
:10AE600002B010BD830707D102680E4B9A4203D18E
:10AE70002AF060FFC0B2F3E7204657F08AFE48B1DF
:10AE800020462AF0DFFEFCEEC07ACDED017A9DF877
:10AE90000400E5E720462AF05FFF5E22C1880248F1
:10AEA00045F0E8FE803209008C4009002DE9F04FA2
:10AEB0000546E3B058484FF0F2F8061E09DB574C40
:10AEC0006388B3F57F7F08D340F2512323803DF0A0
:10AED0000FFB002063B0BDE8F08F1A1DAA4200F2FC
:10AEE0009880591E251D4E486A5C2F2A4FF000029B
:10AEF0000CBF6A54EA5405A954F075FD494B074646
:10AF0000186010B11BF0E8F820B940F251332380EB
:10AF10003046DCE707F18000059A06A953F0FAFEF7
:10AF200040F2511345F8043C0023C4E901330746BD
:10AF3000E36010B103236370EAE71AAD294606A85F
:10AF400053F0D4FF08B9AB7E93B9002106A853F0A3
:10AF5000CDFF4FF00009A7604F450FD106A853F071
:10AF6000DAFB0023A26863806260E360A361CFE73D
:10AF7000294606A853F0BAFF0137E3E7294606A899
:10AF800053F0B4FF6B892989C4F8049003F01F02C1
:10AF90005200480A0192C3F344120092DB0A01F006
:10AFA0001F0200F2BC70C1F3431161F096FA1E4B10
:10AFB000A0FB0303C4E904032B7B13F0100318BFA9
:10AFC00001230DF1820B15BFE360E36000232B68C2
:10AFD000A361584660F0D0FB6080824630463DF069
:10AFE00087FA4FF00008C24502D809F10109B3E71A
:10AFF000AAEB0802042A4FF0000328BF04220BEB3F
:10B0000008010548009303920FF066F9039A9044F3
:10B01000E9E701205EE700BFD84F0120A0510120E1
:10B02000A45101209C50012000CA9A3BF8B5284B3E
:10B030001D68284B1B681A68012151641B68264A49
:10B04000D3F844650023146814B12179814230D0CB
:10B050000133082B02F10402F5D1F8BD6369A06940
:10B06000E289218AEB1A89B211FA82F2301AA18997
:10B07000B2FBF1F7C3EB034303444FF6FF7001FB50
:10B0800017228342A16828BF034621F81230238A81
:10B09000A2899BB2934203D2238A0133238214E014
:10B0A000E3899BB20133B3FBF2F102FB1133E3817D
:10B0B0000BE0E379002BD1D034F03AFE637900F055
:10B0C0000100834201D00023E3716561A661C4E7FA
:10B0D000BC66012078680120CC4601202DE9FF41A3
:10B0E00004460F464EF0BBFC6368DB6853F82750FC
:10B0F00040F21750294658F031F8064600285CD037
:10B10000436828469847B36801A95B68804698471A
:10B11000B36800219B68054640469847B368002104
:10B120009B694046984763682849DB6853F82700C5
:10B1300057F04EF9C0B190F85030B0F9382023F0F4
:10B14000100380F85030B0F93C309A421FBFADF880
:10B150000830C38F826BADF80A304FF000031ABF7E
:10B16000019201250025836263681949DB6853F861
:10B17000270057F02DF9064668B190F82A3023F0E1
:10B18000020301A980F82A3017F09AFE0021054633
:10B19000304652F0E7FD6DB194F82A30DB070ED44B
:10B1A000019BA361029BE36194F82A3043F0010301
:10B1B00084F82A3004B0BDE8F0810546B3E704F115
:10B1C000180201A9104651F051FFEDE7F8C409003B
:10B1D0005CC509002DE9F74F404B01900020187025
:10B1E0003F4BDFF820A1DFF820C1FF2002EB8109EF
:10B1F00018703C493C48144615464FF001084FF082
:10B20000FF32A94520D1013204D0019B002B51D13E
:10B2100014F05CFD354E364800220023C6E90023B9
:10B2200000231A46A5424BD15AB193ED017ADFEDC6
:10B23000317A67EE277A17EE900AFDF7B3FFC6E979
:10B24000000103B0BDE8F08F55F8047BBB07D8D1EF
:10B250003B685345D5D17B681A79A2F12003C2F12E
:10B26000200628FA06F608FA03F333433E7A08FA72
:10B2700002FEAEB1DCF804600096DCF8006046EA3D
:10B280000E0B009E1E43CCE900B67E7A002EB8D08D
:10B29000D1E9007647EA0E071E43C1E90076B0E720
:10B2A00046680096066846EA0E0B009E1E43C0E9FB
:10B2B00000B6EAE7104A00231360104A1370A9E7AA
:10B2C00021688F0708D10F68874205D112B10C4859
:10B2D00045F0DCFC0B4601220434A3E7446F012057
:10B2E0004C6F0120E00C0120D00C0120E80C012063
:10B2F000908D090000007A44CC660120F86E012090
:10B3000007480900AC8D0900C00C0120242B2DE951
:10B31000F047884601D8012B06D1FDF73DFF1623E3
:10B3200003600020BDE8F087344E0D46294615F82D
:10B33000014B375D17F00807F8D12D2C10D12C7870
:10B3400001278D1C33F0100115D1302C0DD1297837
:10B3500001F0DF01582908D16C78023510230AE08A
:10B360002B2C04BF2C788D1CECE7002BF6D1302C55
:10B3700014BF0A23082307F1004E0EF1FF3E0021FF
:10B38000BEFBF3F90E4603FB19EAA4F1300CBCF145
:10B39000090F10D86446A3421EDDB1F1FF3F07D06C
:10B3A000B14516D301D1A24513DB06FB03460121AB
:10B3B00015F8014BE9E7A4F1410CBCF1190F01D8D4
:10B3C000373CE8E7A4F1610CBCF1190F04D8573CF5
:10B3D000E1E74FF0FF31EBE74B1C05D1222303607F
:10B3E000764632B930469DE707B17642002AF9D059
:10B3F00009B105F1FF38C2F80080F3E7D97F0A00F0
:10B400002DE9F043344E86460D46284615F8014B8B
:10B41000375D17F00807F8D12D2C10D12C780127B3
:10B42000851C33F0100015D1302C0DD1287800F098
:10B43000DF00582808D16C78023510230AE02B2C45
:10B4400004BF2C78851CECE7002BF6D1302C14BF00
:10B450000A2308234FF0FF380026B8FBF3F803FB5C
:10B4600008F96FEA09093046A4F1300CBCF1090F64
:10B4700010D86446A3421EDDB6F1FF3F07D08045D9
:10B4800016D301D1A14513DB00FB0340012615F8BB
:10B49000014BE9E7A4F1410CBCF1190F01D8373C8D
:10B4A000E8E7A4F1610CBCF1190F04D8573CE1E7BF
:10B4B0004FF0FF36EBE7731C06D12223CEF80030A5
:10B4C000304632B9BDE8F08307B14042002AF9D0D6
:10B4D00006B1691E1160F5E7D97F0A002DE9F74F23
:10B4E00080460D46019260F03EFAD8F80430AC4F29
:10B4F00001225A72D8F804301E791C68342303FBE9
:10B500000677002387F82E30EB6803F06043B3F131
:10B51000005F81468B4607D0A248D8F8043000224D
:10B520005A7203B0BDE8F08F9F4BC4F8083397F808
:10B530002F3003F0FF0A23B1BB689C48C4F80433E2
:10B54000EBE787F82F20AE46BEE80F0007F10C0CA2
:10B55000ACE80F00DEF80030CCF8003087F830A0FF
:10B560006B78C4F888354FF4827120465DF0DFF8BF
:10B570004FF4927120465DF0DAF8C4F850A5C4F893
:10B5800040A52B78032B00F2B380DFE803F0729A1A
:10B5900052022B6903F06043B3F1005FBCD14FF45A
:10B5A0008073C4F800326B68EA68C4F844254FF42D
:10B5B000A871C4F8483520465DF0B9F84FF4B07171
:10B5C00020465DF0B4F84FF4A47120465DF0AFF86A
:10B5D00001232362A360D4F85031002BFBD04FF439
:10B5E000A87120465DF0A3F8AB682A69C4F8442529
:10B5F000C4F848356A4B342202FB06336C4A9A6021
:10B600004FF4827308226B4F2978654D03291CBFC4
:10B610000121A15034227243A918AA58002A79D0D6
:10B620008B68C4F80433634B9F4200F0A8806248E3
:10B6300073E76B68EA68C4F84425C4F848352B6999
:10B6400003F06042B2F1005F7FF466AFAA68C4F80D
:10B6500034354FF48453C4F83825C4F80032504BC5
:10B66000342202FB063340F202229A600123236255
:10B67000C6E701996B68EA68C4F84425C4F8483500
:10B680003422474B89B102FB06334FF48071C4F872
:10B690000012474A9A604FF4A47120465DF047F8C3
:10B6A0004FF4A47301222262ACE702FB06334FF48D
:10B6B000007140F20222C4F800129A604FF48273C3
:10B6C000F0E76B68EA68C4F83425C4F838354FF4FD
:10B6D0008053C4F80032324B342202FB063340F26E
:10B6E00002229A600123236200224FF482738AE7C8
:10B6F000314F4FF48273082286E7D4F8242152B1E7
:10B700004FF4927120465DF012F8012323626361C9
:10B710004FF4827323441A68002AEED03422D4F8FE
:10B72000C434C4F8C43402FB0651002281F82F202F
:10B730008BB1224A224813F0010F08BF104613F0C4
:10B74000020F02F5803218BF104613F0040F1D4B94
:10B7500018BF1846E1E6204648F090FF00287FF425
:10B7600062AF1648D9E660F0FEF8814574EB01013E
:10B7700009D2D8F80430144800225A72D1E619F5DB
:10B780007A794BF10004D8F804305A7A002AEAD1C9
:10B790009B7A042B96BF0D4A084852F82300C0E656
:10B7A000E06101200A00AD0B02029C010B00AD0B11
:10B7B000000204000000AD0B0400AD0B0100AD0B56
:10B7C0000000AE0B0200AE0B0700AD0BA0230A0079
:10B7D000F8B590F82A309B0704462DD4F8BDDB68F5
:10B7E00053F8256040F21750314657F0B7FC074632
:10B7F00068B1436830469847BB6804F108019B680C
:10B800009847013563689A689542E8D3E6E70B49A3
:10B81000304656F0DDFD20B104F1080152F0FFFC86
:10B82000EFE70749304656F0D3FD0028E9D004F190
:10B83000080152F097FAE4E70025E3E7F8C40900AD
:10B840005CC5090090F950301F4A10B5002B836A7F
:10B85000B4BF418A018AB0F90C40002B08BF1346DF
:10B860000C44997B8289B9B193F9051011FB02F15F
:10B870005A88114409B2A0F8461093F905205B8854
:10B8800012FB04331BB29942D2BFA0F84A30A0F891
:10B890004A10A0F8463010BD93F9041011FB02F1D4
:10B8A0001A88114409B2A0F8441093F904201B88A7
:10B8B00012FB04331BB29942D2BFA0F84830A0F863
:10B8C0004810A0F84430E6E75A05012090F95030BE
:10B8D0001F4A10B5002B836AB4BF018A418AB0F9B0
:10B8E0000E40002B08BF13460C44997BC289B9B1A6
:10B8F00093F9041011FB02F11A88114409B2A0F85F
:10B90000441093F904201B8812FB04331BB29942A4
:10B91000D2BFA0F84830A0F84810A0F8443010BDBD
:10B9200093F9051011FB02F15A88114409B2A0F8ED
:10B93000461093F905205B8812FB04331BB2994231
:10B94000D2BFA0F84A30A0F84A10A0F84630E6E787
:10B950005A05012008B510EE103A23F00042B2F16A
:10B960007E5FF0EE405A10D308D19FED2F0ADFED35
:10B970002F7A002BB8BFB0EE670A08BD70EE405AB0
:10B98000DFED297A87EEA50AF7E7B2F17C5F11D2E5
:10B99000B2F14A5F9FED266A42D920EE000AFCF719
:10B9A00041FEDFED247AE0EE657A75EEE75A36EE79
:10B9B000650AE2E7002BB7EE000AF6EE007A14DA29
:10B9C00075EE805A25EEA70AB1EEC06AFCF72AFE92
:10B9D000DFED197AE0EE067A9FED150A77EE867AAA
:10B9E00030EE670A30EE000AC7E730EE650A20EE57
:10B9F000270AB1EEC05AB0EE407A15EE103A6FF356
:10BA00000B0305EE903AA5EEE57A75EE257A87EE02
:10BA1000276AFCF707FEA0EE056A36EE250AE1E785
:10BA2000B0EE460AA9E700BF00000000DA0F494067
:10BA3000DA0FC93F6821A2336821A2B308B510EE1E
:10BA4000103A5A00F0EE407A0FD4B7EE007A70EE5A
:10BA5000477ABDE8084037EEA77AA7EEA77AB1EE9D
:10BA6000C70A37EE800A22F0C9B823F00043B3F1C9
:10BA70008B4F13D2FFEE006AE0EE006ABDE808408B
:10BA8000B1EEE67AF7EE006A37EE007A86EE870AC4
:10BA9000B0EE007A97EE870A22F05CB922F05AF9EC
:10BAA000DFED027A30EE270A08BD00BF1872313F81
:10BAB00030B589B0084611461A4602AB0193194BBE
:10BAC0000093032355F0C0FD1749029D0C2057F049
:10BAD00020F99DF80C30037245609DF81030044643
:10BAE000EBB128460DF064FD606805AA40F21151E3
:10BAF00028F044FE237A5B0043F0010305AA0021ED
:10BB00000120079355F0E9FE57F04FF805466068AD
:10BB10004EF03FF91DB9217A044845F0BFF82046A0
:10BB200009B030BD90260A0000CD09003249090055
:10BB300010B58EB003AB51F8044B0193194B009331
:10BB40000138032324F036FA40F23451606806AA23
:10BB500028F014FE237A5B0043F001030893039B53
:10BB6000099340F626130A93049B5B0043F00103FC
:10BB70000B93059B6FF0004293421FBF40F2E642D9
:10BB80005B000C9243F0010314BF0221012106AABD
:10BB90004FF0020018BF0D9355F09FFE0E200EB01F
:10BBA00010BD00BF78260A0010B58EB003AB51F867
:10BBB000044B0193194B00930138032324F0FAF945
:10BBC00040F29261606806AA28F0D8FD237A5B00F3
:10BBD00043F001030893039B099340F626130A934D
:10BBE000049B5B0043F001030B93059B6FF0004245
:10BBF00093421FBF40F2E6425B000C9243F0010308
:10BC000014BF0221012106AA4FF0020018BF0D93B4
:10BC100055F063FE0E200EB010BD00BF60260A0076
:10BC200010B596B003AB51F8044B01932D4B009324
:10BC30000138062324F0BEF909AA606840F2936136
:10BC400028F09CFD237A5B0043F001030B93039BD8
:10BC50000C93049B0D9344F6D6530E93059B5B0007
:10BC600043F001030F93069B6FF00042934235D0DF
:10BC70005B0043F0010344F6A6521193109209238E
:10BC8000032116AA02EB830244F2862042F8340C08
:10BC900016AA02EB8300079A520042F0010240F814
:10BCA000302C089A6FF00040824210D016A800EBAA
:10BCB000830044F2562440F82C4C16A800EB830372
:10BCC000520042F00102013143F8282CC9B209AAFE
:10BCD000032055F002FE0E2016B010BD07230221EE
:10BCE000CFE700BF30260A00F0B58BB008461146FA
:10BCF0001A4603AB01931B4B0093072355F0A4FC9A
:10BD0000DDE903600E2816D010F0030203D10168AC
:10BD1000154B99420CD02AF01FF8C38800931348A2
:10BD200040F2AF1340F2411240F2163144F0A2FF4C
:10BD300001214EF0C9FA0E49182056F0EAFF9DF88D
:10BD400020409DF824109DF81C50069F049A9DF8F1
:10BD500014300573C0E90167447381730261037590
:10BD60000BB0F0BDF8250A0034C6090001510900E6
:10BD7000E4CC090030B58BB004466A464068244DD7
:10BD800040F23C6128F0FAFC00216A46084655F072
:10BD9000A4FD56F00AFF002831D060686A4640F2E0
:10BDA000363128F0EBFC42F646530293A3685B0061
:10BDB00043F00103039345F256030493237B5B0096
:10BDC00043F00103059344F656730693637B5B00CF
:10BDD00043F00103079342F636621123CDE90823AD
:10BDE00004216A46002055F078FD23690E2B03D00C
:10BDF000217D58684EF054FA60680BB030BD04F0F5
:10BE00000FFFAB6A002BBFD0012027F0D1FFBBE7AB
:10BE1000BC6201202DE9F743054601F134000E46CE
:10BE200004F0C2FE2B88102B05D0112B5FD0002010
:10BE300003B0BDE8F083404C002388224FF6FF7129
:10BE400002FB03F7E05B884205D00133052BF7D1F5
:10BE50004FF408770423882101FB03F0B5F804C0F0
:10BE600024F800C022180E20D065002082F85A0065
:10BE7000A2F87600EA7B01FB0343022A14BF96F87E
:10BE800045200122DA704FF000084FF6FF7207F1EB
:10BE90000800A3F8582041465022204483F87880B7
:10BEA00004EB070983F8798055F075FA07F1600013
:10BEB0004A462044214909F0A3FBC6F818802869A6
:10BEC00069696C373C4403C468465EF0A4F9BDF868
:10BED00000302A8A9A4202D86A8A9A4203D2A888F3
:10BEE00069465EF080F90023F3600120A0E7AB888B
:10BEF000114F0024882202FB04F1785A984205D0A1
:10BF00000134052CF7D14FF40871042439440B484F
:10BF100009F08CFB88235C433A194FF6FF733B53BF
:10BF2000002382F85A30D26D0E2A1EBF5360297A40
:10BF30001172B361D9E700BF60090120F5FD03006C
:10BF40002DE9F0418AB0084611461A4605AB019327
:10BF5000234B0093052355F077FB0522059802A992
:10BF600027F0ACFD039EA6F11002102A03D81D4B4A
:10BF7000D340DB0702D41C4844F088FE069C022C08
:10BF800004DC002C04DC194844F024FE062CFAD111
:10BF90000798DDF80880A0B9074615494FF48A7064
:10BFA00056F0B7FE089B80F80C41C0F810313246BD
:10BFB0003B46414605464DF0A4FF28460AB0BDE881
:10BFC000F081012202A927F079FD0028E4D003982E
:10BFD00040F28512102124F091F8029FDDE700BFA6
:10BFE000B8260A00010101002F4A0900EE460900A7
:10BFF000A0CC090070B588B003AB51F8045B019385
:10C00000184B00930138022323F0D4FF0522039834
:10C0100005A927F053FD069CA4F11002102A03D8AD
:10C02000114BD340DB0702D4104844F02FFEDDE96A
:10C03000040640B903462846224631464DF061FFCA
:10C040000E2008B070BD012205A927F037FD002899
:10C05000F0D0069840F28512102124F04FF8059B8D
:10C06000E9E700BFA8260A00010101002F4A0900E4
:10C0700010B50446084656F079FA022804DC002878
:10C0800004DC044844F0A6FD0628FAD184F80C012B
:10C090000E2010BDEE4609001FB503AB01930F4BF8
:10C0A0000093054601230E46002023F083FF31460E
:10C0B000284646F0A1FF03982AF008FD441004D05A
:10C0C000074840F20D5144F08DFD294601203246CB
:10C0D000FFF780F80348214660F06DFF3C270A0017
:10C0E000DF51090018270A0070B505460E460028E2
:10C0F00044D046F081FF324629460020FFF76AF817
:10C1000000F0A4F900231A4642F07AF81C4B9C6A0E
:10C1100094BB4DF015FF78B3FEF750FC012818D002
:10C1200002280BD1174A234656F82340A10702D113
:10C130002168914203D001339D42F5D10E2420465F
:10C140003CF0D8FD00F060F820463CF0D3FD2046DE
:10C1500070BD0D4B0D491A78234656F82340A007B1
:10C1600006D12068884203D1606800799042E6D009
:10C1700001339D42F1D1E1E70E24E3E70E24E6E727
:10C18000BC620120908D09004C6F0120AC8D09002C
:10C1900010B586B0084611461A4602AB0193114B02
:10C1A0000093042355F050FA40F2F941029861F0EF
:10C1B000DDF80D4904460C2056F0ABFD9DF810202B
:10C1C00012B10A4844F062FD22792F2A01D95DF0AC
:10C1D0002DFA9DF814209DF80C10017244604272F3
:10C1E00006B010BDF8260A00AC8D0900834D090089
:10C1F00010B5044C23781BB913F068FD012323709C
:10C2000010BD00BFF86E0120F8B5344C344A2368E5
:10C210006FF3172393421CD04FF4807200213148F2
:10C2200055F0B9F8304A00231370304A4FF44031CA
:10C2300013701A0102F180420133082BC2F804196D
:10C24000F7D14FF080434FF47C12C3F88429244B7C
:10C250002360274E274D0024D5E90001D6E900329E
:10C26000C4F1200703430A430120A4F1200100FA8E
:10C2700001F120FA07F73943A04003400A40134375
:10C2800008D0E0B23AF05EF9204633F067FE20466F
:10C2900033F052FF0134402CDED1174917480022F9
:10C2A0000023C6E90023C5E90023C1E900234FF4B8
:10C2B0000033C0F84833D0F80423920308D5C0F8FF
:10C2C0000833D0F844311BB14FF4A2715CF02FFA5F
:10C2D0000B4B00200021C3E90001F8BD486F01208D
:10C2E000AF0000AD4D6F0120446F01204C6F012065
:10C2F000C00C0120D00C0120E00C012000400240C5
:10C30000E80C0120F0B50E4687B000251446002A3F
:10C310005ED08A075FD10A68414B9A425BD16A4678
:10C320004FF4807057F057F810B93E4844F052FC73
:10C33000DDE90035042CA5EB030536D0A30732D187
:10C340002368394A934208D0384A934205D0384A84
:10C35000934202D0374A934225D1052203A92046B1
:10C3600027F0ACFB049BAB4202D0334844F08EFC78
:10C370009DF81410039C0022402023F05FFF012849
:10C3800001D02E48F2E7009B5A19B2F5807F07D8FA
:10C390002B482A462146184454F0BCFF0E2417E0CF
:10C3A000284844F041FC2848C0E7284654F0C3FE22
:10C3B000009B5A19B2F5807F044604D820492A46CA
:10C3C000194454F0A7FF214628462AF02FFC0446C2
:10C3D000204607B0F0BD3246006800234FF480715C
:10C3E00027F08AFB042C064600F1010708D1B7F5B7
:10C3F000807F9CBF124B1D5C6D0045F00104E7E798
:10C40000204656F0B3F84223FF220021044655F09F
:10C410004EF9B7F5807FC3D8094B9C55BEE700BFE6
:10C420001C5C0900A237090090650900CC5D090079
:10C43000EC5C0900986109009C460900144F090052
:10C440004D6F012063440900C941090038B5084B0C
:10C45000D3E9004554EA050305D05FF084FA201AB9
:10C4600065EB010138BD4FF0FF300146FAE700BF30
:10C47000E80C012010B52DED028B88B0084611465E
:10C480001A4603AB01932E4B0093022355F0DCF8C0
:10C49000DDE90304B0F10E0218BF0122B4F10E036E
:10C4A00018BF01239A4202D1264844F0EFFB0E2820
:10C4B00038D029F0C7FBB0EE408A5FF054FAFBF7A2
:10C4C00089F8DFED217A07EE100A0E2CC7EE278AD5
:10C4D00021D040F2AA31049823F080FE04463AF0BD
:10C4E0009DFF05A93FF0B2F89DF81A3001939DF821
:10C4F000193000939DF817209DF818309DF81610FC
:10C50000BDF8140042F082FE231A08EE103AB8EE8D
:10C51000C88A38EE288AB4EEE88AF1EE10FA04D51B
:10C520000A48C2E79FED0A8AC7E70A49082056F081
:10C53000F0FB80ED018A08B0BDEC028B10BD00BF9E
:10C54000E8260A003D46090000007A4465450900D6
:10C5500000000000908D09001FB5084611461A46DC
:10C5600003AB0193084B0093012355F06DF840F2A3
:10C57000F941039860F0FAFE0449082056F0C9FB1F
:10C58000002044F027FB00BFE0260A00748D09005C
:10C5900010B5094B094C1B6823B1A34202D00848CF
:10C5A00044F042FBC0220021064854F0F4FE054B43
:10C5B00043F8044C181F10BDC0550120F06309005A
:10C5C00033450900C455012010B5084C20681EF001
:10C5D00019FF014610B1064844F026FBB422201D85
:10C5E00054F0D9FE034B2360204610BD080C0120F7
:10C5F0002C450900F063090038B51C460846114671
:10C600004FF0021223F09EFC206840F2F94160F0E6
:10C61000ADFE09490446082056F07BFB63790546C8
:10C620000BB95DF003F8207933F020FB20790CF092
:10C6300035FD6C60284638BD1CCC090008B5406843
:10C640004DF0DEF9BDE808409FED010A2AF0A8BBD5
:10C650003333534070B5064640683C4D4DF0D0F939
:10C660003B4A002303212B80C2F8F0150121C2F8B8
:10C67000F435C2F8001519461A0102F1804202F59C
:10C68000E0420133082BC2F81415C2F81015F3D19B
:10C690002F4C4FF49053C4F81835736801265B791A
:10C6A000C4F814354FF48071C4F810352046C4F82E
:10C6B0002C56C4F830665CF03AF84FF4827120468C
:10C6C0005CF035F84FF4847120465CF030F84FF49C
:10C6D000867120465CF02BF84FF48A7120465CF09E
:10C6E00026F82660D4F80031002BFBD018484FF410
:10C6F00080715CF01CF801236360154CD4F80431A0
:10C70000002BFBD012484FF482715CF010F801232B
:10C71000A360D4F81431002BFBD00D484FF48A717C
:10C720005CF005F80023C4F80035C4F81435C4F8EB
:10C7300010352B881BB223EAE373181340EA8300F9
:10C7400080B2400040F0010070BD00BFD068012001
:10C75000007000401C4608B5084611464FF0021212
:10C7600023F0F0FB40F2F941206860F0FFFD04493E
:10C77000042056F0CEFA0348F12144F033FA00BF0A
:10C7800000CC0900DF5109002DE9F04F2DED088B99
:10C790008FB009AB01936D4B0093052323F00AFC86
:10C7A0000021099830F02EFF002180460A9830F0D1
:10C7B00029FF044600210B9830F024FFE379012B78
:10C7C00005460AD1C379012B07D1A268012A04D9F1
:10C7D0008368012B01D99A4202D05D4844F056FA91
:10C7E0006621D8F808005BF085FEE6692779059098
:10C7F000394630465BF00DFEA368A069013B00FBA3
:10C8000003603946B0EE40AA5BF003FE0C98EE6977
:10C810000E28F0EE40AA28D1297930465BF0F9FDC8
:10C820000D980E28F0EE408A22D1A868AB692979CC
:10C83000013803FB00605BF0ECFDEB690493D8F872
:10C840001C300293059BD4F81CB0DB690393B0EE57
:10C85000409A4FF00009D8F808304B450BD805989E
:10C860000FB0BDEC088BBDE8F08F29F0EBF9D7E7EE
:10C8700029F0E8F9E1E7029898F804105BF0C9FDA7
:10C88000029AD8F81830B4EEC0AA1A44F1EE10FAA1
:10C89000B0EE408A029252DCF4EEC0AAF1EE10FA39
:10C8A00050D4A668D4F818A02179013E0027F31BC4
:10C8B000012B32D80AFB07B006915BF0AAFD06995E
:10C8C00006FB0AB0F0EE40BA5BF0A3FDAB69049A38
:10C8D0002979079103FB0720F0EE409A06935BF05D
:10C8E00098FD049A069B079906FB0320B0EE40BA18
:10C8F0005BF08FFD38EE6B8A30EE4B0A79EEEB9AE7
:10C9000028EE008A88EE290A30EE0B0A039BA3EC7E
:10C91000010A039309F101099DE707EB530303FBA8
:10C920000AB0079106935BF074FD069B0799B4EE7D
:10C93000C80AF1EE10FAB4BF1F461E46B7E7B0EEC4
:10C94000680AE3E7B0EE490AE0E700BFF86C0A00C6
:10C95000163B09002DE9F04F2DED048B87B003AB9A
:10C960000193504B0093032323F024FB03980021F1
:10C9700030F048FE8368012B044640F28C80C67973
:10C98000012E02D0484844F081F9007930F0BEFE13
:10C9900081460498E5690E2857D0002130F032FE18
:10C9A000C779012F834603D1A26883689A4201D0D8
:10C9B0003E48E8E700799FED3E8A30F0A7FE8246C8
:10C9C0002846DBF81C80C847A3694046EE18F0EE05
:10C9D000408AD047DBF81830B0EE409A9844A568FA
:10C9E000BD4211D86B1E00EE103AF6EE007A28EE2A
:10C9F000278AB8EE400A20EE080A07B0BDEC048B87
:10CA0000BDE8F04F2AF0CCB93046C847A36940468C
:10CA1000F0EE409A1E44D04778EEA98A30EE499A4B
:10CA2000F0EE486AD9EE286ADBF8183007EE907A03
:10CA3000B8EE677A9844C6EE877A0137B0EE409A2E
:10CA400038EE278AF0EE698AC9E705989FED188AC3
:10CA500029F0F8F82846B0EE409AC847A568F0EEED
:10CA6000408AB54202D828EE098ABBE732462179CE
:10CA7000E0695BF095FC07EE906A78EE808AB8EE8C
:10CA8000677A78EEC88A0136C8EE877AF0EE408A77
:10CA900038EE278AE5E7074807B0BDEC048BBDE810
:10CAA000F08F00BFE06C0A00713409007B3409008C
:10CAB00000000000020080801E280CD03E280AD012
:10CAC00010F0010307D1820707D10068044BC31A95
:10CAD000584258417047012070471846704700BFC0
:10CAE00080320900F0B51B288DB006460C4615466D
:10CAF00072D03CD80E2800F09C8004D8042840F264
:10CB0000B580002430E01028FBD115F0010206D1D9
:10CB100015F00303F5D12968704A9142F1D12846F6
:10CB200055F024FD0122054609A9204600F024F90C
:10CB3000102E0A9F3DD121790022402023F07EFB58
:10CB4000A3686B4300FB03F1E06854F015FBA36896
:10CB5000E0606B43A360636803F0FF0363601DB193
:10CB6000013DC319002F34D120460DB0F0BD1D2862
:10CB7000CBD02428C5D1012203A9284626F09EFF48
:10CB8000002860D0A10712D12268554B9A420ED1DD
:10CB9000012209A9204600F0EFF801230093DDE906
:10CBA0000901DDE9032353F0D5F800285CD11E24E8
:10CBB000DAE7A1689DF82C00694300F035F9C368F5
:10CBC0000446CFE7184609993A4654F0A3FB013DC5
:10CBD000C319002DF6D1C7E70A68424B9A4290D09C
:10CBE00009A90122204600F0C7F806A90522284617
:10CBF00026F064FF9DF82C100022402023F01EFB3D
:10CC0000A168079DB5FBF0F5064629449DF82C0068
:10CC100000F00AF90446DDE90912C06854F07AFB15
:10CC2000E0680A9B069905FB06F2184454F072FB73
:10CC30009AE70A682B4B9A423FF463AF2946204695
:10CC40004BF0BEFB90E7EA0702D5002043F0C2FF9D
:10CC5000AB0703D12A68214B9A42F6D0284655F0FB
:10CC600098FF0028A3D0F0E73E247DE7012209A920
:10CC7000204600F081F8012206A9284626F01EFF72
:10CC8000002894D00B9A012A21D05A2A21DC203284
:10CC90000146089B012B1ED05A2B01DC2033014694
:10CCA0009342D2D123F00203642BCED0022E01D0C6
:10CCB0000029CAD0079B0093DDE90912069B304684
:10CCC00056F0FBFA002814BF3E241E244CE74222F3
:10CCD000DDE70021DDE74223E0E700BF8032090005
:10CCE000CC5D0900EC5C0900F0B5012885B0074671
:10CCF0000E4608D08B0727D10B681C4A934202D0FE
:10CD00001B4A934220D1012201A9304626F0D6FECB
:10CD1000D0B139460022402023F090FA029BB3FBA9
:10CD2000F0F100FB01F5AB4202D0124843F0AEFF38
:10CD3000384600F079F8019904462A46C06854F054
:10CD4000E9FA204605B0F0BD304629F0CFFE58B1D3
:10CD500045102946384600F067F82B463A463146DA
:10CD600004464BF073FBECE70546F2E798610900D7
:10CD7000CC5D0900DB40090070B50D460179044621
:10CD800001F07F0116464020002223F057FAE368A5
:10CD90002B60A26842436A60227902F07F02AA6097
:10CDA0002168094A91420BD194F90420002A01DB41
:10CDB000B20707D46268C2F3172200FB02332B606C
:10CDC000002070BD0120FCE7EC5C0900074BC1E9C5
:10CDD00000300023C1E90233054B02689A4202BFCA
:10CDE0004368C3F317238B60084670470066090049
:10CDF000EC5C090038B50D461C4611462846094A28
:10CE000023F0A0F820682BF0A7F8012D007804D1BA
:10CE1000BDE83840002100F007B86168BDE838403F
:10CE2000FFF762BF040002007828F8B505460E46F9
:10CE300002D10F4843F02AFF00220146402023F090
:10CE4000FDF90C4B0C490746012D18BF194610205F
:10CE500055F05FFF0571436803F0FF030446C0E926
:10CE6000013606FB07F054F084F9E0602046F8BD77
:10CE70004341090090650900CC5D090070B50A794D
:10CE8000012A05460C460DD1184956F04BF9D4E954
:10CE9000022128462CF02EFE28461549BDE8704098
:10CEA00056F040B9134956F04CF9A368002BF3D063
:10CEB0001149284656F036F90026A368B34204D833
:10CEC0000E49284656F02EF9E6E71EB10C492846D1
:10CED00056F028F93246E168207923F087FA0122DA
:10CEE000014628462AF0B8F90136E6E76CE1080069
:10CEF000F521090078E1080083E108000D20090010
:10CF00002C2309002DE9F04F044687B00D46164644
:10CF10000AB90025D0E011F003078068DFF82CA2E1
:10CF200040F0DF800B68814A934240F0DA806A4625
:10CF300056F051FA10B97E4843F04CFE2179042E88
:10CF400001F07F013A464FF0400000F0968023F058
:10CF500075F916F00302054655D131688B7B002B1D
:10CF600042D001EB83031869724B98423CD131796E
:10CF7000402001F07F0123F061F9A84202D06E4801
:10CF800043F084FE33685345D6E9028B38D1736889
:10CF9000C3F3172905FB09F9DDE900062368E768F3
:10CFA000361A5345A8EB06062FD194F90430002B0E
:10CFB000AFDA002EE3D16368C3F3172305FB0377D1
:10CFC00005FB08F20BEB090105FB007054F0CDF9ED
:10CFD0000199A268009B521A08EB03006A4305FB03
:10CFE000017105FB007039E0544B99420BD1012DC2
:10CFF000C5D1052203A9304626F060FDDDE903B85E
:10D000004FF00009C8E74E4896E7002ED8DD636868
:10D01000B6EB132F2FD9A16831446943384654F039
:10D02000ABF86368E06066F31F2382466360BB452C
:10D0300008BF83460098A268019940443244121AFE
:10D040006A4301FB05A105FB00A054F08EF900988E
:10D0500005FB08F20BEB090100FB05A054F085F974
:10D060006368C6EB132262F31F236360A368334433
:10D07000A3600E2520E0BA46DCE723F0DFF8216844
:10D08000009B514506461BD1B3F1807F03DB2D4940
:10D090002D485FF090FF102055F03BFE054694E8C8
:10D0A0000F0085E80F00009A02EB112363F31F21A4
:10D0B0006960019B9B1AAB60284607B0BDE8F08F02
:10D0C00001992079C91AFFF7AFFEDDE90032E16866
:10D0D000D21A0546724306FB0311C06854F01AF9D0
:10D0E000EAE700232A460146206826F005FD23686A
:10D0F0005345024620790ED16368042E02EB1322B9
:10D100000BD003067FF505AFE168334600F07F00E2
:10D1100023F064FCADE7042EF6D1E16800F07F0057
:10D1200007B0BDE8F04F23F061B900BF1C5C0900F7
:10D13000A237090005CF0200273A090098610900CB
:10D14000C941090071390900F0570900EC5C090078
:10D1500010EE102A08B522F00043B3F17E5FB0EE66
:10D16000406A12D319BF76EE467A9FED1F7ADFED43
:10D170001F7A9FED1F7A12BF87EE276AE0EE077ACB
:10D18000B0EE676AB0EE460A08BDB3F17C5F0BD221
:10D19000A3F50003B3F1645FF4D320EE000AFBF7BC
:10D1A00041FAA0EE066AEDE7B0EEC06AB7EE000AFB
:10D1B00030EE460AF6EE007A20EE270AB1EEC06A9B
:10D1C000FBF730FA002ADFED0B7AA0EE066AB0EE2C
:10D1D000007AE6EE077A9FED066A36EE676AB8BF18
:10D1E000B1EE466ACEE700BF0000000000008003F9
:10D1F000DA0FC93F6821A2B31FB58DED010A019B6B
:10D2000023F00042B2F18B4F00EE102A4FEAD370A8
:10D210000AD320F09FFDDFED1E7A30EE270A08B119
:10D22000B1EE400A05B000BD5B0014D5B7EE007A40
:10D23000F0EE476AE0EE006AF1EEE67A77EE807A89
:10D24000C7EE276AF0EE007AE0EE276AB0EE660AD3
:10D2500020F080FDE3E7B2F1665F10D320EE007AA4
:10D26000F7EE006A37EE266AF1EEC67A77EEA67A16
:10D27000C7EE276A36EE800A20F0C0FCCFE7DFED6C
:10D28000057A70EE277ACDED037A039BC7E700BFDE
:10D290001872313F0000807B08B5044B1A68044BBC
:10D2A0009A4202D00D2039F037F908BD009C0320C6
:10D2B000EF2978011FB5044690B10E2810D00079EF
:10D2C0004DF094FA60B94FF4FF73039301A920461F
:10D2D00003AB02AA1BF04CF90399024843F0DEFCB1
:10D2E00004B010BDA2510900F4EE400AF1EE10FAAC
:10D2F00010B5F0EE407A04D770EE207AB0EE670AEF
:10D3000010BD10EE902AB2F17E5F03D1BDE810404F
:10D3100000F082B810EE103A940F04F0020444EAD0
:10D32000D37433F0004308D1022C59D09FED317AE9
:10D33000032C08BFF0EE477AE0E732F0004209D153
:10D34000DFED2D7A9FED2D7A14F0010F08BFF0EE7E
:10D35000477AD3E7B2F1FF4F10D1B3F1FF4F04F199
:10D36000FF3407D1022C3ED8254B03EB8403D3EDC9
:10D37000007AC3E7022C39D8224BF6E702F150615C
:10D380009942DDD3B3F1FF4FDAD0A10703D503F102
:10D39000506393420CD387EEA00AB0EEC00A00F0AF
:10D3A0003BF8012CF0EE407A04D1F1EE407AA5E78B
:10D3B000DFED157A022C0AD0002C9FD09FED137A56
:10D3C00077EE877A9FED127A77EEC77A96E79FED30
:10D3D0000F7A77EE877A9FED0E7A77EE677A8DE790
:10D3E000DFED0B7A8AE7DFED0B7A87E7DFED067A70
:10D3F00084E700BFDB0F49C0DB0FC9BFDB0FC93FAC
:10D4000098670A008C670A00000000002EBDBB333D
:10D41000DB0F4940DB0F493F10EE102A22F000439A
:10D42000B3F1994F82B04FEAD2700ED3B4EE400AF6
:10D43000F1EE10FA07D69FED410ADFED417A0028A0
:10D4400018BFB0EE670A02B070473E498B420BD856
:10D45000B3F1665F5AD212F0FF4FF4D160EE007A5A
:10D46000CDED017A019BEEE7374A9342F0EEC07AA8
:10D4700037D8A2F5D002934229D8F0EE006ABFEE69
:10D48000007AA7EEA67A002377EEA67A87EE270A1F
:10D490005A1C60EE006A9FED2D6ADFED2D7ADFEDFC
:10D4A0002D5A26EEA67AE7EE067A9FED2B6AA7EEB6
:10D4B000876ADFED2A7AE7EE257A67EE877AE6EE6D
:10D4C000267A67EE807A24D130EE670ABBE7B7EEA2
:10D4D000007A77EEC76A77EE877A012386EEA70A8D
:10D4E000D6E71F4A93420BD8F7EE086AB7EE007AE8
:10D4F000A7EEA67A022337EEE66A86EE070AC7E7AA
:10D50000BFEE007A87EE270A0323C1E74FF0FF330F
:10D51000BEE7144A144902EB830201EB830393ED47
:10D52000007A77EEC77A37EEC00AD2ED007A37EE8E
:10D53000C00A002887D0B1EE400A84E7DA0FC93F5D
:10D54000DA0FC9BFFFFFDF3EFFFF973F25AC7C3DF1
:10D550000DF5113E4712DABDA9AAAA3E98CA4CBEE3
:10D56000FFFF1B40B4670A00A4670A002DE9F84FCB
:10D57000D1F800800128064640468CBF01F1040B1B
:10D580004FF0000B0F46914629F0E0F930B94046C4
:10D5900028F0E2FBC188274843F06CFB06F1FF3A14
:10D5A000B9F1000F2DD0D9F80050C5F3DC051AEB06
:10D5B000050404D02C44A00053F0BDFD0446002215
:10D5C000924520D804EB86000022954221D11A4EC4
:10D5D000DFF868903168D9F800000131090153F093
:10D5E000CBFD3368C9F800005A1C32601A0100EB09
:10D5F000031340F802A0C3E90158DC603868BDE8B5
:10D60000F88F4D46D3E75BF8223044F822300132E0
:10D61000D6E7D9F80830083053F8323040F80C3CDF
:10D62000D9F8083003EBC20301325B6840F8083CCC
:10D63000CBE700BF84500900C0500120B850012042
:10D64000F0B50023DFF838E00C4E19460E27DEF85F
:10D650000020934201D30E20F0BD346804EB031286
:10D660004FEA031C9568854208BF44F80C1003F18B
:10D67000010304BFC2E90117D160E8E7B8500120F7
:10D68000C050012038B590F82330FF2B044629D034
:10D69000154B01225A600022C3F8002590F826306D
:10D6A0009B0707D590F8210032F0E0FA94F82200A9
:10D6B00032F0DCFAFF2594F8210038F043FF94F8AB
:10D6C000220084F8215038F03DFF94F8230084F8BC
:10D6D000225038F037FF054B84F8235000221A609F
:10D6E0003EF09EFD0E2038BD00500240E05E01205D
:10D6F0002DE9F04788B0084611461A4602AB01935F
:10D70000434B0093062353F09FFF9DF81C70029833
:10D710004FF437710FB345F04DFC40F2866105467A
:10D72000039845F047FC40F25131044604985FF0FD
:10D730001DFE40F27741824605985FF01FFE354995
:10D740008046282055F0ECFA0646B8F1000F0DD0BF
:10D75000314840F2774143F045FA5FF007FE40F26E
:10D760008661054603985FF001FEDCE72B4BD3F89A
:10D770000080B8F1000F02D0294843F055FA186034
:10D7800028799DF818900BF089FC20790BF086FC25
:10D790009AF804000BF082FC96F8263067F34103F8
:10D7A00086F826301F4B2A7986F82120C3F8642595
:10D7B000227986F82220C3F868259AF8042086F892
:10D7C0002320C3F8702507B32879414632F05EFA6A
:10D7D0002079414632F05AFA0122124B0121C3F856
:10D7E00004254F400022C3F80825C3F80C15C3F8E0
:10D7F0001075C3F81C15C3F82025C3F824953EF016
:10D8000029FD304608B0BDE8F0873A46E5E700BF9D
:10D810002C280A00D0CB0900DF510900E05E01206E
:10D82000754C09000050024010B5044690F82300E2
:10D830004CF0E0F80A4AD2F8083143B194F82630A7
:10D8400023F0040384F826300023C2F8083194F84A
:10D85000263013F0040F0CBF1E203E2010BD00BF69
:10D860000050024010B5044690F823004CF0C2F876
:10D870000C4AD2F8083143B194F8263023F004035F
:10D8800084F826300023C2F8083194F826305A076D
:10D8900001D400F009F843F0200384F826300E206C
:10D8A00010BD00BF0050024008B5014843F0BCF96C
:10D8B000834809002DE9F04F0D4685B055F8044B1B
:10D8C000064694F8230017464CF094F802AB0193F7
:10D8D0006D4B00933A4602232946701E22F06AFBE4
:10D8E0006A4A029DD2F808319DF80C6043B194F861
:10D8F000263023F0040384F826300023C2F80831D0
:10D9000094F8263059070BD5604A0123536094F8E8
:10D91000263043F0080384F826302023C2F8083369
:10D92000294640F216502BF041FC94F826306560F1
:10D9300066F3861384F826302A7B6968534FD20831
:10D9400084F82520AB7BE87B6D7B84F82450003B7A
:10D9500018BF0123DB0143EA0023E08C013A03F402
:10D96000C07320F4C07018BF01220343E384C7F8DA
:10D970001C2594F824305A1E53425341C7F82835C9
:10D9800094F8263013F002033DD00B4694F825009E
:10D99000638394F824304843584300014FF47A736A
:10D9A000B0FBF3F0033020F0030080B2208353F08B
:10D9B000E0FBA060208B53F0DCFBE06060684BF084
:10D9C00039F80023C4E9043384F8203094F8263071
:10D9D00023F03C0343F00403204684F826301CF077
:10D9E0004FFB228B294B9208C3F850252022C3F805
:10D9F00004230122C3F800251A601CF023FB0E202B
:10DA000005B0BDE8F08F2248DFF88C90B7EE007AC1
:10DA10009E4698461E46D7F81C25012A01D18279D8
:10DA20003AB307EE901A1B4AD0F800B0B0F904C020
:10DA300099FBFCFCF8EE676A02F1580A55689CFBFA
:10DA4000F5F507EE905AF8EEE77A76EEE77AF0EE23
:10DA5000E77A87EEA66AB4EEC76AF1EE10FA05D54A
:10DA6000D2F800E0B0EE467A2B46D846083292450E
:10DA7000E4D10136092E00F10800CCD1034AC2F8E6
:10DA80001885C2F814E581E71C280A0000500240FE
:10DA9000D4270A007C270A000048E80110B5044694
:10DAA00090F823004BF0A6FF064A0123536094F838
:10DAB000263043F0080384F826302023C2F80833C8
:10DAC0000E2010BD0050024038B5084B1B680022E4
:10DAD0000446C3F80025FF25007938F033FD60794E
:10DAE000257138F02FFD65710E2038BD44020120EC
:10DAF0002DE9F0432DED028B8BB0084611461A46F6
:10DB000003AB01933E4B0093072353F09DFD40F27E
:10DB10001D3103985FF02AFC4FF4557107460498B5
:10DB20005FF024FC9DF818506A07064604D040F2C6
:10DB3000DD21344843F0B2F89DF820305B0702D075
:10DB400040F2E241F5E70998DDF814809DF81C9059
:10DB500010B328F077F8B0EE408A40F2EB52012182
:10DB60000020B0EE480A53F084FD2749082055F004
:10DB7000D7F8044638790BF091FA30790BF08EFA29
:10DB800084F806903A79227133796371B8F57A5F37
:10DB900005D01E4843F07AF89FED1D8ADDE7102D71
:10DBA00001D01C48F6E71C4BDFED1C7A1B681C49B2
:10DBB000C3F840256279C3F8442528EE278A4FF040
:10DBC0000462C3F804250022C3F82025FCEEC87ABD
:10DBD0002822C3F81825C3F81C250122C3F8002504
:10DBE00017EE900AC3F86015C3F864251A6026F092
:10DBF00021F820460BB0BDEC028BBDE8F08300BFDE
:10DC000044270A000E510900B4CB0900B7370900B8
:10DC1000AE47E13DCE3709004402012000007A44BE
:10DC2000845601202DE9FF411446074600790D4630
:10DC30004BF0DAFE4FF48C61204622F0CFFA4FF41D
:10DC40008C620021044653F03EFDAB0706D12A68E2
:10DC50002D4B9A4202D12D4842F0BCFF062201A969
:10DC6000284625F02BFF9DF80C10029D0022402035
:10DC700022F0E4FAB5FBF0F5A54202D2244843F0C5
:10DC800005F8039B482B01D02248F8E7DFF8908085
:10DC9000019DD8F800300122C3F80825C3F860556B
:10DCA000C3F864451C4B4FF4485043F001039847B8
:10DCB000D8F800300022C3F80821184AC3F86025BC
:10DCC00001222E46C3F86425D8F80030D3F8083175
:10DCD0006BB105EB4405B5420CD1BB7983B124F09F
:10DCE0000104640044F0010004B0BDE8F08102F0DA
:10DCF00097FFE9E73388A3F5004326F8023BEAE7FC
:10DD000024F00304EDE700BFDC190A00BA4D090056
:10DD10008B4C0900533E090080280A0084560120DC
:10DD20004402012070B58AB0084611461A4606AB77
:10DD30000193264B0093042353F086FC069805229A
:10DD400003A925F0BBFE059C622C0ED0682C0FD0D9
:10DD5000482C1FD0422C01D1002507E0012C1BD0FC
:10DD60001B484FF43F7142F099FF0125012401E067
:10DD7000012502249DF8243083B9079B049A63434C
:10DD80005B00B2FBF3F103FB11223AB111484FF4EF
:10DD90003F71E8E70025ECE70025EBE70E49182086
:10DDA00054F0B7FFE4009DF824309DF81C10089A49
:10DDB000039E0473049CC37300230661857384600F
:10DDC0004173426003750AB070BD00BF5C280A0051
:10DDD00027510900F649090094CB09002DE9F041CB
:10DDE0001C460D4692B011462846824A22F0AAF8F7
:10DDF0002668814B3340062B05D0B10710D132681D
:10DE00007E4B9A4208D145F2F62231467C4853F0C7
:10DE10005AFD8207064603D132687A4B9A4202D0F5
:10DE2000794842F01FFF012D14D9062208A9606825
:10DE300025F044FE4FF43F730998089F4FF4806229
:10DE4000082122F07BF94307054605D06F480821D9
:10DE500042F024FF00252F466D49402054F059FF21
:10DE6000044606630022002306F1080050F05CFC23
:10DE7000206B10226B460DEB0201083050F085FF3D
:10DE800010B1052042F0BAFE009B102B0BD1614966
:10DE9000042204A853F02AFA28B95F49082206A8E8
:10DEA00053F024FA18B140F2C53022F075F8206B17
:10DEB00004226B460DEB0201083050F066FF00288B
:10DEC000DFD1009B042B02D1019A282A02D95348A2
:10DED00042F0DCFE206B6B4608A9083050F055FF7D
:10DEE0000028CED1019A282A03D0BDF82030012B7A
:10DEF0000CD1BDF82210022908D8BDF82E30102B05
:10DF000004D8122A04D1BDF830208AB14448DFE792
:10DF1000282A0DD1BDF820004FF6FE729042F5D1AF
:10DF2000BDF83820012AF1D1BDF832209A42EDD156
:10DF3000082B099A237394BF00230123A3734FF482
:10DF40000073A360002362606173E373206B6B4610
:10DF5000042202A9083050F018FF002891D1009E39
:10DF6000042E8ED12F49324602A853F0BFF98046C5
:10DF7000206B6B46324603A9083050F006FF00289C
:10DF80007FF47FAF009B042B7FF47BAF206B039A61
:10DF9000B8F1000F0AD0D0E91013521843F1000372
:10DFA000083050F0C1FB0028D0D06AE72262036C31
:10DFB000A38465B94FF48070E06253F0DAF8034649
:10DFC0002061E06A63B9A561657342F0C9FD6D081F
:10DFD00027612F44E562A761204612B0BDE8F081B9
:10DFE00053F0C7F8A0610028F6D1E06A2561657397
:10DFF000EBE700BF040002000F0080FFF4300900CF
:10E00000A05A0900DC190A00773D0900904E09006A
:10E0100074CB0900F7210900FC210900534A0900CB
:10E02000304B09001AFF08002DE9F04F2DED028B4F
:10E0300095B004460C920993426A002943D00C9B88
:10E04000012B00D1826A209BA1691960216A237F7C
:10E05000914240F04284D4E90421002B18BF1146BC
:10E06000099B07911960237F83F001032377A3693C
:10E070009B080B9304F130030E9300230D9306933A
:10E0800094F82C300D9A93421FDC069B3BB9079AFB
:10E090000B99069B02EB8101914240F0FD83A37B2B
:10E0A000002B00F0FD83236A013323620C9B002BBD
:10E0B00040F01B84636A01336362012015B0BDEC3C
:10E0C000028BBDE8F08F0C91BDE70E9B53F8045F07
:10E0D0000E93AB680A93002B40F0D0830D9B013365
:10E0E0000D93CDE7AB60069B002B00F0CE830123A0
:10E0F0000693F3E76B699B086B61431E58425841D6
:10E1000068730A98637B407BD5F810B06A699842BF
:10E110004FEA032140F0B180914228BF1146089A8E
:10E12000D4ED017A8A4294BF05920591F8EE677AA0
:10E13000F7EE000A80EEA77A059AB2FBF3F3A74A3E
:10E1400005F1180007EE903AF8EEE77AA44B9FED40
:10E15000A50A67EE877A27EE287AC3ED007AA24BEC
:10E1600083ED007A1378013313705DF0D0FCDFED9E
:10E170009F0AB0EE408A05F11C009FED9D0A5DF0FC
:10E18000E2FCDFED9C7A627B28EE278A022ABCEE55
:10E19000C88A18EE103A9BB2029374D110F4004F63
:10E1A00047F6FF73029909BF1B1AC0189BB24FF4C0
:10E1B00000401CBF80B24FF400434B434843C1139F
:10E1C000DB13039102932B6A11936B6A12930698E7
:10E1D0000A9B217B5B7B00261396002840F08D81F3
:10E1E000102940F00981A17B002900F084809A4227
:10E1F0007FD0DDF810A0DDF81880059B434565D978
:10E200005BF81890039B01931FFA89F0029B00931F
:10E2100040EA094012AB11AA13A94AF05DF9119E18
:10E22000360436FB00F6129F3F0437FB10F726F347
:10E23000CF3627F3CF37C6EA07464AF8086B4FEACE
:10E240001940039E01960004029E009640EA194080
:10E250004AF042F9119B1B0433FB00F3129A12049B
:10E2600032FB10F223F3CF3322F3CF32C3EA02435F
:10E270004AF8043C08F10208BFE752008A4228BF6E
:10E280000A4608994CE7029B03939CE7039B5BF8C3
:10E2900026000193029B009311AA12AB13A94AF026
:10E2A0001BF9119B1B0433FB00F3129A120432FB7F
:10E2B00010F223F3CF3322F3CF32C3EA0243049A9E
:10E2C00042F826300136059BB342DFD1059A089B00
:10E2D000607B9B1A0893049B03EB820304930A9BC5
:10E2E0005B7B9842D5E9041200F09B82059B5B089A
:10E2F00098E2069EE7E79A426BD0DDE904A35B084B
:10E300000BEB8303D9460F934FF0802B0F9B4B45AC
:10E31000DCD059F8043B93FA4BF8039B01931FFAA6
:10E3200088F0029B009340EA084012AB11AA13A99F
:10E330004AF0D2F8119E360436FB00F6129F3F04D5
:10E3400037FB10F726F3CF3627F3CF37C6EA074659
:10E350004AF8086B4FEA1840039E01960004029E9B
:10E36000009640EA18404AF0B7F8119B1B0433FBB3
:10E3700000F3129A120432FB10F223F3CF3322F38C
:10E38000CF32C3EA02434AF8043CBFE75BF82600F9
:10E3900090FA47F0039B0193029B009311AA12ABE2
:10E3A00013A94AF099F8119B1B0433FB00F3129A4E
:10E3B000120432FB10F223F3CF3322F3CF32C3EA3D
:10E3C0000243049A42F826300136059BB342DDD160
:10E3D0007CE7069E4FF08027F7E700BF116F012012
:10E3E0005C680120000000005868012000FE7F3FAB
:10E3F00000FE7FBF000000479A42059B4FEA430999
:10E400002BD1069E4FF080274E45BFF45FAF3BF8FF
:10E4100016005EF0F1FDA37B0BB990FA47F0039B69
:10E420000193029B009311AA12AB13A94AF054F86E
:10E43000119B1B0433FB00F3129A120432FB10F2FF
:10E4400023F3CF3322F3CF32C3EA02405AF001FB69
:10E45000049B23F816000136D6E7069F4FF080286C
:10E460007B1C4B45BFF432AF3BF807005EF0C4FDA8
:10E47000A37B06460BB990FA48F6039B0193B0B212
:10E48000029B009340EA064012AB11AA13A94AF07E
:10E4900023F8119B1B0433FB00FC129B1B0433FB72
:10E4A00010F32CF3CF3C23F3CF33CCEA03405AF0E4
:10E4B000D0FA049B23F81700039B0193300C029BB6
:10E4C0000093000412AB40EA16404AF005F8119B95
:10E4D0001B0433FB00F3129A120432FB10F223F3F5
:10E4E000CF3322F3CF32C3EA02405AF0B2FA049B90
:10E4F000023323F817000237B2E7102940F0F88002
:10E50000A17B002975D09A424CD0DDE90483D9461D
:10E510004FEA530B09EB8B0BD9453FF4D7AE59F8B3
:10E5200004AB039B01931FFA8AF0029B009340EA1D
:10E530000A4012AB11AA13A949F0CEFF119E36046E
:10E5400036FB00F6129F3F0437FB10F726F3CF3659
:10E5500027F3CF37C6EA074658F8080B96FA10F6A5
:10E5600048F8086C4FEA1A40039E01960004029E88
:10E57000009640EA1A4049F0AFFF119B1B0433FBA1
:10E5800000F3129A120432FB10F223F3CF3322F37A
:10E59000CF32C3EA024358F8042C93FA12F348F836
:10E5A000043CB9E7049B1F1F059B0BEB8308D84570
:10E5B0003FF48CAE039B5BF8040B0193029B00932A
:10E5C00011AA12AB13A949F087FF119B1B0433FB5F
:10E5D00000F3129A120432FB10F223F3CF3322F32A
:10E5E000CF32C3EA024357F8042F93FA12F33B6089
:10E5F000DDE79A4251D0DDE904935B080BEB83031E
:10E60000DA460F934FF0802B0F9B9A453FF45EAE96
:10E610005AF8043B93FA4BF8039B01931FFA88F0D6
:10E62000029B009340EA084012AB11AA13A949F0DB
:10E6300053FF119E360436FB00F6129F3F0437FB52
:10E6400010F726F3CF3627F3CF37C6EA074659F837
:10E65000080B96FA10F649F8086C4FEA1840039E2A
:10E6600001960004029E009640EA184049F034FFEB
:10E67000119B1B0433FB00F3129A120432FB10F2BD
:10E6800023F3CF3322F3CF32C3EA024359F8042CE9
:10E6900093FA12F349F8043CB6E7049B1F1F059B4D
:10E6A0004FF080290BEB8308C3453FF40FAE5BF8B6
:10E6B000040B90FA49F0039B0193029B009311AA6B
:10E6C00012AB13A949F008FF119B1B0433FB00F3A5
:10E6D000129A120432FB10F223F3CF3322F3CF321B
:10E6E000C3EA024357F8042F93FA12F33B60DBE7C7
:10E6F00005999A424FEA410A40F08E80049B4FF000
:10E7000080289F1E5645BFF4E1AD3BF816005EF031
:10E7100073FCA37B0BB990FA48F0039B0193029B17
:10E72000009311AA12AB13A949F0D6FE119B1B044A
:10E7300033FB00F3129A120432FB10F223F3CF33AF
:10E7400022F3CF32C3EA024237F8020F5EF054FCE4
:10E7500092FA10F05AF07DF901363880D2E73BF892
:10E7600006005EF049FCA37B07460BB990FA49F717
:10E77000039B0193B8B2029B009340EA074012AB9F
:10E7800011AA13A949F0A8FE119B1B0433FB00FE3C
:10E79000129B4FEA034C3CFB10FC2EF3CF332CF3BF
:10E7A000CF3CC3EA0C430F93049B33F816005EF092
:10E7B00023FC0F9B93FA10F05AF04BF9049B23F8BB
:10E7C0001600039B0193380C029B0093000412ABCC
:10E7D00040EA174049F080FE119B1B0433FB00F315
:10E7E000129A120432FB10F223F3CF3322F3CF320A
:10E7F000C3EA0242049B33F818005EF0FDFB92FA74
:10E8000010F05AF026F9049B023623F8180008F19C
:10E810000208C245A3D859E54FF001084FF08029FE
:10E82000F7E7059B01EB8301D21AC5E90412029BAD
:10E830002B62039B6B62089B002B3FF458AC6B6907
:10E84000002B7FF45EAC6B7B33B92B7B002B3FF44A
:10E8500049ACA8684AF0EEF8A86800283FF451AC2B
:10E8600005F1140205F110014AF099F802287FF42D
:10E8700041AC0023AB606B616B7334E40B9B08937A
:10E88000079BDFED228A0493D5E7089B069904983D
:10E890009A0052F080FD2AE442F8043BFFF7FCBBEB
:10E8A000237B0B9A102B079B03EB82020AD04FF0BD
:10E8B00080309A423FF4F7AB196881FA40F143F88F
:10E8C000041BF6E74FF080209A423FF4ECAB196846
:10E8D00091FA40F143F8041BF6E723B92369099A3A
:10E8E0001360FFF7E3BB6369F9E70C9B012B7FF42F
:10E8F000E4ABA36A227B0133A362099B1B6803EB91
:10E90000D203099A1360FFF7D8BB00BFDB0FC940E1
:10E910002DE9F04788B0084611461A4602AB01932C
:10E92000364B0093062352F08FFE40F27663FF22AF
:10E930000121029852F0BBFE40F212330646022239
:10E940000498012152F0B3FE079D002D804604DC9F
:10E9500040F28A51012021F0BFFBDDF814A0BAF18A
:10E96000080F05D0BAF1100F02D0254842F08EF9F9
:10E9700006F10D002349800054F0CBF9039F9DF868
:10E9800018900446F8088000A06152F0F2FB03469C
:10E990002061A0691BB96373636142F0E1F852F032
:10E9A000E8FB606118B960732061A069F5E76560F4
:10E9B0000025A76084F80CA084F80E9084F80D80E0
:10E9C000E57384F82C6004F13007B5420ADB94F853
:10E9D0002C0004F1340128F06FFB2063204608B0BE
:10E9E000BDE8F087002308481A46194600F068F889
:10E9F000013547F8040F4460E7E700BFBC290A006F
:10EA00002641090054CB0900A0290A00F0B50C46A4
:10EA100087B054F8045B0646687B174649F0BAFF96
:10EA200003AB0193114B00933A4603232146701E1A
:10EA300021F0C0FA95F82C209DF810309A4203D8A6
:10EA400040F2756021F0A8FA05EB8303039E5C6B2E
:10EA50009DF814706068314602F026F82046A660E2
:10EA600027734BF087FA284607B0F0BD88290A00C3
:10EA7000F0B50D4685B055F8044B0646607B174649
:10EA800049F088FF03AB01930C4B00933A460123F6
:10EA90002946701E21F08EFA94F82C209DF80C3037
:10EAA0009A4203D840F2756021F076FA04EB8304B1
:10EAB0000022636B0E209A6005B0F0BD80290A0029
:10EAC00010B508461146002221F03CFA0B492820D7
:10EAD00054F01FF900230446836000F1180140F24E
:10EAE000614207483EF030FB064840F2EB4204F139
:10EAF0001C013EF029FB204610BD00BFA0290A00E2
:10EB0000020000C0020080807FB502AB51F8044BC8
:10EB100001930A4B00930138022321F04BFA029D26
:10EB200060689DF80C60294601F0BEFF2046A56094
:10EB300026734BF01FFA0E2004B070BD70290A0036
:10EB40001FB503AB0193064B51F8044B00930138FA
:10EB5000012321F02FFA00230E20A36004B010BD82
:10EB600068290A002DE9F04FAFB0446A04901CB93F
:10EB7000389B1C60022021E00029049989681491C7
:10EB80003899149C0C60049991F9541008BF002224
:10EB90008A42049915D1049891F9551000EB81012E
:10EBA000496B01EB42021A60FF2380F85430389B16
:10EBB0001A68836D03EB5203836501202FB0BDE813
:10EBC000F08F91F84410049CB1FA81F1490984F85E
:10EBD000441084F85510C2F1010204EB810184F85D
:10EBE00054204A6B1A60069252F06AFC0498002185
:10EBF00052F041FC049B044670B99A68014606989D
:10EC000052F0C9FB389B1C60049B93F8450080F0D0
:10EC100001004000C0B2D1E7049ADB6A126BD21A3D
:10EC20000992049A12690392002A01F01685049A47
:10EC30000398576A1F44394647F042F9421C06467A
:10EC400001F00F85039BD3F80090B9F1000F00F09D
:10EC50003D81D3F80480B8F1000F00F0378199F8B6
:10EC600000B099F81C303C18BBF1000F3ED1032BCB
:10EC70004FF0090114BF4FF0200A4FF0110A2AA8E3
:10EC8000CDE92A4BCDE92CBA5FF0FDF8C8F80000B9
:10EC900099F81C30032B14BF032105212AA85FF02B
:10ECA000F2F8454645F8040F039BD3F8BC379B4563
:10ECB0000DDB4FF0000B039BD3F8C4379B4580F26C
:10ECC000C880902303FB0B850023059392E005F198
:10ECD000100301212AA805935FF0D5F8059B45F89C
:10ECE000040F9D42F5D10BF1010BDDE7032B4FF033
:10ECF000080114BF4FF0110A4FF0090A00232AA897
:10ED0000CDE92B332A94CDF8B4A05FF0BCF8C8F855
:10ED1000000099F81C30032B14BF022101212AA8FE
:10ED20005FF0B1F8C8F80400C3E70C212AA85FF02F
:10ED3000AAF80921A8622AA85FF0A5F80821E862CC
:10ED40002AA85FF0A0F8286399F80030002B14BFC0
:10ED5000092104212AA85FF096F8012168632AA8F6
:10ED60005FF091F8A863002856D002212AA85FF02E
:10ED70008AF80121E8632AA85FF085F80521286454
:10ED80002AA85FF080F8052168642AA85FF07BF864
:10ED90000023EB64A86403212AA85FF074F8032120
:10EDA00028652AA85FF06FF8032168652AA85FF03C
:10EDB0006AF8EB6BA86533BBC5E90A336B63E86D92
:10EDC000C0F11400286699F80030002B3FD10121D2
:10EDD0002AA85FF058F8686601212AA85FF053F866
:10EDE0000121A8662AA85FF04EF8059BE86601336A
:10EDF00005934835039B059AD3F8BC379A4294DBB8
:10EE00000BF1010B57E7022B04D12B6C13B908232C
:10EE1000EB65D4E70723FBE7C5E90F0005212AA826
:10EE20005FF031F8052168642AA85FF02CF805210D
:10EE3000A8642AA85FF027F80421E8642AA85FF0F4
:10EE400022F80321E8652AA85FF01DF8BAE7002040
:10EE5000C1E7039A0999D8F80080C2F8D88706EB71
:10EE60000A028A1A03990992D1F8B817039A04EB97
:10EE70000A05D2F8B02700295AD0002A40F0A48011
:10EE8000039BD3F8CC27099B934280F2AE8006996E
:10EE9000039847F078FF4FF0FF34149A069800214A
:10EEA00052F079FA049B93F845300BB903341BD820
:10EEB000049B06989A68002152F06DFA389A002354
:10EEC0001360049A012382F8453053E606990398AB
:10EED00047F059FF6FF00604049B099A1B6B9B1ABD
:10EEE000049AD362002CD8D1049B149A9B6D03EB37
:10EEF0005203049A9365104652F0E2FA04980021F6
:10EF000052F0B9FA049B049A1B6BD26A9A1A049BBA
:10EF10009B6A9B1AB3F5007F044607DD049AAE4B4B
:10EF200002F11400C2E9053201F03EFE204645E63A
:10EF3000002A49D10399DDF824B00122C1F8B02795
:10EF4000A94659464846059347F031FF431C059BA7
:10EF500018D019F800C039788C4509EB00021DD192
:10EF600092F801C079788C4518D197F802C0917851
:10EF70008CEA0101032911D81CF0020F18BF02F11D
:10EF8000FF32501B039A0028C2F8B4070CDA069926
:10EF9000104647F0F8FE6FF002049DE7033002F1DF
:10EFA0000309ABEB000BCCE7039A0644D2F8C02769
:10EFB00056445643039AD2F8C8275343039AF6009F
:10EFC00096FBF3F3C2F8B837039BD3F8B4271B685A
:10EFD00043B15B69003B18BF01231344039AC2F895
:10EFE000CC374DE74FF0FF33F7E7039B0399D3F896
:10EFF000DC37434501F11C003DDBA3EB0801424631
:10F0000041180A9052F0B1F9039BD3F8D807D3F80E
:10F01000CC270A9B2946184452F07CF9039B03999C
:10F02000D3F8CC27D3F8D8371344C1F8DC37DB004A
:10F030001093039B099903F2DC738A1A1A93002335
:10F0400009920C930593039B059AD3F8C4379A420F
:10F0500081F21E837C2353431193902353431993CE
:10F06000119B013B1F93119B08931A9B189300233C
:10F070000D939B46FEE32946184452F04BF9039B3F
:10F080000399D3F8CC27D3F8DC3703981344C1F89D
:10F09000DC37099B06999B1A09936FF0010447F02E
:10F0A00072FE19E7039B1E68002E00F0D4805B6897
:10F0B0000793002B00F0CF80039B9D68002D00F08C
:10F0C000CA800A9B22930023CDE923330C9A109B1C
:10F0D0009A18D31D48BF02F10E03DB1025930C9B39
:10F0E0001BB1194622A85EF0CEFE059B3178902216
:10F0F0005A43482303FB0B22079B1A44536BD2F855
:10F100003CC0002940F04E81344810F8136000EBF9
:10F110004300BCF1020F477862D1D2F84090B9F1B8
:10F12000000F10D0089B884605EB0309314622A842
:10F130005EF0A9FE08F10108B8F1080F09F8010B0B
:10F14000F4D14FF00309119B05EB03080D9B984484
:10F1500009EB49039844314622A85EF094FE3146FB
:10F1600088F8170022A85EF08EFE314688F8180055
:10F1700022A85EF088FE09F10109B9F1060F88F8AE
:10F18000190008F10308E6D1089BEE18394622A8B9
:10F190005EF079FE394686F8290022A85EF073FEFB
:10F1A000394686F82A0022A85EF06DFE09F10109B1
:10F1B000B9F10C0F86F82B0006F10306E6D1059A8B
:10F1C0007C2353433E2202FB0B332B44002283F863
:10F1D0003B209A8724E000BFE1FE040018660A0085
:10F1E000059B002B3ED10D9BDDF8148005EB030938
:10F1F000314622A85EF047FE08F10108B8F10B0F76
:10F2000009F8010BF4D10D9B1D44394622A85EF08C
:10F210003AFE05F8080008F10108B8F1150FF4D11D
:10F22000059B189A90265E434820079B00FB0B66BF
:10F2300033449B6A5360229B0A9A9B1A249AC2EB1E
:10F24000C302D71007D4189B53F804CF1893109B10
:10F25000634580F2ED810699039847F094FD6FF0C5
:10F26000070439E64FEA0B13079A083302EB030948
:10F2700052F80380B8F1000F1FD00D9B8846EB18A1
:10F280001F9913F8012B5A5408F10108B8F1060F21
:10F29000F6D1D9F80430FBB9089B4FF0060805EB0E
:10F2A000030A314622A85EF0EEFD0AF8080008F1D4
:10F2B0000108B8F10B0FF4D121E0089B05EB030A1C
:10F2C000314622A85EF0DFFD08F10108B8F1060F13
:10F2D0000AF8010BF4D1DCE7059C3E2303FB0BF39A
:10F2E0007C20EA1800FB04332B4491799971D17981
:10F2F000D971117A1972517A5972927A9A72D9F82F
:10F3000008306BB9089B0B2605EB0308394622A889
:10F310005EF0B9FD08F806000136102EF6D112E0B5
:10F32000059C3E2303FB0BF37C20EA1800FB04330F
:10F330002B44D17AD972117B1973517B5973917B0C
:10F340009973D27BDA73D9F80C306BB9089B10260D
:10F3500005EB0308394622A85EF095FD08F8060083
:10F360000136152EF6D112E0059C3E2303FB0BF36C
:10F370007C20EA1800FB04332B44117C1974517C67
:10F380005974917C9974D17CD974127D1A75059A3F
:10F390007C2353433E2202FB0B332B4400225A753D
:10F3A0009A753DE7366A16F0010603D0BBF1010FEE
:10F3B00000F0B280B3F5C87F7BDA1911052291FB0A
:10F3C000F2F2269202EB8202891AC3F3810228929A
:10F3D00003F0030300222791299311461346BCF141
:10F3E000020F40F0CE80059C902060434827079C88
:10F3F00007FB0B002044006C002808BF4FF0010CF5
:10F4000001EB41018948614410F821702A9700EB13
:10F41000810148782B908878C9782C902D910EB373
:10F42000BBF1010F1ED10DF1980C05F1FC070DF198
:10F43000A80E664603CE764538607960B44607F17B
:10F440000807F6D10DF1A80C05F58677664603CEC0
:10F4500079602EA98E423860B44607F10807F5D1CD
:10F46000C5F8F820059990224A43482101FB0B2258
:10F4700007990A445366D36B022B40F0C580176C82
:10F48000002F00F0A880089B0026EF18269922A8DC
:10F490005EF0F9FC0136062E07F8010BF6D14FF0AD
:10F4A00001080327119B05EB030A0D9B0AEB0304DC
:10F4B0008BE0B3F5FA7F12DAA3F5C8739910052231
:10F4C000B1FBF2F2269202EB8202891A03F00303E7
:10F4D0000022279128932992134601217FE7A3F563
:10F4E000FA730321B3FBF1F101EB41020598269178
:10F4F0009B1A0022CDE9282290224243482000FB9B
:10F500000B22079827930244126C0AB1CDE9271306
:10F5100000220123022162E7B3F5B47F03F0010268
:10F520004FEA630110DA242091FBF0F3269300FBED
:10F530001313062093FBF0F100FB113328930023F3
:10F540002791299303214AE7F3290CDCB4390B11E5
:10F550002693C1F38103279301F00301002328912F
:10F56000299304213BE7F4390323B1FBF3F32693FA
:10F5700003EB4303C91A00232791CDE92833052162
:10F580002DE74FF0000C3BE726AB22A853F828A04C
:10F5900051465EF078FC5146F07522A85EF073FC8F
:10F5A0005146307622A85EF06EFC033609F101095F
:10F5B000B0752AAB53F828209145E5DB08F1010826
:10F5C000B8F1040F3FF4FBAD4F4407EB4706264468
:10F5D0004FF00009EDE7B84664E753F8261022A87B
:10F5E0005EF051FC09F8010B013726AB5AF82620D2
:10F5F0009742F2DB0136042E0DD0B84404EB080923
:10F6000000270DF1A80AF1E7089B4FF00008EC185D
:10F61000464626ABF2E7059A7C2353433E2202FB83
:10F620000B331D440023AB756B75F9E538660A0092
:10F63000039B1D68002D00F0C2815B680B93002BBB
:10F6400000F0BD81039B9B68002B00F0B881039BF9
:10F65000D968002900F0B38102F0070313930C9BD3
:10F66000139AC3EBC70313441C93BCEB0303079328
:10F6700000F1A5810A9B6A6B3B441D930B9B1E44C2
:10F68000B36B002B00F02381F36B022B40F01F8142
:10F69000336C002B40F00381059C9023634300FBF7
:10F6A0000B330B9803440320DB6D013393FBF0F322
:10F6B00002EB4303B3F92E0000EB40004FF410724D
:10F6C000059C9023634348250B9C05FB0B33234487
:10F6D000DB6A5B00B3F5107FA8BF4FF41073934251
:10F6E000D4BF2C932C920A932D938342D4BF2B9397
:10F6F0002B9001EB8B03209303F580530A9AC3F8F8
:10F7000000224FF4106303FB0B131593139B0F930D
:10F710001D9B0C93002316930E93199B4033E31803
:10F7200021930E9B169F01332AAA0E9352F8233081
:10F730001693A3EB070EBEF1000F23DD159B0E9A67
:10F740000C9903EB8707219B53F82250B14B03EB35
:10F75000C5031E790F9B5A4202F0070213462AB1D5
:10F7600011F8010BC2F1200200FA02F2002E40F063
:10F77000C08033463A1D47F8263042F8263002361C
:10F78000B645F8DC00230F9A0C991A4401EBE2010C
:10F7900002F007020F92079A0C91D31A07930E9B5F
:10F7A000032BBED1109B1C9A9B1A0E93079B002B18
:10F7B00000F09F82159B0A9A0C9803EB8205059A2C
:10F7C00090235343482202FB0B330B9AD318924ADF
:10F7D000DB6E52F823200B92904A52F823100F9BB5
:10F7E0005B4203F007031A462BB110F8016BC3F11B
:10F7F000200306FA03F3079CA61A0A9C4FF000099F
:10F80000C4F50F7AC1F120014F460AF1010A0A91AD
:10F81000BA4500F3F081209B03F58052D2F8003204
:10F820003B44C2F800320022B3F5107FC0F263827D
:10F83000079A0F9B13440C9A02EBE30203F00703B1
:10F840000C93089B0A923E3308930D9B3E330D9315
:10F85000199B4833199313461D9A9B1A00F1AF80E8
:10F86000139AC2EBC3030C9A13440E9AD31A109343
:10F870000BF1010B039BD3F8BC379B45FFF612AC91
:10F880000599039844F030FF013040F05785069900
:10F89000039847F078FA6FF00904FFF71DBB2B7847
:10F8A0005BB9059C9023634300FB0B330B98034427
:10F8B000DB6D013332F9130000E7B2F93600B2F91B
:10F8C0003430C31AB2F90C0000EB4300F6E6059B96
:10F8D00090255D43482303FB0B550B9B1D44EB6DAB
:10F8E0002D6E013332F913002B44013332F913200A
:10F8F000E6E64B4850F825C04A4800EB4C0017900C
:10F900000798012EA0EB030040F08E80454C34F8A0
:10F910001C6006F00F064FF000094FF0004AC6F1D8
:10F9200020060F2853DD8C46C3F118081CF8025B33
:10F93000497805FA08F5C3F1100801FA08F10D43FA
:10F940002A431033103861460A2BEADD22FA06F505
:10F95000179C013534F815504FEA153C15F0F00F9F
:10F9600002FA0CF218BF02F0004CA3EB1533C5F3FA
:10F9700003181EBF520003F1FF334CEA080815F4C8
:10F98000706FC5F3032C1FBF03F1FF3302F0004576
:10F9900045EA0C0C52004B4511DB47F8088BAEF1E1
:10F9A000020EBEF1000F47F804CCCDDCA3EB090337
:10F9B000079A0344D31A079A93427FF6E4AE069956
:10F9C000039847F0E0F96FF00804FFF785BA1D18B7
:10F9D000002DF4DD002812DD082891F800C0C8BF12
:10F9E0004878C3F118080CFA08FCC8BFC3F110032B
:10F9F00042EA0C02C9BF98400131024302316B1E3A
:10FA00004AFA03F31A404FF00B0905F10B030020EB
:10FA10009AE700BF14430A0010660A0008660A004D
:10FA200038650A0014440A00A6F1020CBCF1010F6B
:10FA3000C5D8DFF8F0C25CF83580DDF85CC0002482
:10FA4000129408F101041B94C8F120041E940F289D
:10FA500027DD8946C3F1180A19F8025B497805FACF
:10FA60000AF5C3F1100A01FA0AF10D432A431033D3
:10FA7000103849460A2BEADDBCF8009009F00F095E
:10FA8000C9F1200522FA05F501353CF815505FEA69
:10FA9000153A2AD1A3EB090302FA09F20CEB450C43
:10FAA000E8E7C518002D8ADD002812DD082891F846
:10FAB0000090C8BF4878C3F1180A09FA0AF9C8BF0C
:10FAC000C3F1100342EA0902C9BF98400131024361
:10FAD00002314FF000406B1E40FA03F30B201A4036
:10FAE000129005F10B030020C4E7C5F30319B9F127
:10FAF0000F0FA3EB0A0302FA0AF2C5F3032523D181
:10FB0000032E24D11B9C03EB000C002D0CBFA2463E
:10FB100004F1010AE2453FF752AF9C46E24552DC50
:10FB20000344B3EB0C0006D5581E9C464FF000432F
:10FB300003411A4000201E9B22FA03F909F10F0924
:10FB4000ACEB080302FA08F2B9F1000F05D002F09D
:10FB5000004C49EA0C095200013B0F2D1DD1032E28
:10FB60001CD11B9C1D18AC423FF729AF9C461B9C27
:10FB7000644533DC0344B3EB0C0006D5581E9C46A9
:10FB80004FF0004303411A4000201E9B22FA03F568
:10FB90000F35ACEB080302FA08F22DB102F0004C6D
:10FBA00045EA0C055200013B129CA342FFF607AF49
:10FBB000AEF1020EBEF1000FC7E9009518DDDDF8C9
:10FBC0005CC0083756E711F8019BCCF1180409FA1C
:10FBD00004F942EA09020CF1080C9FE711F8015BF5
:10FBE000CCF1180A05FA0AF52A430CF1080CBEE715
:10FBF000129A9B1ADCE60F2E56DD8446C2F1180ECF
:10FC00001CF8021B407801FA0EF1C2F1100E00FA46
:10FC10000EF001430B431032103E60465745BFF6CD
:10FC2000F7AD092A7FF7F4AD0A990B9C23FA01F18D
:10FC300021443B4C615C4FEA111C03FA0CF311F0B8
:10FC40000808A2EB11121FBF03F0004802F1FF32B7
:10FC50005B0048F0010811F0040E1FBF03F0004ED6
:10FC600002F1FF325B004EF0010E11F0020C1FBFDB
:10FC700003F0004C02F1FF325B004CF0010C11F07C
:10FC800001011FBF03F0004102F1FF3241F0010109
:10FC90005B004A45FFF6BFAD45F8108B043745E9D8
:10FCA00003EC45F8041CB9E7B11800297FF7B3ADA0
:10FCB000002E12DD082E90F800C0C8BF4678C2F1B1
:10FCC000180E0CFA0EFCC8BFC2F1100243EA0C0376
:10FCD000C9BF96400130334302304A1E4FF0004402
:10FCE00044FA02F213404FF00A0901F10A02002619
:10FCF00094E7079F8FE5159941F82320013393E599
:10FD0000059903982A4645F0AFFC01300CD10699BD
:10FD1000039847F038F86FF00A04FFF7DDB800BF2A
:10FD2000B8650A0014430A000135039BD3F8BC37B9
:10FD30009D42E5DB039AD268002A00F08684039A8C
:10FD400052690B92002A00F08084039A926907920C
:10FD5000002A00F07A84039AD2F8C867059A5643BD
:10FD6000069A5E43022B02EB460640F0E9820B9BAB
:10FD70001193331D089300230E93079B03F5005343
:10FD80000D930E9B0D9A0799119803F001030F93A1
:10FD90000B9B03F580554FF00077D5F8183B009387
:10FDA000D2F800220F9B45F03FF9D5F81C3B0D9A85
:10FDB000079911980093D2F800220F9B803100F52B
:10FDC000106045F031F90F9B0D9A5B42D2F800228A
:10FDD00003F488631344079A02EB830B4FF0000C83
:10FDE00052F82320DBF85C306046C2FB007C6FF0E9
:10FDF0007301C3FB017C4FF00076DBF88020DBF859
:10FE0000DC300546C2FB0065C3FB01654FF4557944
:10FE1000DBF80430DBF85820C3FB097C834BC2FBC2
:10FE2000037CDBF88410DBF8D820C1FB0965C2FB3A
:10FE3000036541F6D478DBF80830DBF85420C3FBC7
:10FE4000087C7B4BC2FB037CDBF88810DBF8D420FA
:10FE5000C1FB0865C2FB036546F2B86EDBF80C30E7
:10FE6000DBF85020C3FB0E7C724BC2FB037CDBF83B
:10FE70008C10DBF8D020C1FB0E65C2FB03656E4A17
:10FE8000DBF81030DBF84C10C3FB027C6B4BC1FB82
:10FE9000037CDBF89000DBF8CC10C0FB0265C1FBF3
:10FEA0000365DBF81420DBF84830C2FB0E7C45F21A
:10FEB0008401C3FB017CDBF89420DBF8C830C2FB73
:10FEC0000E65C3FB0165DBF81820DBF84430C2FB8C
:10FED000087C40F22C71C3FB017CDBF89820DBF836
:10FEE000C430C2FB0865C3FB0165DBF81C20DBF8EE
:10FEF0004030C2FB097C7421C3FB017CDBF89C20F1
:10FF0000DBF8C030C2FB0965C3FB01650C24384631
:10FF10004FF014080CFA04F34CFA08FC20FA08F02D
:10FF200040EA030046F022FC089B23F8040C30460C
:10FF300005FA04F345FA08F520FA08F040EA030050
:10FF400046F014FC089B0BF5805723F8020C3B6825
:10FF50004FF4D0704FF000724FF0000CC3FB002C38
:10FF60004FF00073D7F880100026C1FB003641F631
:10FF70007C007968C1FB002CD7F88410C1FB0036E7
:10FF800049F2FC70B968C1FB002CD7F88810C1FB9E
:10FF900000362B49F868C0FB012CD7F88C00C0FB59
:10FFA000013628493D69C5FB012CD7F89050C5FBA7
:10FFB00001366FF0B3057969C1FB052CD7F89410B1
:10FFC000C1FB05364FF41275B969C1FB052CD7F892
:10FFD0009810C1FB05366FF0130EF969C1FB0E2CAA
:10FFE000D7F89C101D46C1FB0E5610460CFA04F3C0
:10FFF0004CFA08FC20FA08F040EA030046F0B6FB91
:020000023000CC
:10000000089B9887284606FA04F346FA08F620FA71
:1000100008F040EA030046F0A9FB089B0A49D8878C
:1000200004331293089B043B13930FE0D4F8FFFFB3
:100030007CAFFFFF3CB6FDFF78940400C44902008A
:100040004CE803002464FFFFF43E0A00D1F840E0CE
:10005000DBF80051DBF85C014FF000730022C5FBB8
:100060000E324FF000764C6C4FF00009C5FB04696E
:10007000C4F1000CC0FB0C32C0FB0E69DBF8DC01E4
:10008000DBF8804115904FF000774FF0000AC4FB79
:100090000E7A4FF00075486C4FF00008C4FB005812
:1000A0001598C0FB0C7AC0FB0E58D1F848E0DBF87D
:1000B00004C1DBF85801CCFB0E32CC6CCCFB0469DC
:1000C000C4F1000CC0FB0C32C0FB0E69DBF8D80198
:1000D000DBF884411590C4FB0E7AC86CC4FB005851
:1000E0001598C0FB0C7AC0FB0E58D1F850E0DBF835
:1000F00008C1DBF85401CCFB0E324C6DCCFB04691B
:10010000C4F1000CC0FB0C32C0FB0E69DBF8D4015B
:10011000DBF888411590C4FB0E7A486DC4FB00588B
:100120001598C0FB0C7AC0FB0E58D1F858E0DBF8EC
:100130000CC1DBF85001CCFB0E32CC6DCCFB04695A
:10014000C4F1000CC0FB0C32C0FB0E69DBF8D0011F
:10015000DBF88C411590C4FB0E7AC86DC4FB0058C7
:100160001598C0FB0C7AC0FB0E58D1F860E0DBF8A4
:1001700010C1DBF84C01CCFB0E324C6ECCFB046999
:10018000C4F1000CC0FB0C32C0FB0E69DBF8CC01E3
:10019000DBF890411590C4FB0E7A486EC4FB005802
:1001A0001598C0FB0C7AC0FB0E58D1F868E0DBF85C
:1001B00014C1DBF84801CCFB0E32CC6ECCFB0469D9
:1001C000C4F1000CC0FB0C32C0FB0E69DBF8C801A7
:1001D000DBF894411590C4FB0E7AC86EC4FB00583E
:1001E0001598C0FB0C7AC0FB0E58D1F870E0DBF814
:1001F00018C1DBF84401CCFB0E324C6FCCFB046918
:10020000C4F1000CC0FB0C32C0FB0E69DBF8C4016A
:10021000DBF898411590C4FB0E7A486FC4FB005878
:100220001598C0FB0C7AC0FB0E58D1F878E0DBF8CB
:100230001CC1DBF84001CCFB0E32CC6FCCFB046957
:10024000C4F1000CC0FB0C32C0FB0E69DBF8C0012E
:10025000DBF89C411590C4FB0E7AC86F1691C4FB65
:1002600000581599C1FB0C7AC1FB0E580C24184696
:10027000142102FA04F342FA01F220FA01F040EAF2
:10028000030046F073FA129B23F8040C3846142737
:100290000AFA04F34AFA07FA20FA07F040EA0300E0
:1002A00046F064FA129B23F8020C304609FA04F374
:1002B00049FA07F920FA07F040EA030046F056FA37
:1002C000139BA3F87C00284608FA04F348FA07F8C1
:1002D00020FA07F040EA030046F048FA139B16990B
:1002E000A3F87E00129B04331293139B043B1393D9
:1002F000DE4B40318B420BF5807B7FF4A7AE0D9B2C
:100300000F9AD3F800329B1A0D9A03F00703C2F834
:1003100000320E9B01330E93119B80331193089B87
:10032000803308930E9B122B7FF42BAD059B01337A
:1003300005931A9B08331A93FEF785BE0025F4E453
:10034000079B4036002703F5005807F001030E9382
:100350000B9B0B98079903F5805300EBC710D3F85C
:10036000183B0093D8F8002207F0010344F05CFE2C
:1003700007F00103D8F800225B4203F488631344BA
:10038000079A02EB8309002052F82310D9F85C2069
:100390004FF000730446C1FB04306FF07301C2FBE1
:1003A00001304FF4557ED9F80420D9F85810C2FB1B
:1003B0000E30AF4AC1FB023041F6D47CD9F8082098
:1003C000D9F85410C2FB0C30AA4AC1FB023046F2E5
:1003D000B865D9F80C20D9F85010C2FB0530A64AF0
:1003E000C1FB0230A54AD9F81010C1FB0230A44A63
:1003F000D9F84C10C1FB0230D9F81410D9F84820B4
:10040000C1FB053045F28401C2FB0130D9F8181058
:10041000D9F84420C1FB0C3040F22C71C2FB0130F2
:10042000D9F81C10D9F84020C1FB0E307421C2FB52
:1004300001300C2402464FF0140A184602FA04F365
:1004400042FA0AF220FA0AF040EA030046F08EF976
:1004500009F5805126F8400C0A684FF0007000231F
:100460004FF4D075C2FB050341F67C054A68C2FB18
:10047000050349F2FC758A68C2FB0503814DCA6811
:10048000C2FB0503804A0D69C5FB02036FF0B3058B
:100490004A69C2FB05034FF412758A69C2FB050362
:1004A000CA696FF01301C2FB010303FA04F243FAB5
:1004B0000AF320FA0AF040EA020046F057F9DFF8A2
:1004C000CCA126F8200CA6F140030D930896DAE99A
:1004D00010ECD9F80021D9F85C114FF0007000231E
:1004E000C2FB0E034FF000754FF0000BC2FB0C5B1C
:1004F000CCF10002C1FB0203C1FB0E5BDAE912EC96
:10050000D9F80411D9F85821C1FB0E03C1FB0C5BCB
:10051000CCF10001C2FB0103C2FB0E5BDAE914EC73
:10052000D9F80811D9F85421C1FB0E03C1FB0C5BAB
:10053000CCF10001C2FB0103C2FB0E5BDAE916EC51
:10054000D9F80C11D9F85021C1FB0E03C1FB0C5B8B
:10055000CCF10001C2FB0103C2FB0E5BDAE918EC2F
:10056000D9F81011D9F84C21C1FB0E03C1FB0C5B6B
:10057000CCF10001C2FB0103C2FB0E5BDAE91AEC0D
:10058000D9F81411D9F84821C1FB0E03C1FB0C5B4B
:10059000CCF10001C2FB0103C2FB0E5BDAE91CECEB
:1005A000D9F81811D9F84421C1FB0E03C1FB0C5B2B
:1005B000CCF10001C2FB0103C2FB0E5BDAE91EECC9
:1005C000D9F81C11D9F84021C1FB0E03C1FB0C5B0B
:1005D000CCF10001C2FB0103C2FB0E5B0C24142111
:1005E00003FA04F243FA01F320FA01F040EA0200B0
:1005F00046F0BCF80D9B23F8020F14210D932846FA
:100600000BFA04F34BFA01FB20FA01F040EA030075
:1006100046F0ACF8089B23F8020D0893134B0AF13F
:10062000400A9A4509F580797FF451AFD8F8003235
:100630000E9A01379B1A03F00703122FC8F80032F5
:1006400006F140067FF481AE70E60699039846F005
:100650009AFB6FF00B04FEF73FBC6FF00404FEF74B
:100660003BBC6FF00504FEF737BC00BFB4420A0084
:10067000D4F8FFFF7CAFFFFF3CB6FDFF7894040089
:10068000C44902004CE803002464FFFFF43E0A0062
:100690000024FEF721BC00BF2DE9FF411C460D469A
:1006A00028461146424A1FF04DFC2768414B3B400B
:1006B000062B05D0BA070AD13A683F4B9A4206D1B9
:1006C00039463E4845F2F62251F0FDF80746012131
:1006D000384623F045FA067C16F0010602D0384869
:1006E00040F0C0FA012D2BD96068062201A923F041
:1006F000E5F9DDE9015633495C2052F011FBEB07C7
:1007000004461FD50135013EB6F5305F1CD905F50D
:1007100090536563A6F5105605F51055A363656201
:10072000A6620023C4E90B335DF03BFB2061002887
:1007300035D1204649F033FC234924485CF03BFC8A
:100740003546D8E7002DDFD14FF40068C4F8288083
:10075000404650F00EFD606228B9204649F01FFC6B
:10076000404640F0FDF9B6F5105F04D3656305F52A
:100770009055A563D5E74FF4905050F0FAFC6063B4
:1007800028B9204649F00BFC4FF49050E9E74FF4AC
:10079000905050F0EEFCA0630028C2D1F1E7204653
:1007A000394609F025F8204604B0BDE8F08100BFC5
:1007B000040002000F0080FFF4300900A05A090075
:1007C000773D090034CB0900EA4C09007830090074
:1007D00010B50446407B48F0DDF8A3689FED107A21
:1007E0005A0800EE102A94F8442004EB820423F007
:1007F0000103626B13449A4209D1F1EEC77ABDE856
:100800001040B8EEC00A87EE800A26F0C9BA32F965
:10081000021B07EE901AF8EEE77AA7EEA77AEAE74E
:100820000000000038B504460D46407B48F0B2F8A1
:1008300045F2F6222946044851F045F80146204683
:1008400008F0D6FF0E2038BDA05A090038B50D4675
:100850000446407B48F09EF80121284623F080F9A9
:10086000037CDB0702D5044840F0FCF9204629460A
:1008700008F0BEFF0E2038BD773D0900F0B587B007
:10088000084611461A4603AB0193274B00930323F6
:1008900050F0DAFE40F25D4103985CF067FD40F2F3
:1008A0006951074604985CF069FD204906462420FA
:1008B00052F036FABDF814501D49044600220B6868
:1008C000D3F80005C0070AD50132042A01F104015A
:1008D000F5D10023A36033B9164840F0A5F91649B5
:1008E0008A5C2277F6E70022C3F80C25A368012270
:1008F000C3F81025A2683B792376C2F860353879B1
:1009000008F0CCFB3EB1A26833796376C2F8683553
:10091000307908F0C3FBA3682D0A01222046A58286
:10092000C3F8002507B0F0BD042B0A0018CB09005E
:10093000DC230A005E4F0900D6230A00F0B50D46FD
:1009400085B055F8044B0646A068174649F047F8AD
:1009500002AB0193524B0093701E294602233A4684
:100960001FF028FB2046029E9DF80C5049F028FB02
:1009700010B1204649F02FFB314640F2165028F0C6
:1009800015FC666084F82050337B7568DB08E376DD
:10099000F37B84F82230B37B003B18BF012384F83B
:1009A0002130B768737BA37638464FF43F724FF619
:1009B000FF71BF001FF0AEFB384650F0DAFB94F831
:1009C0002230E0601BB9384650F0D3FB206105F5BA
:1009D00074432333B3FBF5F36B43590801F57401FA
:1009E00001F51051B1FBF3F14B08A26803F5740354
:1009F00003F51053B3FBF1F303EB5503B3FBF5F32E
:100A0000013BC2F84835A268C2F828354B1EE38284
:100A1000A368C3F80815A3680122C3F81425606809
:100A200048F008F81F4A00231146106890BB41F8AF
:100A300023403BF00FFCA36800250422A577204645
:100A4000C3F8002229464FF02AF8A368D3F82025DE
:100A5000C3F84025A368D3F82425C3F84425A36828
:100A6000C3F80851A368C3F80C51A368C3F8105128
:100A7000A368C3F81451A368C3F80451A3680C22F7
:100A8000C3F80423A26801230E2093606377E577FF
:100A900005B0F0BD0133042B02F10402C5D1CAE751
:100AA000F42A0A008C50012070B50D46044640F22D
:100AB000165028F07BFB6E7B304647F06BFF6A6870
:100AC00063689A4204D040F28A510D4840F0E6F83B
:100AD000637B022B04D0B34202D040F21231F4E720
:100AE0002A7B237B9A4202D040F2E521EDE7AA7BE4
:100AF000A37B9A4202D040F2BF51E6E770BD00BF2F
:100B0000E545090010B50C4C206890B10B4B1B68F3
:100B100083B95AF028FF236883422368A0EB0300BF
:100B200088BF00F1FF3040F2EE23984294BF0020CE
:100B3000012010BD0020FCE7E45E0120AC50012044
:100B4000024A136823EA000313607047AC50012087
:100B5000024A136803431360704700BFAC50012082
:100B600038B50C4B1B78A3B10B4B1B688BB90B4CE6
:100B700025685AF0F8FE2060236813B92368013312
:100B8000236035B9064B01221A70064B03F1780237
:100B90009A6238BD2D6E0120AC500120E45E012028
:100BA000626D0120BC62012010B504460BF088FA8A
:100BB000E3681BB90A4A1168A14203D1BDE810409D
:100BC0000BF090BAA360074B1968E160196809B18E
:100BD00019688C60116801B914601C60EEE700BFF1
:100BE000BC500120C450012008B50BF069FA044A3A
:100BF0001368013B1360BDE808400BF073BA00BFF7
:100C0000B050012008B50BF05BFA044A13680133B9
:100C10001360BDE808400BF065BA00BFB05001207A
:100C20002DE9F041134E33680BB3134D0BF048FA26
:100C30002C681CB1BDE8F0410BF054BA0F4A0123F7
:100C40002B603368346014601BB92B68013B2B6048
:100C5000F0E7D3E900689F68C3E902440BF042FA69
:100C60000EB14046B0470BF02BFA3B46ECE7BDE82F
:100C7000F08100BFBC500120B0500120C4500120C1
:100C800008B525F069F8C1880348972914BF972251
:100C900042223FF0EFFF00BF6140090010B5064A55
:100CA000002352F83340844202EBC30101D90133DF
:100CB000F7E7486810BD00BF38230A00F0B595B0CB
:100CC000054601A80E4617461C4657F004FD10B114
:100CD000002015B0F0BD3A46314628461FF010FC02
:100CE0002EF096FF830703D10268034B9A42EFD0A0
:100CF00020600120EDE700BFCC300900014A042349
:100D000033F032BDA43A0A00F0B587B00846114668
:100D10001A4602AB0193254B0093042350F094FC38
:100D20002349182051F0FCFFDDE904230361214B26
:100D30009A428CBF0123B3FBF2F3C3601E4BD3F87E
:100D4000AC31DDE9027604465BB317F04BF880F076
:100D50000105EDB204F11503009300222B4640F289
:100D60009351384610F062FC04F1160360600022D3
:100D7000009340F296512B46304610F057FC01226A
:100D80001146A06060684BF0B8FF0122A0681146D0
:100D90004BF0B3FF20465AF089F820B905203FF008
:100DA0002DFF0125D6E7204607B0F0BDD42A0A0062
:100DB000FCCA090020A10700BC620120F0B50C4666
:100DC00087B054F8045B06462846174648F022FED2
:100DD000284648F02CFE02AB0193094B00933A469B
:100DE0002146701E04231FF0E5F8059B009328465A
:100DF000DDE90323029958F0E7FD0E2007B0F0BDAE
:100E0000B42A0A00F0B50C4687B054F8045B0646D5
:100E10002846174648F0FEFD284648F008FE02AB7B
:100E200001930A4B00933A462146701E04231FF09B
:100E3000C1F801230193059B00932846DDE90323B4
:100E400002995CF03FFF0E2007B0F0BD942A0A0023
:100E5000F0B50C468BB054F8045B0646284617469E
:100E600048F0D8FD284648F0E2FD03AB01930E4B55
:100E700000933A462146701E07231FF09BF800237B
:100E80000193079B0093DDE90312069B28465CF063
:100E900019FF099B00932846089B059A039958F06F
:100EA00093FD0E200BB0F0BD5C2A0A00F0B50D4694
:100EB00087B055F8044B06462046174648F0AAFD71
:100EC000204648F0BAFD02AB0193204B00933A460E
:100ED0002946701E04231FF06DF840F205530122CD
:100EE0000021039850F0E3FB40F2F543012200217A
:100EF0000646C5B2049850F0DAFB40F2E32309221B
:100F000008210746059850F0D2FB0299104AB2FB1F
:100F1000F1F301FB132202B101332361237DC3F3FB
:100F20008002AA420AD066F3820323756B1E5942DF
:100F300060684FF0000259414BF0DFFE237D0E2028
:100F400067F3C303237507B0F0BD00BF242A0A006E
:100F500020A107002DE9F04186B0084611461A4647
:100F600003AB01932D4B0093032350F06DFB2C49F1
:100F7000182051F0CEFE2B4B059ED3F8AC31DDE9A5
:100F800003870446002B47D016F02CFF80F00105A4
:100F9000EDB204F11503009300222B464FF4477184
:100FA000404610F043FB217D60600022C1F38001C8
:100FB0004BF0A3FE04F11603009301222B4640F2EE
:100FC000AC41384610F032FB227DA060B0F10E0338
:100FD00018BF012363F341029307227503D5002252
:100FE00011464BF08AFE04F11703009301222B46B1
:100FF00040F29D41304610F019FB05232361237D0B
:10100000E06023F00D030E2818BF43F001032046D3
:10101000237506B0BDE8F0810125BAE7442A0A002D
:10102000E0CA0900BC6201202DE9F04F0D468DB0E9
:1010300055F8044B06462046174648F0EBFC204680
:1010400048F0FBFC08AB0193494B0093294604236D
:101050003A46701E1EF0AEFF062205A9089822F03F
:101060002DFD9DF81C10002240201FF0E7F8099B81
:1010700004930546069B0A99B3FBF0F303AA04A860
:10108000039357F040FB049B039A6B43554304932F
:101090000395002D48D0227DD60704D4354840F270
:1010A0009D413FF0FBFD900742D4059A9DF82C909E
:1010B0002769154403EB02081D444FF0000B4E4610
:1010C0004FF0080A237D990704D5A368F1095868F1
:1010D00049F0E6F8217D0A0732D438462EF034FF75
:1010E000217D636881F004015868C1F3800149F0F3
:1010F000D7F8E06809F0ACFF217D0B0740EA4B0B05
:101100002CD438462EF020FF217D6368C1F3800186
:10111000586849F0C5F87600BAF1010AF6B2D1D1A3
:1011200008F801BB4545C8D10E200DB0BDE8F08FD1
:10113000A3680021586849F0B3F805203FF05EFD30
:101140006368C1F3800181F00101586801F0010179
:1011500049F0A6F838462EF0F7FECAE76368C1F3F7
:101160008001586849F09CF838462EF0EDFED2E731
:10117000EC290A004D490900F0B50C468BB054F833
:10118000045B06462846174648F044FC284648F0CB
:1011900054FC07AB01931D4B0093214603233A46B1
:1011A000701E1EF007FF052204A9079822F086FC96
:1011B0009DF81810002240201FF040F8089B039370
:1011C0000446059B0999B3FBF0F302AA03A8029316
:1011D00057F099FA039B029A634354430393029492
:1011E0008CB1297D049A890704D4094840F2AC41A6
:1011F0003FF054FDD15CAB68C909586849F050F81C
:1012000005203FF0FBFC0E200BB0F0BD0C2A0A00BD
:101210004D490900F0B50C4693B054F8046B0546EF
:101220003046174648F0F6FB304648F006FC0CAB5B
:101230000193344B009321460623681E3A461EF064
:10124000B9FE052209A90C9822F038FC9DF82C1053
:10125000002240201EF0F2FF0E9B0F9905930446DA
:101260000A9BB3FBF0F304AA05A8049357F04BFACA
:10127000062206A90D9822F021FC9DF820100022DC
:1012800040201EF0DBFF109B119903930546079B3E
:10129000B3FBF0F302AA03A8029357F034FA049ABE
:1012A000059B029963435443039A05936A434D4354
:1012B000AC4204940392029502D013483FF0E6FC3E
:1012C000E4B1307D0999850701EB030405D424B10D
:1012D00040F2AC410D483FF0E1FCC00705D4069850
:1012E000D04202D040F29D41F4E7C95CB368C9091D
:1012F000586848F0D5FF05203FF080FC0E2013B061
:10130000F0BD00BF5C2B0A00F44009004D49090004
:101310000E2AF7B506460D46174602D133483FF070
:1013200035FC806848F05BFBAA0706D12A68304B81
:101330009A4202D12F483FF04DFCEB071FD5B288EF
:10134000F3885343B3EB650F4FEA650405D8013BBF
:1013500000225C2128483FF031FC94FBF2F502FBAF
:101360001544042F24B22DB22AD12A4621463046F4
:1013700048F0C2FF400040F0010003B0F0BD01AAF8
:101380000221284624F020FC019B186851F0EEF859
:10139000041EB38801DB9C4204DB013B002240F2C7
:1013A0009461D7E7019B586851F0E0F8051EF38877
:1013B00001DB9D42D5DB013B002240F29A61C9E787
:1013C000384651F0D3F8B27B4FF0FF31C2F1200222
:1013D00021FA02F2A223002150F069F92A460346BD
:1013E0002146304648F0BEFF0E20C6E7F64D090004
:1013F0001C5C090095460900585109002DE9F04F81
:1014000093B00DAB0193684B009305231EF0D2FD02
:101410000D9D664940F26B3228461EF0B1FEDDF8A4
:101420003880624940F2E55240461EF0A9FEDDF8E0
:101430003C905E4940F2E65248461EF0A1FE109CE8
:10144000204625F083FA20B12146594850F02FFA62
:101450000446012120464EF045FF824660B92046F1
:1014600024F07AFCC388009352484FF40873432257
:1014700040F272413FF0FEFB119F0E2F13D04B49FB
:1014800040F27D4238461EF07BFE4146284607F07A
:101490005DFC4946284607F059FCAB7B102B04D075
:1014A00045483FF0F3FB0027EFE7EB880493002665
:1014B000049BB34203DC0D9813B0BDE8F08FAB89F9
:1014C000AA68734302EB83030593AB880693B8F8CD
:1014D0000C30D8F80820734302EB83030393B9F868
:1014E0000C30D9F80820734302EB8303089333B21E
:1014F0004FF0000B0B93069B5B4501DC0136D7E7F1
:10150000039B33F8024B03933FB10B9A0FFA8BF115
:10151000384648F0F1FE00283FD163BAADF82430D8
:10152000089B33F81B305ABAADF82820C3F3C40225
:10153000C4F304210792C4F3002242EA4102C3F338
:10154000042EC3F3002141EA4E014FF0400012FB8C
:10155000001207991AF80220C4F3C40CC3F3C003A5
:10156000C4F3C00443EA410344EA4C04402114FBA1
:101570000134099B1AF804406408E40244EA520466
:101580000A9AC3F34513C2F3451213FB01231AF859
:10159000033044EA431464BAA4B2059B23F81B4009
:1015A0000BF1010BA7E700BF9C2B0A00BCC509008B
:1015B00034C9090001510900D233090070B586B061
:1015C00003AB0193164B009303231EF0F3FC039E21
:1015D00014494FF4387230461EF0D2FD049D124972
:1015E00040F2E94228461EF0CBFDA86840F2E942ED
:1015F0004FF480711EF082FD059C0E2C0DD0094920
:1016000040F27D4220461EF0BBFD30466A6821460E
:1016100037F0CEFB039806B070BD0024F5E700BF9D
:10162000D42B0A00BCC5090018C509002DE9F04FEC
:10163000A7B003AB01934B4B009303231EF0BAFCFE
:10164000039D49494FF4387228461EF099FD049CC9
:10165000204624F081FBC37B002B40D000EB8300AD
:10166000424B02699A423AD1606840F272420321C9
:101670001EF044FDD4E90378A4680DF11809002692
:10168000324621461F2058F0AFFC444509F8010BB3
:1016900004D0324641461F2058F0A6FC0136202EC9
:1016A00089F85F00ECD10DF1370600242246394657
:1016B0003F2058F099FC0134402C06F8010FF5D179
:1016C000059F0E2F0ED0284940F27D4238461EF06D
:1016D00057FDAB7B102B07D025483FF0D7FAA0462B
:1016E0002746CAE70027F4E7B5F806900026B1457B
:1016F00003DC039827B0BDE8F08FAB89AC68B5F880
:1017000004A0734304EB83044FF000080FFA86FB38
:10171000C24501DC0136EAE737B15A460FFA88F1D3
:10172000384648F0E9FDC8B9228853BAC3F34513D7
:1017300098336B4413F8601CC2F30423C2F3C40251
:10174000983398326B446A4413F8203C12F8802C8A
:1017500043EAC22343EA41135BBA238008F101083C
:101760000234D5E7EC2B0A00BCC509001183050043
:10177000D23309002DE9F04FABB00FAB0193924B80
:10178000009303231EF016FC0F9C90494FF438720F
:1017900020461EF0F5FC3022002112A84FF0FBFD80
:1017A000109E16F0030566D13368894A934224D10E
:1017B00012AF294630464EF0DBFB01353B46032D88
:1017C00007F1140783ED000AF3D1119F0E2F63D0A8
:1017D0007E4940F27D4238461EF0D2FC12AD0DF13A
:1017E00078080026731E0B2B71D8DFE803F06D70AC
:1017F000686A706A57706D706873764A934217D141
:101800000DF148084746294630464EF0B1FB4346A5
:10181000691C83ED000A30464EF0AAFB0235062D06
:1018200087ED030A08F1140807F11007EBD1CCE7A4
:10183000694A934211D14FF00308294630464EF0D1
:1018400097FBB5FBF8F72AAB2F44013503EB87076D
:10185000092D07ED180AF0D1B7E7604A93420AD183
:1018600012AF294630464EF083FB01350C2DA7EC14
:10187000010AF6D1A9E7304624F06EFAC388019335
:1018800040F21113009356484FF488734FF40F72CF
:1018900040F23B213FF002FA00279FE7514BB5ECA5
:1018A000010A07EE903AF8EEE77A013627EE800A51
:1018B00035F072FDBDEEC00AA8EC010A92E74A4B72
:1018C000EDE74FF40033EAE74FF40043E7E74FF466
:1018D0008033E4E7A37B102B02D044483FF0D6F9D5
:1018E0001E9B02931F9B0393209B0493219B0593B4
:1018F000229B0793239B0893249B0993259B0A9380
:10190000269B0B93279B0C93B4F80690289BDDF83D
:10191000A4A00D930026B14503DC0F982BB0BDE8C1
:10192000F08FA389A568B4F804B0734305EB830571
:101930004FF0000832B2C34501DC0136EBE747B196
:101940000FFA88F13846069248F0D6FC069A00282D
:1019500035D1B5F800C0039B9CFA9CF1C1F3451149
:1019600003FB01F0029BCCF3C40E03FB0E00049BAF
:10197000CCF3042C03FB0C00059BC3180693089BB7
:1019800007984B4300FB0E33099800FB0C330A9871
:1019900003440C9841430B9800FB0E110D9800FB7B
:1019A0000C110698A3F306435144A0F305405B01D4
:1019B00043EAC023A1F305410B435BBA2B8008F136
:1019C00001080235B7E700BF1C2C0A00BCC509009E
:1019D00060CA090010CA0900B4C909004CC909004D
:1019E0003B330900C1FF3E00E1FF1E00D233090076
:1019F0002DE9F04F2DED028BA7B002AF07F1700378
:101A000001938F4B009308231EF0D4FAD7F870B0DF
:101A10008C494FF4387258461EF0B2FBD7F88C3020
:101A20003B660E2B1CD0874940F27D4218461EF0C3
:101A3000A7FBF86F24F006F9D7F874804046F0EE63
:101A4000408A25F043F8C4070DD4404624F084F9B9
:101A500040F24122C3887C4840F282613FF01EF987
:101A600000233B66E5E7441007EE904AB8EE677A3C
:101A7000F1EEC77AFDEEE77A17EE905AE90703D543
:101A800005FB05F39C4202D070483FF0FFF8A3002D
:101A9000073323F00703ADEB030D02AB4FF0000952
:101AA0007B654E46A1451AD1B86F0E2828D024F088
:101AB000C9F8B0EE408A6B08FB6697F880307B630C
:101AC00097F884303B6397F88830FB62FB6E0133F4
:101AD000BB669BF80E30102B1FD05D48D5E74FEA50
:101AE0004901042241F00101404626F059FB50F023
:101AF0003DFD7B6D064443F8290009F10109D1E75A
:101B0000B7EE007A36B107EE906AF8EEE77A87EE24
:101B1000278AD0E7B0EE478ACDE7BBF804304D4DB9
:101B20004D4CD5F800A001335B10BB65BA6DBB6EA0
:101B300002FB03F6B60040D1BAF1000F02D05046C6
:101B400032F0D2F9002323602B609A469FED430ABE
:101B500028EE000A35F020FCFDEEC07A9FED400A29
:101B6000C7ED127A28EE800A35F016FCFDEEC07A39
:101B7000BBF806303B6217EE903A5B007B61FB6E70
:101B8000C7ED117A5B42FB65FB6E5B003B614FF07A
:101B900000093B6A4B4500F3D181BBF80650FB6E50
:101BA000EC1A24EAE474A54200F33383386F9437C7
:101BB000BD46BDEC028BBDE8F08FBAF1000F00F01E
:101BC000B38123689E42C1D9264B1C6820465AF037
:101BD0006CFD864280F09F8155460C2E55F8043DE1
:101BE000B04623F0030938BF4FF00C08C14580F020
:101BF0009B8005EB09004168CA0706D521F0030167
:101C000009F104030B4443452ED2314620465AF0D5
:101C100053FD0546002800F07E81B1454A465146F5
:101C200028BF32464FF076FB514620463DF0EEFB92
:101C3000AA46084BC3F800A0074B1E6086E700BF0A
:101C40001C2B0A00BCC50900E650090050330900EE
:101C5000D2330900F8660120FC66012000008047AD
:101C600000007C4A085C0120638AC3F3C7139942D1
:101C7000AAF1080980F007812269C2F38532B3FB1B
:101C8000F2F30022B1FBF3F37B66D0E902C1CCF89A
:101C90000C10C1F808C021697B6ED4F820E0C1F3B4
:101CA000853102FB01315EF8213098421AD1A445FA
:101CB0004EF821C016D1D4F81CE07B6E5EF82210DD
:101CC0004FF0010C0CFA03F321EA03014EF8221045
:101CD000E36953F822302BB9A3690CFA02FC23EA1A
:101CE0000C03A3615AF8043C4268043322F0030257
:101CF00013444AF8043C23F0030343F80590BA4B1D
:101D00001BB101221021AFF300805AF8043C23F0EC
:101D100003032B445A6822F002025A605AF8043C2A
:101D200023F001034AF8043C23F0030308F11002F6
:101D30009342FFF47EAF4544A3EB08036A68043B7B
:101D400002F0030213436B605AF8043C03F00303F0
:101D500043EA08034AF8043C6B6805F1080E23F0D7
:101D60000303734443F8045C53F8042942F002026D
:101D70005A60686820F0020320F0030043F001037A
:101D800070446B6050F80419CB074DD5638A21F07D
:101D90000301C3F3C7138B4240F28E8022694FF0D8
:101DA000000CC2F38532B3FBF2F3B1FBF3F37B66B5
:101DB000D0E90212CA60916022697B6ED4F820904B
:101DC000C2F385320CFB023259F82230984219D105
:101DD000A14249F8221015D1D4F81C807B6E58F826
:101DE0002C20012101FA03F322EA030248F82C20F7
:101DF000E36953F82C302BB9A36901FA0CF123EAFB
:101E00000103A3616B684268043322F003021344A8
:101E10006B6023F003039E44734B4EF8045C1BB1CC
:101E200001221021AFF300806968638A206921F0E4
:101E30000301C3F3C7139942C0F3853053D2B3FBF8
:101E4000F0F3B1FBF3F30022216A02FB003051F8FA
:101E50002010C5E90214CD602169206AC1F38531E3
:101E600002FB013140F821500125A16905FA02F079
:101E70000143E069A16150F8221005FA03F3194308
:101E800040F82210D5E6A9B1B1FA81F2C2F12002E0
:101E900094F812C0531ECCF3021CA3EB0C0321FADE
:101EA00003F3012101FA0CF14B40217C7B66A2EB8C
:101EB0005112EAE60A46EBE799B1B1FA81FCCCF19E
:101EC000200CA27C0CF1FF33C2F302129B1A21FA00
:101ED00003F301219140227C4B407B66ACEB521C0A
:101EE00066E78C46EDE7A1B1B1FA81F2C2F12002BA
:101EF00094F812C0531ECCF3021CA3EB0C0321FA7E
:101F000003F3012101FA0CF14B40217CA2EB5112A9
:101F10009AE70A46ECE7504631F0E6FF334B0022E1
:101F20001A6030463EF01CFE304632F08DF82660D6
:101F30008246286000287FF409AEF2E7BBF80C3037
:101F4000DBF8082009FB03F302EB8303BA6EFB63A3
:101F5000BB6EB9FBF3F302FB1393BA6D53430AEB69
:101F60008303FB61BBF80430BB613B690133BB6396
:101F7000FB6EA9EB0303BB600FFA89F34FF0000877
:101F80007B60BB6943451DDCFB6E4B4517DCBBF832
:101F90000C00BD6EBC6EBBF80420A9EB03014843E6
:101FA000B1FBF4F405FB1411BC6DDBF808306143A0
:101FB00052000AEB810103EB80004FF0ABF909F10D
:101FC0000109E6E53B6E9BB17A680FFA88F1184685
:101FD00048F092F960B1FB6B33F81830FA6922F8D7
:101FE000183008F10108CCE700000000F866012075
:101FF000DBF808103964BBF80C103965F96EBBF8D2
:102000000430BBF80620414500F3BC80591A8845CE
:1020100080F2B880F96E494500F3B480511A8945C1
:1020200080F2B080BB683A6DD7F85CC002FB03F465
:10203000A300FB643B6C002003EB4803BB62024639
:10204000786601467B6DFC6CFE6D03EB80033B64A0
:10205000BB6A23447B627B6A33F816503B6C53F8AF
:1020600004EB3B646CBAC5F3C4030EFB0311C4F369
:1020700045137C6E0EFB03437B66FB6E0136C5F396
:102080000425B3420EFB0522E5DABB6B1844D7E901
:10209000134304EB8303FB64FB6E0CF1010C6345FB
:1020A000D0DAD7E911307C6E01FB00317B6904FB8B
:1020B0000033D7E91104A3F3064302FB0402A1F3A2
:1020C00005415B01A2F3054243EAC12313437A6B46
:1020D000002A54D01D1205F0F8027A66DA1002F0D8
:1020E000FC01DB003965D9B2F964F96B31F81800ED
:1020F00041BAC1F3CC0606F0FC043C64FC6CC3F3AB
:10210000421323437C6EC5F3421525433C6DC2F355
:102110008112224302EB8202C2EB0212262415FB3B
:1021200004254FF00F0413FB04533C6C3A6BC6F3C9
:102130008116344300F0F80CC900C0F3421004EBE0
:10214000840401F0F80E4CEA0000C1F34211C4EB24
:1021500004144FF02605C2EBE3134EEA01010F22EF
:1021600010FB054011FB0201B3EBE11FF96AB4BF9C
:10217000012200224FF6FF738A4208BF00235BBA98
:102180009BB22BE70024013A013BFE6DBA627B62F1
:1021900022467C662146BB6AD7F85CC009EB060084
:1021A00020EAE0709842A8BF18463B6D4343FB60AD
:1021B0007B6D03EB8403FB647B6A08EB0C0525EA6B
:1021C000E5759D42A8BF1D463B6C03EB4505FB68CA
:1021D00035F82350FB6C53F804EBFB6468BAC5F385
:1021E000C4030EFB0311C0F34513786E0EFB03030B
:1021F0007B66FB6E0CF1010CC5F3042563450EFBF9
:102200000522D9DABB6B1C44FB6E0136B342C2DA3D
:1022100047E7BE6EBBF80C00B96EB4FBF1F106FBEC
:102220001141BE6DDBF80830BBF8042060437143F8
:1022300052000AEB810103EB80004FF06BF8013490
:10224000B1E400BF2DE9F04F2DED028B89B005AB55
:1022500001935E4B009303231DF0ACFE0698C8B1BA
:1022600023F0F0FCB0EE408A059C59494FF43872D7
:1022700020461DF085FF079F0E2F0ED0544940F2D7
:102280007D4238461DF07CFFA37B102B07D05148C0
:102290003EF0FCFCB6EE008AE6E70027F4E79FED8F
:1022A0004E0A28EE000A35F077F8B4F806A0BDEE25
:1022B000C08A00264FF0260B4FF04009B24505DCDE
:1022C000059809B0BDEC028BBDE8F08FA38803939D
:1022D000A389A568734305EB83054FF00008039BB2
:1022E000434501DC0136E9E73FB132B20FFA88F12C
:1022F000384648F001F8002864D129884BBA01F02B
:10230000F802C1F342111143C3F3CC0202F0FC0CFA
:10231000C2F3811242EA0C00DB0000EB800203F002
:10232000F80EC2EB0212C3F3421343EA0E034FF05E
:102330000F0C18EE10EA11FB0B2213FB0C22BEEB64
:10234000E21F4FEAE21C3DDACCEB4E024FF6D57CA1
:1023500010FB0CFC4FF6EB7E11FB0ECC4FF6CA7E49
:1023600010FB0EF011FB09014FF6F67013FB09CCC0
:1023700013FB0013DB114BF2D2614FEAEC1C594303
:1023800045F61A0000FB0C11144882F30802A2EB78
:102390002141434302EB2343114881F30801C90063
:1023A00083F3080301F4FC6100EA03230B430D49A6
:1023B00001FB0CFC02EB2C4282F3080243EAD2033D
:1023C0005BBA2B8008F10108023588E7042C0A006B
:1023D000BCC50900D233090000008043E966010052
:1023E00000F8FFFFA2C501002DE9F04F2DED028B93
:1023F0009FB014AB0193A94B00930A231DF0DAFDA3
:10240000A74914984FF45B721DF0BAFEA44940F23C
:10241000D752074615981DF0B3FEA14983464FF4E5
:10242000BB6216981DF0ACFE049018980E2836D0AA
:1024300023F008FCF0EE408A19980E2832D1B7EE4E
:10244000008A38EE688A179E964940F22932304653
:102450001DF096FE1A9D944940F2EE2228461DF08A
:102460008FFEBB88BBF80410994215D1FA88BBF8DF
:102470000630934210D1B87B9BF80E2082420BD1DC
:1024800004988088884207D10499C988994203D169
:10249000049B9B7B93420AD084483EF0F7FBF6EE08
:1024A000008AC9E723F0CEFBB0EE408ACBE734794F
:1024B000092C0EDC0121A14011F0AA0F05D1092C35
:1024C00007D1082B07D07A48E7E7102B03D07948CB
:1024D000E3E77948E1E71B98B5F904500E281FD0CF
:1024E00050F044F80023089009931C980E281CD043
:1024F00050F03CF800230A9005931D980E281ED03A
:1025000040F27D4266491DF03BFEBB8882889A42BC
:10251000804603D1C288FB889A420BD06748BCE74B
:1025200000230121CDE90831DFE7012305930023D2
:102530000A93E2E7837B082B03D06148ADE74FF0B5
:102540000008EBB20B93BB88ADF848300025FB8840
:10255000119511A93846ADF84A3013950FF0BEFF1A
:10256000F0EE687AFEEECC7A092CCDED027AF0EE30
:10257000487AFEEECC7ACDED067A40F0BD809DF82B
:10258000203007939DF828300699089378E0BA899F
:10259000BB68DBF808406A4303EB820ABBF80C30E7
:1025A0006B4304EB83030393049B9A899B686A4300
:1025B00003EB8202B8F1000F00F09C80B8F80C0029
:1025C000D8F80830684303EB8000D64652E0099BF8
:1025D000002B5ED1039B079E1B789B1B18BF01231A
:1025E000059E002E57D11678089C361B18BF012671
:1025F00070B190F800C00699BCF1000F0CBF002626
:1026000006F0010601FB0CF17F31FF2491FBF4F190
:10261000002B63D0039C14F8013B0394029C63439A
:10262000002E57D00B9C12F8016B012C01FB06F613
:1026300048D106FB03FC0CF57F4909F1FF093CEA90
:102640002C0C28BFCC461E44A6EB2C46029B4B43C9
:102650009C4648BF03F1FF0C029B0B44A3EB2C23C9
:10266000002B45DD96FBF3F383F308030EF8013BE3
:1026700000B10130BE88AEEB0A039E42A7DC0135F3
:10268000FB889D4283DB0E201FB0BDEC028BBDE8B2
:10269000F08F0123A4E7059EAAE700BFB42C0A002F
:1026A000BCC5090084C5090088C80900C44E0900DA
:1026B000524B0900374B0900C4430900D0490900B7
:1026C000E3490900C1F58074634348BFFF3306EB5B
:1026D0002326BBE7002B06DAFF3304E02EB112F805
:1026E000013B4B43F8D41B12BEE79EF80030BBE71A
:1026F0000023B9E7404668E704F0FB03069E0D930C
:10270000FB889D42BFDABA89BB686A4303EB820348
:10271000BBF80C200C93DBF808306A4303EB820310
:102720000E93049B9A899B686A4303EB82030F9381
:10273000B8F1000F00F00481B8F80C20D8F8083088
:102740006A4303EB820307930023A7E00E9B039ADF
:10275000039933F812200F9B33F811100D9B032BB4
:10276000099B01BF52BA49BA92B289B2002B40F01C
:102770009D80089BB3EB020C18BF4FF0010C059B2A
:10278000002B40F096800A9B5B1A18BF0123079824
:1027900080B10446069814F801EB079400FB0EF68E
:1027A000BEF1000F0CBF002303F001037F36FF20B2
:1027B00096FBF0F6BCF1000F00F0A880002B00F0B3
:1027C0008E80029B0298734348BFFF3300EB0609DB
:1027D000A9EB2329B9F1000F5EDD1312D410D2004A
:1027E00003F0F80304F0FC04D2B2434344434243F1
:1027F0000B984FEA212E4FEAE10CC9000EF0F80EBB
:102800000CF0FC0CC9B2012806FB0EFE06FB0CFC0A
:1028100006FB01F14FD10EFB03FA0AF57F40FF30B2
:102820003AEA2A0A28BF824673440CFB04FEA3EB53
:102830002A430EF57F4A0AF1FF0A3EEA2E0E28BF10
:10284000D646644401FB02FCA4EB2E440CF57F4EFB
:102850000EF1FF0E3CEA2C0C28BFF44602EB010AF5
:10286000AAEB2C4A0D9A93FBF9F394FBF9F41B02A3
:10287000E40003F4784304F4FC6423439AFBF9FA7C
:10288000032ACAF3C40A43EA0A0301D15BBA9BB222
:102890000C9A039922F81130039B01330393039A96
:1028A000BB889A42FFF652AF013529E74FF0010C81
:1028B00065E7059B6BE7C6F5807A5046434348BF02
:1028C000FF33444348BFFF345043024648BFFF3202
:1028D0000EEB23230CEB242401EB222AC2E7029BFC
:1028E000029802F47841594302F4FC6343434FEAEF
:1028F000212148BFFF3341EA2323029902F01F023E
:102900004A4348BFFF3243EA2223C0E79BB101F4A8
:10291000784201F4FC63734306FB02F201F01F01ED
:1029200048BFFF331212714342EA232348BFFF31ED
:1029300043EA2123ABE70C9B039A33F81230A7E755
:10294000CDF81C8000E700BF2DE9F04F99B011AB26
:1029500001933F4B009307231DF02CFB3D49119839
:102960004FF438721DF00CFC054605220BA9129895
:1029700021F0A4F8EB88AA8813A909A801F0DEFACF
:10298000BDF92830BDF92690BDF924A0BDF92AB0C3
:102990000493A3EB0A049DF83410ABEB0903002267
:1029A00040205C431DF04AFC0C9BB3FBF0F6179BE8
:1029B00005900E2B4F46039308D018464FF0D6FDD6
:1029C0000690B44205D924483EF0F0F8002306935F
:1029D000F7E7AB7B0B9C01269E40013EBB4534DCF8
:1029E000049BADF83C30284600230EA9ADF838A072
:1029F000ADF83A90ADF83EB010930FF06FFD0E2099
:102A000019B0BDE8F08F059B022B18D0042B19D00C
:102A100014F8013B03990E2902D00699994207D078
:102A200033400FFA88F1284607920FF07BFD079A92
:102A300008F10108049B4345E5DC0137CEE734F893
:102A4000023BE7E754F8043BE4E7D0463AB2F1E74B
:102A5000C42D0A00BCC50900DF3B09002DE9F04F79
:102A600097B002AF07F140030193B54B00930423E5
:102A70001DF0A0FAB349786C40F2D6521DF080FBED
:102A8000B04906464FF45B72386C1DF079FBFC6C64
:102A9000AD4981464FF42A7220461DF071FBBD6C92
:102AA000AA4940F2DB5228461DF06AFBB9F804A09F
:102AB000B388534509D1D9F80430BB60B9F8063062
:102AC000BB61BA69F388934202D0A1483EF0CAF8CC
:102AD00099F80E30102B03D0012B01D09D48F5E75B
:102AE0002A79092A06DC0121914011F0AA0F03D1AD
:102AF000092A06D09848E9E7B37B102B06D09748FF
:102B0000E4E7B37B082B01D09548DFE7032AB4F94B
:102B1000043053D0072A4FD0052A52D1002242F068
:102B2000020B904ADBB252F8235069780AEB41035A
:102B300003EB43035B0007336A46DB08A2EBC303E6
:102B40009D460A2301EB41084B4302AC03EB8A0389
:102B5000D04404EB410204EB48081C440AF11F0373
:102B600068465B09A0EB43139D46BA62C7F82C8008
:102B70003C6343F8081B30467B62594600234DF006
:102B80002FF86B78009342460123594630464DF0AA
:102B900027F86B78009322460223594630464DF0C1
:102BA0001FF84FF000084446BB69434540F3DC8002
:102BB000BB6A3B62002227E00122B0E74FF0010B25
:102BC000AFE74FF0000BACE73B6A786A33F912309D
:102BD00023447F2BD4BF00210121802B8154B4BF1B
:102BE0000021FF215B1AFB61E81C4FF0000C2978E3
:102BF0008C4544DBAC78FB6914FB03F4002CB8BFB4
:102C0000FF3444F30F2401329245DDDC7A6A4146F9
:102C100048465AF0C8FFFB6AFB61BB623B6B7B61B5
:102C2000FB623B6A3B6308F101037B60BB6908F10F
:102C30000102934200F098806B7800933A6A08F1A1
:102C40000303594630464CF0CBFF5246002A35D19B
:102C50007A6A796848465AF0A6FF7B69BB623B6A8C
:102C6000FB62FB693B636B780093FA6908F104032C
:102C7000594630464CF0B4FF08F1020894E790F949
:102C8000011090F9004007F1500303EB8101FB694B
:102C900051F8281C796190F90210144411FB03F1DA
:102CA0007B69002933F814E0B8BFFF310EEB212E09
:102CB000033023F814E00CF1010C98E7013AFB69AA
:102CC00033F81230234419B27F29D4BF00200120E9
:102CD00080297C6AB4BF0021FF215B1AA0543B61AC
:102CE000E81C4FF0000C29788C4509DBAC783B6977
:102CF00014FB03F4002CB8BFFF3444F30F24A5E702
:102D000090F9011090F9004007F1500303EB8101A5
:102D10003B6951F8281CF96090F90210141B11FB53
:102D200003F1FB68002933F814E0B8BFFF310EEB64
:102D3000212E033023F814E00CF1010CD3E700BF7F
:102D4000A42E0A00BCC509006CC8090084C509008E
:102D50002E41090085350900C23309007735090085
:102D60006E3509009C2E0A00BA68002307F1340171
:102D70004846C7E90E237B630FF0B0FB0E205437A3
:102D8000BD46BDE8F08F00BF2DE9F04395B00AAB1A
:102D90000193304B00930A231DF00CF92E490A9839
:102DA0004FF45B721DF0ECF940F2946382880446A4
:102DB00000210C984EF07BFCE28840F29A630021DF
:102DC00007460D984EF073FC234940F2D6528046D8
:102DD0000B981DF0D5F90546C38882880EA908A86E
:102DE00001F0ACF8A27BAB7B9A4202D21B483DF0CB
:102DF0004DFF12980E2825D04FF0B8FB4FF0000978
:102E0000064613980E2821D04FF0B0FB0023CDE9E1
:102E10000603BDF926300393BDF924300293BDF9B2
:102E200022300193BDF9203000932046CDE904699A
:102E30000FFA88F33AB2294606F076FD0E2015B057
:102E4000BDE8F0834FF001090026DAE701230020F6
:102E5000DDE700BF242E0A00BCC509009535090036
:102E60002DE9F04F91B00BAB0193974B00930523E5
:102E70001DF0A0F84FF45B7294490B981DF080F997
:102E80000E9B827B029301239340029A9A4206464C
:102E900002D38F483DF0FAFE0F9F6FF00042974239
:102EA00003D0BB4201D88B48F4E7BDF93090B9F1AB
:102EB000000F02DBB388994501DB8748EAE7BDF9DB
:102EC0003480B8F1000FF8DBF3889845F5DA029BFF
:102ED000BB4200F0F58000201AF08EFC0546484603
:102EE0004FF05FFF069040464FF05BFF06A907904A
:102EF000022024F0E9F8014628464FF07DFE6FF0ED
:102F000000439F420CD106984FF030FB04460798CF
:102F10004FF02CFB21B202B2304647F0EDF90746E4
:102F2000002304AA05A928460593CA464FF09AFE35
:102F3000CDF80C80059A8AB9039BADF820900AF170
:102F4000010A013308A93046ADF82280ADF824A06B
:102F5000ADF826300A920FF0C1FAB1E004AA05A933
:102F600028464FF07FFE0021284623F0F9FD044655
:102F700080684FF0FBFA8346E0684FF0F7FA0FFAEB
:102F80008BF102B2304647F0B7F9B84205D004AA37
:102F900005A928464FF066FECCE7A0684FF087FCF5
:102FA0008346E0684FF083FCCB45039BB8BF0FFA24
:102FB0008BF9D345C8BF0FFA8BFA4045B8BF0FFA5B
:102FC00080F89842C8BF03B2A068C8BF03934FF00F
:102FD000CDFA8346E0684FF0C9FA029B02B20FFABD
:102FE0008BF130460FF09EFAE0684FF060FC00284D
:102FF00011DDA3680893E0684FF059FC01384000E8
:1030000040F00100099008A9022024F05DF8014673
:1030100028464FF0F1FDA0684FF049FC002811DD73
:10302000A0684FF044FC0138400040F001000890D7
:10303000E368099308A9022024F046F801462846CF
:103040004FF0DAFDA0684FF032FCB38801309842AF
:1030500011DAA0684FF02BFC0130400040F0010075
:103060000890E368099308A9022024F02DF801468E
:1030700028464FF0C1FDE0684FF019FCF38801309D
:10308000984211DAA3680893E0684FF010FC013011
:10309000400040F00100099008A9022024F014F833
:1030A000014628464FF0A8FD04AA05A928464FF07E
:1030B000D9FDFDF7B5FD094B9B6A002B3FF43AAFF4
:1030C0000E2011B0BDE8F08F342D0A00BCC50900F8
:1030D000713309005D410900EA360900BC62012034
:1030E0002DE9F04F93B00DAB0193714B0093052385
:1030F0001CF060FF4FF45B726E490D981DF040F8B4
:10310000827BDDF84480012393409845044602D336
:1031100069483DF0BBFDBDF938A08288BDF940602B
:1031200040F29463002150464EF0C1FABDF93C9044
:10313000E28840F29A63002148464EF0B8FA40F225
:103140002652002130464EF0AAFA0EAA8CCA00255B
:10315000D11BCDE909553A44ADF81C10D91B3B44AD
:10316000ADF82020ADF82230A388ADF81E1007AAD4
:103170001046ADF82C300AA9E388ADF82E300C9536
:1031800049F036FF07A920460FF0A8F94B4940F255
:10319000946347F6FF7250464EF089FA40F29A6304
:1031A00047F6FF72454948464EF081FAA088E2880A
:1031B00050454FEA4703A8BF5046C3F103034A45B1
:1031C0001BB200B2A8BF4A4612B2039320EAE073D2
:1031D000049322EAE277B54203DD0E2013B0BDE886
:1031E000F08F049B06EB070B05EB03090FFA8BF23C
:1031F0000FFA89F1434620460FF094F9049BA7EBA0
:10320000060A591B09B20FFA8AF243462046059175
:103210000FF088F90FFA8BF20599434620460FF01C
:1032200081F90FFA8AF20FFA89F1434620460FF02E
:1032300079F9049B05EB070B03EB06090FFA8BF2F8
:1032400043460FFA89F120460FF06CF9049BA3EB7B
:10325000060A0FFA8BF24346A7EB050B0FFA8AF129
:1032600020460FF05FF943460FFA8BF20FFA8AF10E
:1032700020460FF057F90FFA8BF243460FFA89F107
:1032800020460FF04FF9039B002BC5BF039BAA1BE1
:1032900006330A33D2BF03EB850303EB820306F147
:1032A000FF361BB2C8BF36B20393013593E700BFA8
:1032B000742E0A00BCC50900EA3609000080FFFF31
:1032C0002DE9F0438FB008AB01932A4B00930623FE
:1032D0001CF070FE4FF45B72274908981CF050FFF9
:1032E000827BDDF83490012393409945044602D354
:1032F00022483DF0CBFC0B98099A0C990A9B15B219
:1033000007B21EB20FFA81F8BD42B5BF421C384663
:10331000284601324645B4BF4B1C0133ADF80E3090
:103320004FF00003CDE90433ADF80C20A288ADF8CE
:103330001820E288ADF81A20B4BF3146414602AAEF
:10334000ADF80800ADF80A10104605A9079349F03A
:103350004FFE02A920460FF0C1F82046CDE90089B2
:103360003B46324629464AF072FF0E200FB0BDE8B8
:10337000F08300BF042D0A00BCC50900EA3609002D
:103380002DE9F04F9FB019AB01935B4B00930523E0
:103390001CF010FE594919984FF45B721CF0F0FEB6
:1033A000052210A906461A9820F088FB05220DA9CF
:1033B0001B9820F083FB9DF84810002240201CF051
:1033C0003DFF9DF83C100546002240201CF036FFD2
:1033D000854202D04A483DF059FC119BB3FBF5F3FE
:1033E0000993099A0E9BB3FBF5F39A4201D0454825
:1033F000F1E71C9B0293B37B029A012404FA03F3C6
:103400009A4201D34048E6E79DF874300A93109B36
:1034100007932A460D9B0798089300214DF0E5FA83
:103420002A4607B2002108984DF0DFFA0FFA80F81B
:10343000CDE90378C246CDF81880BB460597099BB5
:10344000A3422BD80A9B43B1029BDDE90312CDE9CD
:10345000008330463B464AF0FAFE059BADF84C30FF
:10346000069BADF84E300023CDE91533ADF852A0E0
:10347000ADF850B0B288ADF85C20F288ADF85E20AF
:1034800013AA16A91046189349F0B2FD304613A9A5
:103490000FF024F80E201FB0BDE8F08F21460798EA
:1034A0002A464DF0A2FA214603B22A4608980B9309
:1034B0004DF09BFA029B0FFA80F9CDE90093DDE90C
:1034C00003120B9B30464AF0C2FE0B9B059A9A42B0
:1034D000D4BF059205939B45069AB8BF9B464A45C3
:1034E000D4BF0692CDF81890CA45CDE90339B8BFCC
:1034F000CA460134A3E700BFFC2D0A00BCC5090081
:10350000FD4C0900124D0900EA360900F0B591B0F2
:103510000AAB0193274B009306231CF04BFD4FF49D
:103520005B7225490A981CF02BFE827B0F9F0123BA
:1035300093409F42044602D320483DF0A7FB828877
:10354000C3880BA902A800F0F9FC029B0493002594
:10355000039B059304A8069549F039FDA388ADF8AF
:10356000203004AAE388079507A91046ADF8223059
:10357000099549F03DFD04A920460EF0AFFFBDF9C5
:103580001050BDF91430AB4202DC0E2011B0F0BD7A
:10359000BDF91260BDF91630B34202DC01352DB21F
:1035A000EFE732463B462946204601360EF0BAFF89
:1035B00036B2EFE75C2D0A00BCC50900EA36090007
:1035C0002DE9F04786B003AB01931F4B0093032313
:1035D0001CF0F0FC4FF438721C4903981CF0D0FD2D
:1035E000827BDDF81090012393409945044603D275
:1035F000DDF814A09A4524D315484FF449713DF0E5
:103600004DFB3A462946204646F076FE814505D1D7
:1036100053463A46294620460EF084FF08F1010839
:10362000E3880FFA88F79F42EBDB0136A38835B2B7
:103630009D4203DB0E2006B0BDE8F0874FF0000886
:10364000EEE70026F2E700BF9C2C0A00BCC509008B
:10365000E05009002DE9F04F2DED0C8B99B00BAB2C
:1036600001930D4B00930D231CF0A4FC0B490B9808
:103670004FF45B721CF084FD40F2D652804607493D
:103680000C981CF07DFD98F80E20837B9A4207462B
:1036900008D203483DF0FAFA342C0A00BCC50900F0
:1036A00095350900B8F804100D98490859F094FEB2
:1036B000B8F806100DEE100A49080E9859F08CFE65
:1036C000B9880CEE100A4908119859F085FEF9885E
:1036D0000BEE900A4908129859F07EFE0023109CC8
:1036E000009307AA0DF11E010BEE100A0F9811F0BE
:1036F00057F9B8F90620B8F904300092204606AA16
:103700000DF11A0111F04CF9BDF91E20BDF91A0096
:10371000824206DD1346ADF81E00ADF81A200246BF
:103720001846BDF91C30BDF918108B4206DD1C4649
:10373000ADF81C10ADF818300B462146002ABCBF6E
:103740000022ADF81E20B8F80440002BBCBF0023B7
:10375000ADF81C30A242B8F80620C8BFADF81E4034
:103760009342C8BFADF81C2000284FF0000380F240
:103770001B829942ADF81A3002DAADF818301946BA
:103780008A424FF00003B8BFADF81820149C13987C
:10379000009305AA0DF1160111F002F9B7F9062000
:1037A000B7F904300092204604AA0DF1120111F07D
:1037B000F7F8BDF91620BDF91200824206DD134666
:1037C000ADF81600ADF8122002461846BDF91430C7
:1037D000BDF910108B4206DD1C46ADF81410ADF893
:1037E00010300B462146002ABCBF0022ADF816203F
:1037F000BC88002BBCBF0023ADF81430A242FA886D
:10380000C8BFADF816409342C8BFADF814200028D9
:103810004FF0000380F2D2819942ADF8123002DA03
:10382000ADF81030194615988A42B8BFADF810208F
:103830000E2800F0CD8122F005FAF0EE40CA16986D
:103840000E2840F0C881B7EE00AA17980E2800F0A5
:10385000CD814EF08BFE002383460293BDF91630D6
:10386000BDF91C20039208EE103ABDF91430BDF9E1
:103870001A60BDF91E90BDF918A008EE903ABDF986
:10388000123009EE103ABDF91030B0EE6C0A09EEB4
:10389000903A35F0BBFDF0EE40AAB0EE6C0A0CF0A9
:1038A00007FCF8EEEB4AB8EECB4A20EE647A2AEE3B
:1038B000843A27EE0A7A23EE0A3AF8EECD3A77EE0A
:1038C000035A6AEEE47A60EE046A02EE906A75EEDC
:1038D000A35A67EE8A7A66EE8A6AF8EEE22AB8EEB2
:1038E000CC5A37EEE66AF4EEE25AF1EE10FA36EE12
:1038F000056A039A40F17F81FDEEE52A12EE903AC7
:103900000FFA83FC02EE909AF8EEE22AF4EEE25A05
:10391000F1EE10FA40F37181FDEEE55A15EE903AA2
:103920001DB205EE90AAF8EEE55AB4EEE56AF1EEA6
:1039300010FA40F16481FDEEC65A15EE903A19B2C4
:1039400005EE902AF8EEE55AB4EEE56AF1EE10FACB
:1039500040F35781BDEEC66A16EE103A1CB2BB8822
:103960001BEE900A1B1A06EE103AB8EEC66A02EE7B
:1039700090CA60EE065A2AEE866A65EE8A5A26EEEC
:103980000A6A33EE253AF8EEE22A33EE233A76EE6F
:10399000666AB4EEE23AF1EE10FA76EE856A05D583
:1039A000FDEEC32A12EE903A0FFA83FC02EE905A13
:1039B000F8EEE22AB4EEE23AF1EE10FA04DDBDEEE2
:1039C000C33A13EE103A1DB203EE101AB8EEC33A22
:1039D000F4EEC36AF1EE10FA04D5BDEEE63A13EE4A
:1039E000103A19B203EE104AB8EEC33AF4EEC36AC5
:1039F000F1EE10FA04DDFDEEE66A16EE903A1CB226
:103A0000FB881BEE100A1B1A06EE903AF8EEE66AE7
:103A100002EE90CA2AEEA63A60EE266A23EE0A3A31
:103A200066EE8A6A75EEC35AF8EEE22A75EEA35A7C
:103A300036EE266AF4EEE25AF1EE10FA36EE056A38
:103A400005D5FDEEE52A12EE903A0FFA83FC02EE60
:103A5000905AF8EEE22AF4EEE25AF1EE10FA04DDA2
:103A6000FDEEE55A15EE903A1DB205EE901AF8EE0D
:103A7000E55AB4EEE56AF1EE10FA04D5FDEEC65A49
:103A800015EE903A19B205EE904AF8EEE55AB4EE0A
:103A9000E56AF1EE10FA04DDBDEEC66A16EE103AE4
:103AA0001CB277EEA67A37EE437A06EE90CA37EE6E
:103AB000237AF8EEE66A77EE857AB4EEE67AF1EEEE
:103AC00010FA05D5FDEEC76A16EE903A0FFA83FCA0
:103AD00006EE905AF8EEE66AB4EEE67AF1EE10FAE7
:103AE00004DDBDEEC77A17EE103A1DB207EE101ACC
:103AF000B8EEC77AF4EEC77AF1EE10FA04D5BDEE4F
:103B0000E77A17EE103A19B207EE104AB8EEC77A04
:103B1000F4EEC77AF1EE10FA04DDFDEEE77A17EE67
:103B2000903A1CB2CAEE8ABA731EE1451BB2B8BF06
:103B3000E146AE42D8BF1D468A42B8BF0A460AF1E6
:103B4000FF331BB2A245D8BF1C466B1CADF8243016
:103B5000631C80EE0ABAADF8263008A9002340465F
:103B60001646ADF82090ADF822200A9365EE2B7A28
:103B700025EE0B5AE3EE8B7AABEEE35A74EEE7AA2E
:103B800007EE902A34EE45AAF8EEE77AEBEEA7AA04
:103B9000ABEE27AA0EF0A2FCB44234DA0E2019B024
:103BA000BDEC0C8BBDE8F08F0029BCBFADF8183020
:103BB00019468442B8BFADF81A40E1E50029BCBF00
:103BC000ADF8103019468442B8BFADF812402AE66D
:103BD000DFED37CA33E622F035F8B5EEC00AF1EE74
:103BE00010FAB0EE40AA7FF530AE2CE60123029326
:103BF0004FF0000B32E6B44684E64D4691E651465E
:103C00009EE61446ABE607EE909AF8EEE77AB0EE41
:103C10006ACAF0EE4ACAABEE27CACA46EBEEE7CA5A
:103C2000554506DA01367AEEABAA3AEE0BAA36B261
:103C3000B2E7F8EEC87AF4EECC7AF1EE10FA2DD8AD
:103C4000F8EEC97AB4EEE7CAF1EE10FA26D5F8EE2E
:103C5000E87AF4EEEC7AF1EE10FA1FD8F8EEE97A91
:103C6000F4EEE7CAF1EE10FA18D5FDEEEC7A38461C
:103C7000CDED037AFDEECC7ABDF90C20CDED037AC3
:103C8000BDF90C1046F038FB029A03460AB9834589
:103C900004D03246514640460EF044FC0AF1010A77
:103CA0003CEE0BCA7CEEEBCA0FFA8AFAB8E700BF0B
:103CB000000000002DE9F04F9DB002AF07F14C036A
:103CC0000193974B009307231CF074F99549F86C06
:103CD0004FF438721CF054FABE6D731E012B8246ED
:103CE00005D9042E03D0904831463CF0D7FFD7F8D1
:103CF0005480B8F1020F05DCB8F1000F14DC8B48DA
:103D00004146F2E7A8F104031C2BF8D8884A0121A8
:103D100099400A4042B9142BF1D1012E04D08548B4
:103D2000182231463CF0BAFF3B6DBB6297F85C301D
:103D3000FB6297F860303B6297F86430FB619AF859
:103D40000E30B86A012101FA03F3013B7B611FF0D9
:103D500007FFBAF8043078600024A7F8443007F170
:103D60004001BAF80630A7F8463050463C64BC64BF
:103D70000EF0B4FBBAF804307C6308FB03F303EBEA
:103D8000C603F200013BB3FBF2F373433B6303331F
:103D900023F003037B623B6B013323F00103BB6120
:103DA0007B6A073323F00703BB60BAF806907B6B8E
:103DB000994504DC0E206C37BD46BDE8F08FBB682A
:103DC000C7F810D0ADEB030DFB6902AD9BB17B6B67
:103DD00009F1FF39A9EB03090023FB637B683A6B08
:103DE0005C68B86A294607F13C03A047F96B29B122
:103DF00008463CF003FFD7F83490EDE73B6B834275
:103E000002D04D4859F0D7F83B6A93B1022E0BD03F
:103E1000042E0ED17A6A2B46A918994209D01A6845
:103E200012BA43F8042BF8E7BA692B4651199942A4
:103E300010D108F1FF33AB460024FB600FFA89F97B
:103E4000BAF804309C420ADB7B6BD7F810D0013300
:103E50007B63AAE71A8852BA23F8022BE7E7B8F186
:103E6000080F08DCFA68072A0ED8DFE802F00F27EF
:103E70000D360D0D0D45B8F1180F42D0B8F1200FD9
:103E80004AD0B8F1100F39D0002309E0FA6AE310E4
:103E90008AB1E24302F00702EB5C134103F0010335
:103EA0007A6921B2134050464A460EF03BFB01347A
:103EB0000BF1030BC4E704F00702EDE7FA6AA31065
:103EC00042B1E24302F00302EB5C5200134103F003
:103ED0000303E5E704F00302F6E7FA6A631042B170
:103EE000E24302F00102EB5C9200134103F00F0386
:103EF000D6E704F00102F6E72B5DD1E735F8143080
:103F0000CEE79BF801309BF800201B0243EA0243F6
:103F10009BF802201343C3E755F82430C0E700BFE5
:103F20008C2D0A00BCC50900CB3A0900EC3A090007
:103F300011100010DE3A0900C459090073B5044697
:103F40000D461E466846084B44F026FF291D0DF11C
:103F50000200064B324644F01FFF6B4603CB206045
:103F60002046616002B070BD942B0A008C2B0A00C1
:103F70002DE9F04F0D4687B00021924629F042FB13
:103F800004460021284629F03DFB2379662B02D008
:103F90000379662B02D1C8483CF078FE00230390D9
:103FA00008208DF817304DF0C6F8074608204DF070
:103FB000C2F8064608204DF0BEF80399CDE900602E
:103FC00005463B460DF11702204654F0DEF80399F2
:103FD00050B9384613F04AFD304613F047FD2846E5
:103FE00013F044FDB548D7E70AF1FF3A9DF81700F2
:103FF000D4F81C90D1F81C802279BAF1030F05D8AF
:10400000DFE81AF0E901BD0398053B08AA46B3466C
:104010002379D4F81C90D1F81C80422B40F0C18049
:104020000A79422A3DD1394654F05CFAC269044605
:104030000020134698F800C099F8001001EA0C011E
:1040400003F8011BDAF80410D4F810C0DBF804E020
:1040500003918844991A8C45F144EBD8DBF80010A1
:10406000DAF800200CFB1E11894403990CFB112285
:104070009044E2680130904211D3384613F0F6FCC8
:10408000304613F0F3FC284613F0F0FC204607B04E
:10409000BDE8F08F5A461C46D3469246B8E71A460A
:1040A000C7E7622A28D13946682254F01BFAC16951
:1040B00004460023002298F900C099F8000000EAA5
:1040C0000C0021F8020B2069DBF804E0DAF804C0E8
:1040D00001328242F144E044EDD3DBF8002000FBE2
:1040E0001E229144DAF8002000FB1C229044E26872
:1040F00001339342DED3C0E7482A27D1394654F032
:10410000F1F9C169044600230022B8F800C099F80B
:10411000000000EA0C0021F8020B2069DBF804E043
:10412000DAF804C001328242F144E044EDD3DBF816
:10413000002000FB1E229144DAF8002000FB1C2224
:104140009044E26801339342DED396E7682A41F057
:104150003782394654F0C6F9C1690446002300226B
:10416000B8F800C099F8000000EA0C0021F8020B32
:104170002069DBF804E0DAF804C001328242F1443D
:10418000E044EDD3DBF8002000FB1E229144DAF876
:10419000002000FB1C229044E26801339342DED3EE
:1041A0006BE7622B40F08C800A79622A2CD1394669
:1041B00054F098F9C26904460020134698F800C0EC
:1041C00099F8001001EA0C0103F8011BDAF8041059
:1041D000D4F810C0DBF804E003918844991A6145D3
:1041E000F144EBD3DBF80010DAF800200CFB1E11D1
:1041F000894403990CFB11229044E26801309042FB
:10420000BFF43BAF1A46D8E7482A27D1394654F0C5
:1042100069F9C169044600230022B8F800C099F981
:10422000000000EA0C0021F8020B2069DBF804E032
:10423000DAF804C001328242F144E044EDD3DBF805
:10424000002000FB1E229144DAF8002000FB1C2213
:104250009044E26801339342DED30EE7682A0B46AE
:1042600021467FF417AF394654F03CF9C169044642
:1042700000230022B8F800C099F9000000EA0C0001
:1042800021F8020B2069DBF804E0DAF804C00132FF
:104290008242F144E044EDD3DBF8002000FB1E2213
:1042A0009144DAF8002000FB1C229044E2680133BC
:1042B0009342DED3E1E600BF3438090088370900B5
:1042C000482B57D10A79482A27D1394654F00AF9A0
:1042D000C169044600230022B8F800C0B9F8000004
:1042E00000EA0C0021F8020B2069DBF804E0DAF8A0
:1042F00004C001328242F144E044EDD3DBF80020F7
:1043000000FB1E229144DAF8002000FB1C2290449E
:10431000E26801339342DED3AFE6682A0B462146BA
:104320007FF4B8AE394654F0DDF8C1690446002385
:104330000022B8F800C0B9F8000000EA0C0021F82B
:10434000020B2069DBF804E0DAF804C00132824293
:10435000F144E044EDD3DBF8002000FB1E22914441
:10436000DAF8002000FB1C229044E26801339342FB
:10437000DED382E6682B41F023810A79682A0B4656
:1043800021467FF487AE394654F0ACF8C169044643
:1043900000230022B8F800C0B9F8000000EA0C00C1
:1043A00021F8020B2069DBF804E0DAF804C00132DE
:1043B0008242F144E044EDD3DBF8002000FB1E22F2
:1043C0009144DAF8002000FB1C229044E26801339B
:1043D0009342DED351E6AA46B3462379D4F81C9023
:1043E000D1F81C80422B40F0B5800A79422A31D1A5
:1043F000394654F077F8C26904460020134698F80D
:1044000000C099F8001041EA0C0103F8011BDAF82A
:104410000410D4F810C0DBF804E003918844991A22
:104420006145F144EBD3DBF80010DAF800200CFB17
:104430001E11894403990CFB11229044E26801305B
:104440009042BFF41AAE1A46D8E75A461C46D346E5
:104450009246C2E7622A28D13946682254F042F8CF
:10446000C16904460023002298F900C099F80000B1
:1044700040EA0C0021F8020B2069DBF804E0DAF8CE
:1044800004C001328242F144E044EDD3DBF8002065
:1044900000FB1E229144DAF8002000FB1C2290440D
:1044A000E26801339342DED3E7E5482A27D1394653
:1044B00054F018F8C169044600230022B8F800C07F
:1044C00099F8000040EA0C0021F8020B2069DBF8A3
:1044D00004E0DAF804C001328242F144E044EDD352
:1044E000DBF8002000FB1E229144DAF8002000FBDC
:1044F0001C229044E26801339342DED3BDE5682A72
:1045000041F05E80394653F0EDFFC1690446002357
:104510000022B8F800C099F8000040EA0C0021F829
:10452000020B2069DBF804E0DAF804C001328242B1
:10453000F144E044EDD3DBF8002000FB1E2291445F
:10454000DAF8002000FB1C229044E2680133934219
:10455000DED392E5622B40F087800A79622A2CD163
:10456000394653F0BFFFC26904460020134698F84D
:1045700000C099F8001041EA0C0103F8011BDAF8B9
:104580000410D4F810C0DBF804E003918844991AB1
:104590006145F144EBD3DBF80010DAF800200CFBA6
:1045A0001E11894403990CFB11229044E2680130EA
:1045B0009042BFF462AD1A46D8E7482A27D139465F
:1045C00053F090FFC169044600230022B8F800C0F0
:1045D00099F9000040EA0C0021F8020B2069DBF891
:1045E00004E0DAF804C001328242F144E044EDD341
:1045F000DBF8002000FB1E229144DAF8002000FBCB
:104600001C229044E26801339342DED335E5682AE8
:104610000B4621467FF419AF394653F063FFC16959
:10462000044600230022B8F800C099F9000040EACF
:104630000C0021F8020B2069DBF804E0DAF804C072
:1046400001328242F144E044EDD3DBF8002000FB6C
:104650001E229144DAF8002000FB1C229044E268FC
:1046600001339342DED308E5482B57D10A79482A13
:1046700027D1394653F036FFC16904460023002292
:10468000B8F800C0B9F8000040EA0C0021F8020BAD
:104690002069DBF804E0DAF804C001328242F14418
:1046A000E044EDD3DBF8002000FB1E229144DAF851
:1046B000002000FB1C229044E26801339342DED3C9
:1046C000DBE4682A0B4621467FF4BFAE394653F03F
:1046D00009FFC169044600230022B8F800C0B9F8F8
:1046E000000040EA0C0021F8020B2069DBF804E02E
:1046F000DAF804C001328242F144E044EDD3DBF841
:10470000002000FB1E229144DAF8002000FB1C224E
:104710009044E26801339342DED3AEE4682B40F06C
:104720004F870A79682A0B4621467FF48EAE3946B8
:1047300053F0D8FEC169044600230022B8F800C037
:10474000B9F8000040EA0C0021F8020B2069DBF800
:1047500004E0DAF804C001328242F144E044EDD3CF
:10476000DBF8002000FB1E229144DAF8002000FB59
:104770001C229044E26801339342DED37DE4AA46D2
:10478000B3462379D4F81C90D1F81C80422B40F01A
:10479000B7800A79422A31D1394653F0A3FEC26963
:1047A00004460020134698F800C099F8001081EAEA
:1047B0000C0103F8011BDAF80410D4F810C0DBF880
:1047C00004E003918844991A6145F144EBD3DBF886
:1047D0000010DAF800200CFB1E11894403990CFB31
:1047E00011229044E26801309042BFF446AC1A4670
:1047F000D8E75A461C46D3469246C2E7622A28D1D9
:104800003946682253F06EFEC16904460023002237
:1048100098F900C099F8000080EA0C0021F8020B1A
:104820002069DBF804E0DAF804C001328242F14486
:10483000E044EDD3DBF8002000FB1E229144DAF8BF
:10484000002000FB1C229044E26801339342DED337
:1048500013E4482A28D1394653F044FEC16904467E
:1048600000230022B8F800C099F8000080EA0C008C
:1048700021F8020B2069DBF804E0DAF804C0013209
:104880008242F144E044EDD3DBF8002000FB1E221D
:104890009144DAF8002000FB1C229044E2680133C6
:1048A0009342DED3FFF7E9BB682A40F08986394698
:1048B00053F018FEC169044600230022B8F800C076
:1048C00099F8000080EA0C0021F8020B2069DBF85F
:1048D00004E0DAF804C001328242F144E044EDD34E
:1048E000DBF8002000FB1E229144DAF8002000FBD8
:1048F0001C229044E26801339342DED3FFF7BDBB34
:10490000622B40F089800A79622A2CD1394653F013
:10491000E9FDC26904460020134698F800C099F8E2
:10492000001081EA0C0103F8011BDAF80410D4F836
:1049300010C0DBF804E003918844991A6145F14402
:10494000EBD3DBF80010DAF800200CFB1E118944D1
:1049500003990CFB11229044E26801309042BFF4AD
:104960008CAB1A46D8E7482A28D1394653F0BAFD0D
:10497000C169044600230022B8F800C099F900007C
:1049800080EA0C0021F8020B2069DBF804E0DAF879
:1049900004C001328242F144E044EDD3DBF8002050
:1049A00000FB1E229144DAF8002000FB1C229044F8
:1049B000E26801339342DED3FFF75FBB682A0B4600
:1049C00021467FF416AF394653F08CFDC169044689
:1049D00000230022B8F800C099F9000080EA0C001A
:1049E00021F8020B2069DBF804E0DAF804C0013298
:1049F0008242F144E044EDD3DBF8002000FB1E22AC
:104A00009144DAF8002000FB1C229044E268013354
:104A10009342DED3FFF731BB482B59D10A79482A9C
:104A200028D1394653F05EFDC169044600230022B7
:104A3000B8F800C0B9F8000080EA0C0021F8020BB9
:104A40002069DBF804E0DAF804C001328242F14464
:104A5000E044EDD3DBF8002000FB1E229144DAF89D
:104A6000002000FB1C229044E26801339342DED315
:104A7000FFF703BB682A0B4621467FF4BAAE3946DE
:104A800053F030FDC169044600230022B8F800C08D
:104A9000B9F8000080EA0C0021F8020B2069DBF86D
:104AA00004E0DAF804C001328242F144E044EDD37C
:104AB000DBF8002000FB1E229144DAF8002000FB06
:104AC0001C229044E26801339342DED3FFF7D5BA4B
:104AD000682B40F075850A79682A0B4621467FF4D9
:104AE00088AE394653F0FEFCC1690446002300221B
:104AF000B8F800C0B9F8000080EA0C0021F8020BF9
:104B00002069DBF804E0DAF804C001328242F144A3
:104B1000E044EDD3DBF8002000FB1E229144DAF8DC
:104B2000002000FB1C229044E26801339342DED354
:104B3000FFF7A3BA422A40F0A8800B79422B28D174
:104B4000394653F0CFFCC26904460020134698F85A
:104B500000C099F8001001FA0CF103F8011BD4F819
:104B600010C0D6F804A0D5F804E0991A6145D144E4
:104B7000F044ECD32A6831680CFB1E229044E268B2
:104B800001300CFB1A1190428944BFF476AA1A46F0
:104B9000DCE7622B27D16822394653F0A3FC044698
:104BA000C0690023002298F900C099F8001001FAAA
:104BB0000CF120F8021B2169D6F804E0D5F804C0F6
:104BC00001328A42F144E044EDD3326801FB1E22F7
:104BD00091442A6801FB1C229044E268013393420D
:104BE000E0D3FFF74ABA482B27D11A46394653F08B
:104BF00079FC0446C06900230022B8F800C099F887
:104C0000001001FA0CF120F8021B2169D6F804E02B
:104C1000D5F804C001328A42F144E044EDD3326851
:104C200001FB1E2291442A6801FB1C229044E26889
:104C300001339342E0D3FFF720BA6822394653F09C
:104C400051FC0446C06900230022B8F900C099F85D
:104C5000001001FA0CF120F8021B2169D6F804E0DB
:104C6000D5F804C001328A42F144E044EDD3326801
:104C700001FB1E2291442A6801FB1C229044E26839
:104C800001339342E0D3FFF7F8B9622A40F0A880DD
:104C90000B79422B27D16822394653F023FC044676
:104CA000C0690023002298F800C099F9001001FAA9
:104CB0000CF120F8021B2169D6F804E0D5F804C0F5
:104CC00001328A42F144E044EDD3326801FB1E22F6
:104CD00091442A6801FB1C229044E268013393420C
:104CE000E0D3FFF7CAB9622B28D1394653F0FAFB5B
:104CF000C26904460020134698F900C099F90010D3
:104D000001FA0CF103F8011BD4F810C0D6F804A086
:104D1000D5F804E0991A6145D144F044ECD32A68EF
:104D200031680CFB1E229044E26801300CFB1A1122
:104D300090428944BFF4A1A91A46DCE7482B27D149
:104D40001A46394653F0CEFB0446C06900230022C0
:104D5000B8F800C099F9001001FA0CF120F8021B14
:104D60002169D6F804E0D5F804C001328A42F14442
:104D7000E044EDD3326801FB1E2291442A6801FB16
:104D80001C229044E26801339342E0D3FFF775B9E7
:104D90006822394653F0A6FB0446C069002300226E
:104DA000B8F900C099F9001001FA0CF120F8021BC3
:104DB0002169D6F804E0D5F804C001328A42F144F2
:104DC000E044EDD3326801FB1E2291442A6801FBC6
:104DD0001C229044E26801339342E0D3FFF74DB9BF
:104DE000482A40F0A7800B79422B26D1394653F050
:104DF00079FB0446C0690023002298F800C0B9F886
:104E0000001001FA0CF120F8021B2169D6F804E029
:104E1000D5F804C001328A42F144E044EDD332684F
:104E200001FB1E2291442A6801FB1C229044E26887
:104E300001339342E0D3FFF720B9622B29D11A4600
:104E4000394653F04FFBC26904460020134698F9D7
:104E500000C099F9001001FA0CF103F8011BD4F815
:104E600010C0D6F804A0D5F804E0991A6145D144E1
:104E7000F044ECD32A6831680CFB1E229044E268AF
:104E800001300CFB1A1190428944BFF4F6A81A466F
:104E9000DCE7482B26D1394653F024FB0446C06991
:104EA00000230022B8F800C0B9F8001001FA0CF194
:104EB00020F8021B2169D6F804E0D5F804C00132BD
:104EC0008A42F144E044EDD3326801FB1E22914452
:104ED0002A6801FB1C229044E26801339342E0D32C
:104EE000FFF7CBB86822394653F0FCFA0446C06994
:104EF00000230022B8F900C0B9F8001001FA0CF143
:104F000020F8021B2169D6F804E0D5F804C001326C
:104F10008A42F144E044EDD3326801FB1E22914401
:104F20002A6801FB1C229044E26801339342E0D3DB
:104F3000FFF7A3B8682A40F043830B79422B394628
:104F400025D153F0CFFA0446C0690023002298F817
:104F500000C0B9F9001001FA0CF120F8021B216918
:104F6000D6F804E0D5F804C001328A42F144E044A6
:104F7000EDD3326801FB1E2291442A6801FB1C22FA
:104F80009044E26801339342E0D3FFF776B8622B96
:104F900025D153F0A7FA0446C0690023002298F9EE
:104FA00000C0B9F9001001FA0CF120F8021B2169C8
:104FB000D6F804E0D5F804C001328A42F144E04456
:104FC000EDD3326801FB1E2291442A6801FB1C22AA
:104FD0009044E26801339342E0D3FFF74EB8482B88
:104FE00025D153F07FFA0446C06900230022B8F9A6
:104FF00000C0B9F8001001FA0CF120F8021B216979
:10500000D6F804E0D5F804C001328A42F144E04405
:10501000EDD3326801FB1E2291442A6801FB1C2259
:105020009044E26801339342E0D3FFF726B853F08F
:1050300059FA0446C06900230022B8F900C0B9F942
:10504000001001FA0CF120F8021B2169D6F804E0E7
:10505000D5F804C001328A42F144E044EDD332680D
:1050600001FB1E2291442A6801FB1C229044E26845
:1050700001339342E0D3FFF700B8422A40F0A88002
:105080000B79422B28D1394653F02CFAC2690446D9
:105090000020134698F800C099F8001041FA0CF16E
:1050A00003F8011BD4F810C0D6F804A0D5F804E02A
:1050B000991A8C45D144F044ECD82A6831680CFB2D
:1050C0001E229044E26801300CFB1A119042894480
:1050D000BEF4D3AF1A46DCE7622B27D168223946EB
:1050E00053F000FA0446C0690023002298F900C07A
:1050F00099F8001041FA0CF120F8021B2169D6F84A
:1051000004E0D5F804C001328A42F144E044EDD312
:10511000326801FB1E2291442A6801FB1C22904444
:10512000E26801339342E0D3FEF7A7BF482B27D1B3
:105130001A46394653F0D6F90446C06900230022C6
:10514000B8F800C099F8001041FA0CF120F8021BE1
:105150002169D6F804E0D5F804C001328A42F1444E
:10516000E044EDD3326801FB1E2291442A6801FB22
:105170001C229044E26801339342E0D3FEF77DBFE6
:105180006822394653F0AEF90446C0690023002274
:10519000B8F900C099F8001041FA0CF120F8021B90
:1051A0002169D6F804E0D5F804C001328A42F144FE
:1051B000E044EDD3326801FB1E2291442A6801FBD2
:1051C0001C229044E26801339342E0D3FEF755BFBE
:1051D000622A40F0A8800B79422B27D168223946F9
:1051E00053F080F90446C0690023002298F800C0FB
:1051F00099F9001041FA0CF120F8021B2169D6F848
:1052000004E0D5F804C001328A42F144E044EDD311
:10521000326801FB1E2291442A6801FB1C22904443
:10522000E26801339342E0D3FEF727BF622B28D117
:10523000394653F057F9C26904460020134698F9DD
:1052400000C099F9001041FA0CF103F8011BD4F8E1
:1052500010C0D6F804A0D5F804E0991A8C45D144C2
:10526000F044ECD82A6831680CFB1E229044E268B6
:1052700001300CFB1A1190428944BEF4FEAE1A466E
:10528000DCE7482B27D11A46394653F02BF9044660
:10529000C06900230022B8F800C099F9001041FA53
:1052A0000CF120F8021B2169D6F804E0D5F804C0FF
:1052B00001328A42F144E044EDD3326801FB1E2200
:1052C00091442A6801FB1C229044E2680133934216
:1052D000E0D3FEF7D2BE6822394653F003F9044604
:1052E000C06900230022B8F900C099F9001041FA02
:1052F0000CF120F8021B2169D6F804E0D5F804C0AF
:1053000001328A42F144E044EDD3326801FB1E22AF
:1053100091442A6801FB1C229044E26801339342C5
:10532000E0D3FEF7AABE482A40F0A7800B79422BB3
:1053300026D1394653F0D6F80446C069002300222E
:1053400098F800C0B9F8001041FA0CF120F8021BDF
:105350002169D6F804E0D5F804C001328A42F1444C
:10536000E044EDD3326801FB1E2291442A6801FB20
:105370001C229044E26801339342E0D3FEF77DBEE5
:10538000622B29D11A46394653F0ACF8C26904465B
:105390000020134698F900C099F9001041FA0CF169
:1053A00003F8011BD4F810C0D6F804A0D5F804E027
:1053B000991A8C45D144F044ECD82A6831680CFB2A
:1053C0001E229044E26801300CFB1A11904289447D
:1053D000BEF453AE1A46DCE7482B26D1394653F0CB
:1053E00081F80446C06900230022B8F800C0B9F86B
:1053F000001041FA0CF120F8021B2169D6F804E0F4
:10540000D5F804C001328A42F144E044EDD3326859
:1054100001FB1E2291442A6801FB1C229044E26891
:1054200001339342E0D3FEF728BE6822394653F099
:1054300059F80446C06900230022B8F900C0B9F841
:10544000001041FA0CF120F8021B2169D6F804E0A3
:10545000D5F804C001328A42F144E044EDD3326809
:1054600001FB1E2291442A6801FB1C229044E26841
:1054700001339342E0D3FEF700BE682A40F0A080DB
:105480000B79422B394625D153F02CF80446C069DC
:105490000023002298F800C0B9F9001041FA0CF17D
:1054A00020F8021B2169D6F804E0D5F804C00132C7
:1054B0008A42F144E044EDD3326801FB1E2291445C
:1054C0002A6801FB1C229044E26801339342E0D336
:1054D000FEF7D3BD622B25D153F004F80446C06912
:1054E0000023002298F900C0B9F9001041FA0CF12C
:1054F00020F8021B2169D6F804E0D5F804C0013277
:105500008A42F144E044EDD3326801FB1E2291440B
:105510002A6801FB1C229044E26801339342E0D3E5
:10552000FEF7ABBD482B25D152F0DCFF0446C06925
:1055300000230022B8F900C0B9F8001041FA0CF1BC
:1055400020F8021B2169D6F804E0D5F804C0013226
:105550008A42F144E044EDD3326801FB1E229144BB
:105560002A6801FB1C229044E26801339342E0D395
:10557000FEF783BD52F0B6FF0446C0690023002247
:10558000B8F900C0B9F9001041FA0CF120F8021B7B
:105590002169D6F804E0D5F804C001328A42F1440A
:1055A000E044EDD3326801FB1E2291442A6801FBDE
:1055B0001C229044E26801339342E0D3FEF75DBDC4
:1055C0000024FEF75ABD00BF38B50C4BD3F8B430F9
:1055D00004460D4643B90C204BF0ADFD2A4621464A
:1055E000BDE8384000F00CB89A68A24202D15A686F
:1055F000AA4201D01B68EDE738BD00BFBC620120A4
:1056000070B5094CD4F8B4502B462BB9C0E9005200
:105610008160C4F8B40070BD9E688E4202D15E689D
:105620009642F8D01B68F0E7BC62012030B5094A09
:1056300052F8B43F4BB19C6884421C6806D15D6847
:105640008D4203D1146000221A6030BD1A462346F1
:10565000F0E700BFBC620120044B1B7823B1044873
:1056600043680BB144F0FABC184670475B6D0120EB
:10567000B04F012008B50348012104F02FFA0E2095
:1056800008BD00BF4851012070B52DED028B8EB0D2
:1056900006AB0193574B00930431022301381AF0F3
:1056A00089FC40F29F22544906981AF069FD40F2A5
:1056B000236104469FED510A07981AF04FFD2046DA
:1056C00004A9B0EE408A42F04FF90E2200210AA848
:1056D0004BF061FEDFED4A7A9FED4A7A4A4B4B4A26
:1056E0000A9328EE278AA023C8EE077AADF82C305B
:1056F00010685168B6EE007A77EE877AFCEEE77AAA
:1057000017EE903AADF82E3008AB03C3404803A91A
:10571000FFF75AFF00238DF80E3008AA01230AA9CB
:1057200004A854F064FD044630B1394803A9FFF7DA
:105730007DFF204644F08EF99DF80E3063B1344869
:1057400003A9FFF773FFBDF80C604FF6FF739E428D
:1057500005D1304823F066FDFBF762FAECE7002044
:105760002AF00CFA0446B8B16378012B36D12378BD
:10577000DB0733D506220DF1110104F151004BF086
:10578000B5FD58BB04F1240204F13601304654F053
:105790003CFDB0FA80F46409002502A93046ADF85A
:1057A000085054F036FD4FF40071304654F047FD78
:1057B00044F050F929462A46304654F01CFD44F086
:1057C00049F9154B882101FB05F2D0189A5AB242CB
:1057D00006D00135052DF6D11048BBE72046BFE7BE
:1057E0000123837080F85A4000F066FD0EB0BDECD6
:1057F000028B70BD08250A00F4B309000000000008
:105800000024744900401C460001A00020E008006C
:10581000D7C50700944B0900600901209C4B090083
:105820002DE9F0410746806986B0F0B9104D044675
:1058300006464FF6FF782B8843450CD0E86D0E28BE
:1058400003D1284600F038FDE86506AB03EB84037E
:10585000013443F8140C0136052E05F18805EAD110
:1058600001A9204621F028FCB86106B0BDE8F0810E
:105870006009012008B501483BF0ACF9FD4D090075
:1058800007B50A799DF8003062F347038DF80030C0
:10589000D1F80530CDF801306846B1F80930ADF8DF
:1058A000053054F094FC10B1024823F0BBFC0E20EC
:1058B00003B000BDF54C09002DE9F04F2DED028B32
:1058C00095B00CAB51F8044B01935F4B009301383A
:1058D00008231AF06FFB0C98052209A91EF0EEF8B8
:1058E0000D9800230E28CDE90633089303D0052236
:1058F00006A91EF0E3F8119808B95448119040F237
:105900003B411AF053FCDFED527AB4EEE70AF1EEB8
:1059100010FAB0EE408A06D4DFED4E7AB4EEE70A14
:10592000F1EE10FA04DD4C4A4C494D483BF0B6F913
:10593000DDF840A0BAF1000F04DA40F22361002044
:105940001AF0CAFB0A9B9DF838601F2B05D926B1B7
:10595000079B13B1434823F065FC13980E280DD024
:105960000EB94148F7E7414940F27B321AF008FC92
:10597000074694F844301BB13D48ECE70027F8E7B0
:10598000E3689DF83C80DDF8489013B1204604F0B0
:1059900013FA0A9D3146284603F02EF9DDF81CB0B3
:1059A0003146584603F028F91F2D04D9BBF1000FEA
:1059B00002D03048CFE715B10FB12F48CBE7B8F18F
:1059C000000F09D12D4B2E4A03FB0AF3934205D950
:1059D0002C48B42123F026FC4FF0B40A616819B9B1
:1059E000FF2011F079FC6060A16819B9FF2011F067
:1059F00073FCA060DDE9091260684BF08BFCDDE907
:105A00000612A0684BF086FCCDE90497BDF81C3067
:105A10000393A3680293BDF8283001936368009351
:105A2000B0EE480A5346424631462046F4F7E0FDC0
:105A300044F010F840F201130E20A4F8443015B0E1
:105A4000BDEC028BBDE8F08F08240A00CECC4CBE22
:105A50000AD7A33C0AD72341C7200900CD2009005B
:105A60000A3B0900C34D090017480900F4B30900B7
:105A7000554F0900D04B0900BA4C090040420F00B5
:105A80000FBCBA0A4A4509002DE9F04F2DED068BEF
:105A900093B00AAB51F8044B0193834B0093013848
:105AA00008231AF087FA0D980E2828D09FED7F0A58
:105AB00040F223611AF052FBF0EE408A0E9808B9CA
:105AC0007B480E900F9B0BB9794B0F9340F23B41F3
:105AD0001AF06CFBDFED777AB4EEE70AF1EE10FA1C
:105AE000B0EE408A06D4DFED747AB4EEE70AF1EE48
:105AF00010FA07DD714A724972483BF0CFF8DFEDCA
:105B00006B8ADBE7F5EE408AF1EE10FA07D0F4EE8F
:105B1000C08AF1EE10FA02D56B483BF0B7F80F9847
:105B200040F285611AF042FBB4EEC08AF1EE10FA41
:105B3000B0EE409A01D56548EFE70A980023049338
:105B400058B1052203A91DF0B9FF049B2BB103989E
:105B500012F048F908B95E48DFE70B9F002F04DC1C
:105B600040F2FD2101201AF0B7FA23699DF8305068
:105B7000DDF840909DF84480DDE903BA3BB193F82D
:105B8000293013B9534823F04DFB00232361E36808
:105B900043B16268934202D1112003F001F920461B
:105BA00004F00AF94C499FED4DAA2C204DF0B1F8B4
:105BB00039460646083054F07AF9002DC6E907BA8E
:105BC000C6F8249026610CBF1F26FF2606F10800A8
:105BD0004BF0CFFA2369586000F108030360868018
:105BE0000746012042F0FCF943F034FF21693C48AC
:105BF000FFF7EAFC68EE8A6A9FED3A7AC6EE877A8A
:105C0000F6EE009A77EEA97AFCEEE77A17EE906A44
:105C1000B6F5803F01D334487FE736B9F5EEC08A48
:105C2000F1EE10FA01DD314877E70E22002106A8D7
:105C30004BF0B1FB28EE0A8A9FED2D7AADF81E607D
:105C4000C8EE077A45F4807545EA880525F0FA051F
:105C5000394606A8ADF8185029EE0A9A77EEA97AC7
:105C6000FCEEE77A17EE903AC9EE077AADF81A30F3
:105C700077EEA97AFCEEE77A17EE903AADF81C3091
:105C800054F0CFFA054640B115482169FFF7CEFC24
:105C900000232361284643F0DDFE206913B0BDECEC
:105CA000068BBDE8F08F00BF48240A00000000000A
:105CB000CECC4CBE0AD7233B66D62342D220090065
:105CC000DC2009000A3B0900533809003033090081
:105CD00084470900AB4609001CB30900002474493D
:105CE000817C060000401C46E93409006338090045
:105CF00000401C44022808B50B46114613D18A0700
:105D000013D108680A4A90420FD118790A79904253
:105D10000BD106220531581D4BF0E8FA00280CBFC4
:105D20003E201E2008BD0020FCE71E20FAE700BF31
:105D3000F4B3090010B588B0084611461A4603AB03
:105D40000193134B009302234BF07EFC05A90398AB
:105D500005221DF0B3FE069840F29F2206211AF09C
:105D6000CDF9049840F2A223032200214BF09FFCBE
:105D7000084904460C204CF0CCFF059B1A68C0F87B
:105D800005209B88A0F80930047108B010BD00BF41
:105D9000F8240A00F4B309001FB54B7903938B79FB
:105DA0000293CB7901930B7A00934B7A8A7A02495A
:105DB0004DF0C7F905B000BDE32009002DE9F04F13
:105DC00097B00DAB0193344B009304310923013894
:105DD0001AF0F0F831490D9840F2A6521AF0D0F9B5
:105DE0002F49089040F267620E981AF0C9F99DF8A1
:105DF0003C603F2E834603D940F214501AF0CCF891
:105E00009DF84070384644F017F99DF844804046AC
:105E100044F012F9129C002C04DA40F28641002072
:105E20001AF05AF914989DF84C500E2804D15DB31D
:105E300054B320464CF098FF0DF12809052249463D
:105E40001DF03CFE0B9840F22F422146F5B11AF0AE
:105E500055F915980E281CD022F07EF8824611497B
:105E600028204CF056FFCDE9059ACDE90345CDE950
:105E70000178089900965B460022099004F004F826
:105E8000099817B0BDE8F08F0748D5E71AF042F936
:105E9000DFE74FF0000AE2E7B0240A00FCB2090095
:105EA000D4B20900A8B309003862090010B54368EC
:105EB000044653B101460648FFF7B8FB0023C4E986
:105EC0000333C4E90633636063610E2010BD00BF75
:105ED0000399070070B52DED028B86B00846114678
:105EE0001A4603AB01931F4B009303234BF0ACFB0B
:105EF0001D49039840F213321AF042F940F223612F
:105F00000646B7EE000A04981AF028F9059D002D00
:105F1000B0EE408A04DC40F2FD2101201AF0DCF8EA
:105F2000124924204CF0F5FE044628464BF021F996
:105F3000DFED0F7A666028EE278A0023BCEEC88A60
:105F4000C4E90305C4E905330A4884ED028A84F8EC
:105F50002030E3612146FFF737FB204606B0BDEC59
:105F6000028B70BD88240A00A8B3090084B309001D
:105F700000007A440399070008B501483AF02AFE68
:105F8000754D090010B50446808A43F03EFDE36973
:105F90002BB1BDE81040D3E9020121F08DB80148D2
:105FA00010BD00BF3C31090070B58B6804460D463A
:105FB00016466BB107494DF0C4F8A9682046324631
:105FC00000F082FE04492046BDE870404DF0B9B8AB
:105FD0000249F9E70B210900F52109001B210900FD
:105FE000F0B50C4685B054F8045B0646A88A1746FF
:105FF00043F00BFD02AB0193084B00933A4602239A
:106000002146701E19F0D6FF28469DF80C209DF8F9
:10601000081004F07BF80E2005B0F0BDA0240A00A3
:1060200008B501483AF0BAFD89480900084930B579
:106030000022882505FB02F463180C5B844204D01F
:106040000132052AF6D1002030BD1846FCE700BF1A
:10605000600901202DE9F04F8BB004AB51F8048B9F
:106060000193784B00930138012319F0A3FFD8F86E
:106070000440204600F0F6F87348049D2146FFF7DF
:10608000A3FA002017F0B8FB0E2D606030D101217B
:106090000AE062689368D26803F18043013B52F8DA
:1060A0002330D98A013189B2002220460BF0B2FF99
:1060B0000028EED1654F002663689A68964236D371
:1060C00021466148FFF7B2FAD8F80440204600F0B4
:1060D000C9F86368D3E9020120F0EEFFD8F8043074
:1060E000044658684CF0ABFD20460BB0BDE8F08F7D
:1060F000284606A91DF04EFD554E054628461DF0C2
:106100000DFF0028D6D0830702D10368B34202D026
:1061100050483AF0A7FD8388ADF8143005AA83797A
:106120008DF81630012120460BF074FFE6E7DB689E
:1061300053F82650AB680BB90136BDE7AB8ADFF8E0
:106140001C91EA8A9A4212D3ADF81830DFF810A1F8
:10615000C9F800500023ADF81A203B7020880123B5
:1061600006A98AF8003054F066F800283DD02B6963
:106170009B6802930023029A9A42DDD02A69D16873
:106180005A1C0392029A51F823B0501E834216BF44
:1061900001EB830100234B68DBF8081009B3BBF85F
:1061A0001410013189B2002B32D09B8A013B1FFAB7
:1061B00083F9E88A884214D3494512D8264BADF8B2
:1061C0001810DFF89CA0C3F800B000213970ADF8BA
:1061D0001A9001218AF80010208806A954F02DF8A1
:1061E000D8B1039BC7E7FAF71BFD9AF80030002BE4
:1061F000F9D13B78002BBAD02A699368D26803F1B1
:106200008043013B52F823309B8A01339BB298E7CD
:10621000B5F81690CDE7FAF703FD9AF800100029BB
:10622000F9D139780029DCD0DBF81C008168C0681E
:1062300001F18041013950F82110898A013189B278
:10624000B7E700BF50250A0055200400E76E012083
:10625000D4B209008B3809009C62012098620120A9
:10626000E66E012008B543F009FF10B901483AF085
:1062700095FC08BD244D090038B544680D4D2046F5
:10628000FFF7F0FF94F874306BB9B4F86C3000EE9F
:10629000103AB8EEC00AF7EE047ABDE8384020EEB6
:1062A000270A20F07DBDAB6A002BEED1FAF7B8FCCF
:1062B000E8E700BFBC62012010B50446C06D0E289F
:1062C00005D103490C204CF024FD4460E06510BD6D
:1062D000C4B3090030B585B003AB51F8044B01934A
:1062E000224B00930138012319F064FE9DF80C3015
:1062F00033B91F4840F26B124FF43D713AF072FC13
:1063000064681C4D2046FFF7ADFF94F85A30012B0E
:1063100001D1AB6AEBB194F85A30022B22D00123A1
:10632000154984F85A302088124D53F05AFF43F033
:1063300091FB94F85A30012B01D1AB6A63B1AB6A7F
:1063400083B994F85B1069B1882908D10B4822F011
:1063500077FFFAF765FCD8E7FAF762FCE9E7084847
:1063600022F06EFF0E2005B030BD00BF58250A0098
:10637000B0500900BC620120A0220A00E0430900DD
:10638000374409002DE9F04796B00FAB01935B4B02
:10639000009304310723013819F00CFE58490F9877
:1063A00040F2133219F0ECFE564940F2676207469C
:1063B000109819F0E5FE9DF844908246484643F057
:1063C0003BFE9DF84880404643F036FE139E002E6B
:1063D00004DA40F28641002019F07EFE15989DF8FF
:1063E00050500E2804D14DB346B330464CF0BCFC9F
:1063F000052204A91DF062FB059840F22F423146A8
:10640000F5B119F07BFE404918204CF082FCC0E940
:10641000017A00230446838280F8169080F8178062
:10642000DDE9040120F010FCE060002D5CD1B6F540
:10643000007F08DD354A4FF400715BE03448D7E750
:1064400019F068FEDFE72682A574FB69002B47D0B0
:10645000A368A17D9A889B798DF80E3085F001059F
:106460000DF1080845F002050026404605F0070535
:10647000ADF80C20ADF808608DF80A5042F025FD0B
:10648000E17D0DF1090042F020FD052207A9E06839
:106490001DF014FB03ABCDE90A38089BADF8303092
:1064A000238AADF8343004F11402079BB88A0E93A6
:1064B0000AA9ADF8326053F0D2FE43F0CBFA154A88
:1064C000A18A1388F8698B4228BF0B461380124AB1
:1064D00013888B4238BF0B46214613804CF08CFB4F
:1064E000204616B0BDE8F087B6F5FF7FABDD0B4A5E
:1064F0004FF4FF710A483AF0D1FB00BF18250A009B
:10650000A8B30900D4B2090068B30900C5E00800C7
:106510003862090058050120D46A0120D0E0080043
:10652000D739090070B58B6804460D4616466BB125
:1065300007494CF006FEA9682046324600F0C4FB2D
:1065400004492046BDE870404CF0FBBD0249F9E724
:1065500043210900F52109004F2109007FB50446B8
:106560000522084601A91DF0A9FAA58A65B163684C
:106570005E68F06842F07CFDB37901463BB10023D0
:1065800001AA284642F0F8FD0E2004B070BDA07CA0
:10659000029B228A20B19A4206D006483AF076FB46
:1065A0009A4201D20448F9E701AA284642F00BFEBC
:1065B000EAE700BF9E43090093430900022A70B531
:1065C00004460E4615460BD14FF4227052F0DAFF06
:1065D000014620464CF0A6FD054920464CF0A2FDA0
:1065E0002A4631462046BDE870401FF047B800BF3C
:1065F000BAE0080070B5064686B008460D46144657
:1066000042F026FD00234FF400722048019401A9B6
:10661000CDE90223ADF810508DF81430FEF7D4FF09
:1066200000223146284653F010FE11280446F7D0C8
:1066300030B1164801A9FEF7F9FF204643F00AFAE7
:106640009DF81430B3B1BDF8100042F001FD01A96E
:106650000E48FEF7EBFFBDF8121089B291B140F27F
:106660000513994209D040F20F13994208D0084807
:1066700022F0D8FDFAF7D4FAE2E7064822F0E0FD6E
:106680000548FBE7039806B070BD00BFA579070079
:106690004C440900D54A0900CC4A090008B5014814
:1066A0003AF0F4FA204909002DE9F04788B008468D
:1066B00011461A4605AB01932D4B009303234AF074
:1066C000C3FF2C49059840F2133219F059FD069D7D
:1066D000002D074604DC40F2FD21012019F0FCFCEE
:1066E00007980E2836D17E8A234930204CF011FBC2
:1066F00040F2FD139E4228BF1E467B68BA7D9B79FF
:1067000002F03004804602F0060213B91346224616
:106710001C4642B306F1020905FB09F948464AF056
:1067200028FD054614B330464AF023FD8246304624
:106730004AF01FFD04460023CDE902634046CDE93F
:1067400000A44B462A463946F4F73EF8404608B0C6
:10675000BDE8F0874FF4916119F040FD061EC3DCDF
:106760004FF49161B9E715469146DBE7A246E2E7AF
:1067700090250A00A8B309004CB3090030B50D46B6
:1067800085B00446406843F03BF9062201A928463B
:106790001DF094F9DDE90112204643F0BBFC00280E
:1067A00003DA414203483AF079FA400040F0010030
:1067B00005B030BD834E090010B58AB002AB0C465F
:1067C0000193144B009304310223013819F0F2FBBA
:1067D0002468606843F014F90298052207A91DF0A7
:1067E0006DF9039800230E28059303D0052204A910
:1067F0001DF064F9059B0093DDE90712049B204618
:1068000003F06AFD20EAE070400040F001000AB0A9
:1068100010BD00BF80250A002DE9F041494D4A4BCB
:106820002B6043F0EAFB002800F08980474B1A7880
:10683000002A00F0848000221A70454B1A781AB999
:10684000444A1278012A2DD1434800241C7003F0D9
:1068500011FD424B9A8A02B19C82414B9A8A0AB13D
:1068600000229A823F4C6368BBB13F4B1B78A3B1B7
:10687000204603F019FD204603F0FCFC3B4B9A8AAE
:106880000AB100229A823A4B9A8A0AB100229A826D
:10689000384B9A8A0AB100229A82374B9A8A0AB1F7
:1068A00000229A82274803F0A5FAEB6813B1254825
:1068B00003F082FA0024AC61304D4FF6FF782E468B
:1068C0000E272888404502D0132153F09CFC013448
:1068D000052CEF6505F18805F3D155F044F84FF626
:1068E000FF7704460D4600231A4636F8131044334A
:1068F000B94218BF42F00102B3F5AA7FF5D142B107
:1069000055F031F8001B61EB0501802871F10001A1
:10691000E9D30C48002103F0E1F84FF42A23184A88
:106920001B68934205D14FF43122D2F8FC2F9A42D2
:1069300001D000F00DFCBDE8F04135F021BFBDE80D
:10694000F08100BF485101201CB409002A6E0120CB
:106950002E6E0120196F0120D84F0120F867012009
:1069600028680120085001205B6D01202867012064
:1069700078670120A8670120A45B0120600901203D
:106980003130444230B589B003AB51F8045B019318
:106990000E4B00930138022319F00CFB9DF81040B8
:1069A000039805A905221DF089F884F00104E86820
:1069B0000094DDE90523D0E9021042F048FC0028EC
:1069C0000CBF1E203E2009B030BD00BF70250A005C
:1069D0007FB5084611461A4602AB0193114B00934E
:1069E00002234AF031FE40F2676202980E4919F024
:1069F000C7FB0E499DF80C60054618204CF090F935
:106A00000446002016F0F8FE32460346294620468A
:106A1000F3F740FF43F01EF8054B012220461A70A1
:106A200004B070BD60250A00D4B20900FCB20900B0
:106A30002A6E012070B58B6804460D4616466BB170
:106A400007494CF07EFBA9682046324600F03CF92D
:106A500004492046BDE870404CF073BB0249F9E799
:106A600073210900F52109007C21090008B50148BE
:106A70003AF0B0F81747090010B5022888B00B4665
:106A8000144624D1A20720D12168124A91421CD178
:106A90009A79012A09D1A279012A06D19A88A38874
:106AA0009A4212D13E2008B010BD1846694643F004
:106AB00078FB04A9204643F074FB10220DEB020181
:106AC00068464AF013FC0028ECD01E20EBE70020BB
:106AD000E9E700BFD4B2090008B58B7813B90448C0
:106AE00022F0A0FB0B8883808B78837108BD00BFE8
:106AF000564409001FB58379012B02D105483AF0AD
:106B000045F8694643F04DFB1021684620F09CF89B
:106B100005B000BD46380900F0B51C4608468FB0E8
:106B200011464FF0021219F00DFA2068C20706D480
:106B300010F0030317D10168414A914213D14BF081
:106B400015FDA2234FF6FF7200214AF0B0FD3D492A
:106B5000054608204CF0DDF801230446858083714A
:106B600020460FB0F0BD384A0240062A05D0002B5F
:106B70004DD10268354B9A4249D101A921F0C4F99F
:106B8000019B242B02D032483AF080F8037A2D2B57
:106B9000F9D1437B2D2BF6D1837C2D2BF3D1C37DF3
:106BA0002D2BF0D1461E00F12304002516F8017F9D
:106BB000384639F0CBFF28B105F138036B44013575
:106BC00003F8207CB442F1D1202DDCD106AD0F2496
:106BD00002AE287856F0E7F90746687856F0E3F9F0
:106BE00040EA0710A055013C631C05F10205F0D1F5
:106BF00000231449BDF81450ADF8143008204CF0AF
:106C000088F802A98580044643F0B5FAA8E7012276
:106C100006A91CF053FF08B90E48B5E70798A22251
:106C2000102119F06BFA069B02AC03F110051868ED
:106C30005968224603C20833AB421446F7D1D7E75E
:106C400080320900D4B209000F0080FFF43009003F
:106C5000B6440900A7440900F0B589B003AB51F868
:106C6000044B0193174B00930138022319F0A2F94A
:106C7000062205A903981CF021FF069F0498002115
:106C800040F2CD433A464AF012FDA679012E14BFD8
:106C9000802110210546C9084FF43F72381A4AF086
:106CA00012FD059B012E03EB050107D1A2885A5561
:106CB000A3881B0A4B700E2009B0F0BD204643F09C
:106CC00070FAF8E7B8250A0010B58A79012A92B05F
:106CD000044606D18A881F4912B0BDE810404CF026
:106CE00030BA08460EA943F05CFA9DF838300D938F
:106CF0009DF839300C939DF83A300B939DF83B305A
:106D00000A939DF83C3009939DF83D3008939DF817
:106D10003E3007939DF83F3006939DF84030059331
:106D20009DF8413004939DF8423003939DF8433021
:106D300002939DF8443001939DF8453000939DF8EF
:106D400047209DF84630044920464CF0FAF912B02D
:106D500010BD00BF9D210900AA2109002DE9F047BF
:106D60002DED048B84B002AB0193344B00930223CE
:106D700019F020F9039C0E2C04D14FF480504BF0F5
:106D8000E5FF04460221204649F0ACFA074660B907
:106D900020461EF0E1FFC3880093294840F26D238E
:106DA0002E224FF4C26139F065FFDDF808809FEDB7
:106DB000258ADFED258A002507EE905AB8EEE70A0E
:106DC00007EB851920EE080A1FF0EAFF002682462D
:106DD000B7EE009A07EE906AB8EEE70A20EE080ACE
:106DE0001FF0DEFF5146024640464AF06CFD1EF0A1
:106DF00029FFB5EEC00AF1EE10FA1AD4B4EEC90AB2
:106E0000F1EE10FA17DC20EE280A30F0C5FAFCEE9D
:106E1000C07A17EE903A09F806300136402ED9D1E3
:106E20000135402DC8D1204604B0BDEC048BBDE82F
:106E3000F0870023EFE70123EDE700BFC42B0A0032
:106E4000015109002108823C00007C4238B50E4DFA
:106E50000E4C2B7813B1A37AFF2B13D10C4B0D489A
:106E60002360F6F727FA0C48F6F724FAFF23A372FB
:106E700000236360084A094B0649044803F058FBA5
:106E800001232B70014838BDD86E0120D45E01204B
:106E9000D4C6090074C709006CC70900A0860100A8
:106EA00038B5104D104C2B7813B1637AFF2B16D1E7
:106EB0000E4B0F482360F6F7FDF90E48F6F7FAF986
:106EC0000D48F6F7F7F9FF23637200236360094A60
:106ED000094B0749044803F0B3FC01232B70024817
:106EE00038BD00BF0F6F012000670120B8C6090040
:106EF00064C7090054C709005CC7090030B5164CC7
:106F0000164B227889B01AB193F82720FF2A20D196
:106F1000134A1A60134A1448C2F8EC30F6F7CAF95B
:106F20001248F6F7C7F901254023CDE90653082298
:106F30000023CDE904234FF41652CDE90232CDE906
:106F400000330A4A08490548B7EE000A03F026FE56
:106F50002570024809B030BD136F012094680120EC
:106F600094C60900BC6201200CC8090004C80900CD
:106F70002DE9F04F754C85B0002600AFA4F108084C
:106F80004FF0880909FB068393F87830002B65D011
:106F900054F0E9FCD4E91E23801A61EB0301B0F53B
:106FA0007A7F71F1000159D3002134F8080CF9807F
:106FB0000323BA1D6D4653F060F9002847D1FB88C2
:106FC00034F8080C0733DB08A5EBC3039D46BA1D54
:106FD00003236946EA4653F050F9002837D1B4F844
:106FE000502014F8060C022148F09FFE834660B141
:106FF000FB88C2889A4205D100F1080168464AF030
:1070000075F920B3584649F03EFC00233B7214F852
:10701000063C3A89F888F88143F4007302F0FE02D6
:1070200023F0FE0313433B81B4F850307B8134F8E6
:10703000083CBB810FF002F90222834607F10801E8
:1070400030F084FFFA885146584656F023FD8823D5
:1070500003FB06830022AD4683F8782009FB0683F4
:1070600093F87930002B41D014F8060C002847D053
:10707000B4F82EA05246012148F057FE054650B103
:10708000C288502A04D1214608304AF02FF940B373
:10709000284649F0F8FB002028F070FD054690BB1B
:1070A000387214F8063C3A89A7F80AA043F48073B2
:1070B00002F0FE0223F0FE03134350253B812846D5
:1070C00034F8083CBB81FD810FF0B8F802228246FB
:1070D00007F1080130F03AFF2A462146504656F0A3
:1070E000D9FC09FB0683002283F879200136052E9E
:1070F00004F188047FF446AF1437BD46BDE8F08F35
:10710000B4F812A0B6E76B78012B1DD12B7814F8D8
:10711000062C03F001039A4216D1B5F806B0BBF174
:10712000500F11D1062204F1490105F151004AF036
:10713000DDF848B95A46214605F108004AF0D6F86C
:1071400010B1284649F09FFB2846A5E768090120B1
:1071500073B5104D4FF42A244FF00106200B2E700A
:1071600053F0A7F808B930F0E1FE04F58054B4F507
:10717000322FF3D1084B019301A901224FF42A20A9
:1071800030F0E4FE0548012201A930F0DFFE02B034
:1071900070BD00BFFD6E012031304442FC1F0B006A
:1071A000032A05D11E2914BF044905494BF0BABF73
:1071B0001E2914BF03490449F8E700BF69E008002D
:1071C0006EE00800D0E00800C5E0080030B587B0E8
:1071D0000C460592D1E90123174904935528CDE9BE
:1071E0000212236809D054F8042C02A9184620F092
:1071F000D7FFA4F1080007B030BD184600931EF079
:10720000ABFD827B009B82B100EB820002A9056985
:10721000019318460422A8470090F6F73DF8DDE9EF
:10722000000310B120602046E5E718464BF0AAF9AC
:107230000146024839F01EFD1C5C09003F50090060
:107240002DE9F04F2DED028BB9B00AAF084611467B
:107250001A4607F150030193BA4B00931A234AF0E0
:10726000F3F93B6D786D3B60052207F144011CF09A
:1072700025FC40F2D121D7F8900056F07FF8F86352
:10728000D7F898001EF0DEFCD7F868B05A229BFBB6
:10729000F2F302FB13B3B0EE408A13B1AA4839F0FF
:1072A000F5FC97F8B0A0FE6EBAF1000F08D0012EE1
:1072B00006D0A64840F22F2240F2273139F0EEFCEA
:1072C000F5F782F9A24B036097F88450B7F9603064
:1072D0007D6297F888503B633D62B7F9643097F858
:1072E0008C50FB62FD6197F870307D6C7B63BD61F3
:1072F00097F8A030BD6C7D610446B7F8945097F8BC
:107300007400FB6097F8A43097F87CC097F880E091
:10731000B7F85810B7F85C20D7F8A890B8623D616C
:1073200097F8780097F89C50BB6397F8AC30BB6037
:107330004FF00008D7F8B4307B6084F8B380CDE913
:1073400004CE0390BB6A02937B6BB6B2CDE90063B7
:1073500004F108001FFA8BF346F0CCFA04F1500355
:107360007B63012E14BF00230AF00103CDE90783DC
:10737000CDF82480FB6806934FF48073CDE9043385
:107380003B6A03937B6A0293FB6A01933B6B009316
:10739000C5F58075ABB21A46396804F150000BF0A0
:1073A00073F9FB6984F8B2303B69A4F8AC30BB6B6D
:1073B000A4F8AE9083F0010384F8B430BB6884F87D
:1073C000B5301FFA89F94FF47A73B3FBF9F3A4F8D7
:1073D000B030BB8AFB62C346FB6A9B4537D35D4B2B
:1073E000C4F88430FB6BD3B1187943F0FFF9B0B126
:1073F00000220092BB88F96B04F1840005F08AF941
:10740000002800F08B80544BC4F88430F96B04F1F1
:10741000840042F028FFFB6B187943F0FCF9B0EED2
:10742000480A204602F0D6FF4C4991F82A309B07C3
:1074300002D4204642F0D4FEB96B204642F0BCFE96
:107440002046BC37BD46BDEC028BBDE8F08FBB6962
:1074500003EB0B0898F80150786B0BF007F9002844
:107460003AD094F880906BB23B6305F07F05B9F198
:10747000000F3CD005F1080303F0F803E946ADEB3B
:10748000030D98F800208DF828200AAB6E1C2A46C0
:1074900008F102010DF12900BB6249F03BFF0096A3
:1074A000266EBB6A206D01220021B047CD46786B65
:1074B00046F09BF83B6B002B2DDA6E1C023518F85A
:1074C0000500FF2808BF4FF4FA701CF0B3FB0BF166
:1074D000020306EB030B7FE7F9F7A2FB204B9B6A45
:1074E000002BB9D01F4840F2853139F0A5FB0123AC
:1074F0000093B5EB0902206D266E434618BF0122AA
:107500004946B0470095206D266E08F102034A46B1
:107510000121B047CBE72E460A20D6E7124BD4F81C
:107520008800C4F884302DF009FF94F88C200F49AE
:1075300002F07F02012393400A5C13430B54D4F8FA
:10754000903069E7D42E0A00554C09004F510900CC
:10755000F0C60900F063090034C6090044010120A7
:10756000BC6201208251090098BF0900EA6E012027
:10757000F0B58DB002AF07F108030C460193264B1E
:10758000009304310223013818F014FD206823F021
:1075900041FBD7E902650446062207F11C01284693
:1075A0001CF08CFA94F83A30102B02D01B4839F0BA
:1075B0006DFBA28E386ABA8202F00103002103EB50
:1075C00052033961B0EB830F7E8206F10106B96187
:1075D000FE821ED3520901327A607A68FB699200FA
:1075E000073222F00702ADEB020D02AA8C467E683C
:1075F00088B2864209D807F1100104F1080046F06C
:10760000AFF928462C37BD46F0BD42F820C0013105
:10761000EDE70348CBE700BFE4300A00674C090000
:107620007D4E090008B5014839F0FEFAA44E090064
:107630007FB502AB0C4601932B4B00930431022320
:10764000013818F0B7FC206823F0E4FA039B0446E5
:107650000298002BCABF4FF47A764FF0FF3696FBA4
:10766000F3F60E2811D04AF081FF4FF47A7595FB9E
:10767000F0F594F8B3305BB10023204684F8B430C1
:1076800040F003FA3E2004B070BD4FF0FF35F0E744
:1076900094F8B430002BEFD16B1CEDD054F063F9AB
:1076A0002369C31A9E4202D2104839F0BDFAD4F8B9
:1076B000A020821A9542C4E9280112D3B3FBF5F247
:1076C00005FB1233ED1A54F04EF9D4E92832C01AF2
:1076D00061EB0201A84271F10001CDD2F9F7A0FAE5
:1076E000F1E71E20CFE700BFC42E0A00D34E0900E9
:1076F00038B50D4623F08EFA044628461EF0A2FA4D
:10770000B5EEC00AF1EE10FA06D4B7EE007AB4EE88
:10771000C70AF1EE10FA01DD00F00CF8204602F085
:1077200059FE10B9024839F07FFA0E2038BD00BF6B
:10773000A44E090008B503480123002240F2FA21B3
:1077400039F0ACFA5851090008B5014839F01EFA71
:10775000BF4F090070B586B0084611461A4602AB05
:107760000193144B0093042349F06EFF40F29351B0
:10777000029855F0FBFD40F296510546039855F0EE
:10778000F5FD0D4906460C204BF0CAFAFF22049B7A
:107790008272297932799142044601D151F04BFF2E
:1077A000002242602946324602F0C2FE204606B060
:1077B00070BD00BFC4300A00D4C60900F0B50C4645
:1077C0008DB054F8045B0646A87A174642F001F9DA
:1077D000284642F039F908AB01931D4B009321462E
:1077E0000423701E3A4618F0E5FB062205A9099805
:1077F0001CF064F99DF81C100022402018F01EFDBA
:10780000069B0B99B3FBF0F30446049304AA0A9B6E
:10781000039303A850F077FF049E4FF43F720121B9
:10782000304649F050FF039A06FB04F3624303928B
:10783000049353B1059928460A44BDF8201002F07C
:10784000BBFF10B1404239F0D9F90E200DB0F0BDA8
:10785000A4300A00F0B50C468DB054F8045B06461F
:10786000A87A174642F0B5F8284642F0EDF808AB82
:1078700001931A4B0093214604233A46701E18F0D8
:1078800099FB052205A909981CF018F99DF81C1010
:107890000022402018F0D2FC069B0B99B3FBF0F3BA
:1078A0000446049304AA0A9B039303A850F02BFFF9
:1078B000039A049B0121009105996243039263435B
:1078C0000A442846BDF820100493F3F713F810B1CA
:1078D000404239F093F90E200DB0F0BD84300A001B
:1078E0002DE9F0410C4694B054F8046B0546B07A8B
:1078F000174642F06EF8304642F0A6F80DAB019301
:10790000314B00933A4607232146681E18F052FB7C
:1079100005220AA90E981CF0D1F89DF8301000221B
:10792000402018F08BFC0B9B1199B3FBF0F305463C
:10793000069306AA109B059305A850F0E4FE0622C4
:1079400007A90F981CF0BAF89DF8241000224020D7
:1079500018F074FC089B1399B3FBF0F304460493EE
:1079600004AA129B039303A850F0CDFE049F40F29B
:10797000D9420121384649F0A6FE0598069BBDF87C
:107980003480002268436B430092039D0A9A05905D
:10799000654302447C4341463046079F0693039566
:1079A0000494F2F7A7FF38B94CB123467A1941463F
:1079B000304602F001FF10B1404239F01FF90E20AD
:1079C00014B0BDE8F08100BF4C300A00F0B50C46A1
:1079D00087B054F8045B0646687A174641F0F3FF17
:1079E000284642F031F802AB0193184B0093214630
:1079F000701E04233A4618F0DDFA40F205530122C6
:107A00000021039849F053FE40F2F5430122002182
:107A10000446049849F04BFE40F2E323064609224F
:107A20000598082149F043FEC0B2082802D005207D
:107A300039F0E4F80299F3B2E2B2284642F0D9FBF9
:107A40000028F4D00E2007B0F0BD00BF0C300A00B3
:107A5000F0B587B0084611461A4602AB01931A4B9F
:107A60000093042349F0F0FD4FF44771029855F05C
:107A70007DFC40F2AC410746039855F07FFC40F294
:107A80009D410546049855F079FC064618B915B98C
:107A90000E4839F0FBF80E490C204BF041F99DF8E7
:107AA0001430FF220446427223B10A4840F20F41CB
:107AB00039F098F843602A463346394602F0C0FE52
:107AC000204607B0F0BD00BF2C300A0090490900E5
:107AD000B8C60900DF51090010B50446407A41F0EC
:107AE00072FF63681B68D3F82435B3F1805F23D03D
:107AF00013D8B3F1006F21D00BD8B3F1007F1FD0A2
:107B00001248B3F1806F18BF0020400040F0010020
:107B100010BD0F48B3F1206FF5E7B3F1804F11D0DE
:107B200006D8B3F1A05F0FD00A48B3F1005FEAE7CF
:107B30000948B3F1004FE6E70848E6E70848E4E7FC
:107B40000848E2E70848E0E70848DEE790D003008D
:107B50000024F40080841E0000127A0040420F00CE
:107B600020A1070048E8010000093D000048E801A5
:107B7000F0B50C468DB054F8045B0646687A17469B
:107B800041F021FF284641F05FFF08AB01931A4BFB
:107B90000093214604233A46701E18F00BFA062281
:107BA00005A908981BF08AFF9DF81C1000224020B0
:107BB00018F044FB099B0A9904930446069BB3FB07
:107BC000F0F303AA04A8039350F09DFD0499039BCE
:107BD000614303FB04F20491039252B105989DF8AE
:107BE0002C300144284642F023FB10B9052039F01F
:107BF00005F80E200DB0F0BDD42F0A00F0B50C46EC
:107C00008BB054F8045B0646687A174641F0DBFEF9
:107C1000284641F019FF07AB0193194B0093214609
:107C200003233A46701E18F0C5F9052204A90798E7
:107C30001BF044FF9DF818100022402018F0FEFAB7
:107C4000089B03930446059B0999B3FBF0F302AA32
:107C500003A8029350F057FD039B029A63436243CB
:107C60000393029242B104992846194402F05CFF42
:107C700010B9052038F0C2FF0E200BB0F0BD00BFD8
:107C8000F42F0A00F0B50C4693B054F8046B054687
:107C9000707A174641F097FE304641F0D5FE0CABA6
:107CA00001932B4B009321460623681E3A4618F099
:107CB00081F9052209A90C981BF000FF9DF82C10F2
:107CC0000022402018F0BAFA0E9B0F990593044643
:107CD0000A9BB3FBF0F304AA05A8049350F013FD2C
:107CE000062206A90D981BF0E9FE9DF8201000223F
:107CF000402018F0A3FA109B119903930546079BA7
:107D0000B3FBF0F302AA03A8029350F0FCFC049B1F
:107D1000039A0298059963436A4345436143AB4222
:107D2000059104930392029502D00A4838F0AEFF01
:107D300053B10698024409980144304602F0BCFE53
:107D400010B9052038F05AFF0E2013B0F0BD00BF67
:107D5000A42F0A00F44009002DE9F04F2DED028B0D
:107D600099B0084611461A460CAB0193494B009353
:107D70000C2349F069FC40F287510D9855F0FEFA4A
:107D800040F23E6104460C9855F0F8FA40F28351F7
:107D90000646149855F0F2FA40F24D310746159810
:107DA00055F0ECFA40F27E518046169855F0E6FA0E
:107DB00081461EB95CB9384838F068FFB44216D025
:107DC000BE4214D0464512D0864210D02CB1BC42DF
:107DD0000DD044450BD04C4509D01FB1474506D0C6
:107DE0004F4504D0B8F1000F03D0C84501D151F080
:107DF00022FC40F2E323092205210F9849F057FCA9
:107E0000C3B2099313984FF4A7634FF6FF72012191
:107E100049F04DFC109D214B9D421FFA80FB36D04E
:107E20001F4BEB1A5D425D416D009623022201213A
:107E3000119849F03CFC824612981DF003FFB0EE09
:107E4000408A55F0D1FA9DF85C2016490B922C20FF
:107E50004AF066FF5FFA8AF30B9ACDF81CB0CDE9C1
:107E60000553099B04930E9B0393CDE90192CDF832
:107E70000080B0EE480A3B46224631460A9002F0A6
:107E80008DFE0A9819B0BDEC028BBDE8F08F01257C
:107E9000CBE700BF3C310A0063340900D06709001A
:107EA000D467090094C6090010B522F01BFF0446F0
:107EB00090F8270041F081FD94ED030ADFED047A8C
:107EC000B8EE400ABDE8104080EE270A1EF068BFF9
:107ED00000007A4410B522F005FF044690F8270010
:107EE00041F06BFD6368186840F30730002801DB40
:107EF000F1F71EF90023C4E90733A36163681B6827
:107F000043F30733002B08DB5909012203F01F0359
:107F100002FA03F3024A42F821300E2010BD00BFDE
:107F200000E100E038B52DED028B0D4622F0DAFEBF
:107F3000044690F8270041F040FD28461DF082FEDF
:107F4000B0EE408A55F050FADFED057A28EE278A28
:107F50000E20BCEEC88A84ED038ABDEC028B38BDCE
:107F600000007A4413B50A4C40F2B31240F2611398
:107F7000A14218BF1346019340F2FD130093054937
:107F800040F2592340F201324BF0DBF802B010BD51
:107F9000D0670900052209002DE9F04715460E4675
:107FA0001F4622F09FFE044690F8270041F005FD91
:107FB0001DB900252846BDE8F08763681B68D3F823
:107FC0001435013304D12E4840F2875138F066FE53
:107FD00053F0C9FCDFF8B0A080468946A3699D42F2
:107FE00038D86368186840F30730002844DA2A4616
:107FF000314604F1100051F07DFF94F8253005461C
:1080000093B1012204F1240104F1100051F099FF11
:1080100004F12401606828F0F5F994F8290027F0AC
:1080200069FE002384F8253063681B6843F3073337
:10803000002B08DB5909012203F01F0302FA03F3A6
:10804000104A42F82130002DB4D10B233B604FF091
:10805000FF35AFE753F087FCE368B0EB080061EB56
:108060000901984271F10001BBD2F8F7D9FDDAF8A5
:108070002830002BB2D09CE7F1F75AF8B7E700BFE1
:108080004D49090000E100E0BC62012038B50C4612
:108090002046114606221D4617F054FF2CB92146F2
:1080A0000120BDE83840F4F7BFBE2968CB0706D4ED
:1080B00011F0030308D10868144A904204D1012C3E
:1080C00014D0134838F0CEFD124A0A40062A04D0D4
:1080D0003BB90A68104B9A4203D1012C01D10F48D9
:1080E000F0E7BDE838400120F4F7FEBD08464AF04D
:1080F0003DFA054601462046F4F796FE2A46044618
:108100000021C06849F047F9204638BD8032090097
:10811000F53209000F0080FFF43009003C350900FA
:10812000012807B50B4606D10B68009340F61623CD
:10813000019302206B460146002202481FF028FFEF
:1081400003B000BDF4300900014601481CF0E8BD51
:1081500098610900014A1CF029BE00BF986109001E
:10816000014A1CF023BE00BFF430090008B50846E0
:108170000AB117F019FF21B11946BDE8084000F017
:1081800005B8014808BD00BF3862090070B5064651
:10819000086810F003038EB00D4603D10168454A0C
:1081A00091422AD0444C00EA0402062A04D043BB80
:1081B0000268424B9A4224D1023E012E02D9404825
:1081C00038F050FD0AA91FF09FFE0646286800EA15
:1081D0000403062B13D1000951F0C0F904460A9D8F
:1081E00024B92946304651F090F90446314910200F
:1081F0004AF08FFDC0E9025644600EB070BD44687D
:10820000EDE7012E01D02F48DAE710F0010411D07C
:10821000441002D5002038F039FD21460AA855F057
:1082200079FB0C982246002149F0B5F80AA81EF007
:1082300013FDE2E701AA40F275211CF0C3FA019B8D
:108240002BB101AA2146204649F047FBD5E7286813
:10825000324603A91BF032FC20B1DDE903011EF018
:10826000F3FCCAE728681EF041FC0446B8B91020A8
:10827000CDE90A0448F05FFF8DF834400C9028687F
:1082800006A91BF087FC044620461BF047FE002889
:10829000CCD04AF06BF9FF2806D90B48BBE7411058
:1082A0000AA855F029FBEAE7C1B20AA855F070FA0E
:1082B000EAE700BF986109000F0080FFF430090071
:1082C0003C350900F5320900D2400900F0B585B00F
:1082D000054617460C461DF03FFD694606462846F2
:1082E0001FF012FE042F054622D1A307009814D1D7
:1082F0002268104B9A4210D101AA21464BF06BF82C
:1083000010B90D4838F066FCDDE901123046521A0A
:1083100029441EF077FE05B0F0BD01460023224639
:1083200030461BF0E9FB285C400040F00100F2E71A
:108330000020F0E71C5C0900A23709002DE9F14F8D
:108340008F0705460C46164613D001F00F03022B8B
:1083500019D102F0FD06012E4FEA111104D001B02F
:10836000BDE8F04F07F0F0B901B0BDE8F04F06F0FE
:10837000F9BE4968CBB22D2B00F087800BD8062BB5
:108380000ED02C2B13D0554A2146284601B0BDE80B
:10839000F04F07F0E7B92E2B00F08C809D2BF2D127
:1083A000002EF0D104F10802090A284687E0022ACB
:1083B00002D0A16806F02CFFE768002FE3D017F089
:1083C0000309E0D17B68DAB28E2AB8460DD1022EBD
:1083D0004FEA132805D007F1040A08F1FF3BD945FD
:1083E00015DB08F1010857F8288098F80430312B84
:1083F0002BD1022E13D1686A49F003FC686A562219
:108400006FF0020101B0BDE8F04F45F0F2BF5AF83D
:10841000041F284606F0FCFE09F10109DFE72846A3
:10842000D8F8081006F0F4FE012E686A09D1582227
:10843000022145F0DEFF686A01B0BDE8F04F49F067
:108440000ABC56226FF00201DCE7322B9BD1012ED1
:10845000686A0AD149F023FBD8F80810686A09094C
:1084600001B0BDE8F04F49F0CBBA022E01D149F07E
:10847000CCFBD8F80830686A1B0918226FF001019C
:1084800001B0BDE8F04F46F034B8A268002A3FF4CE
:108490007AAF002E7FF477AF5168090A022907D11D
:1084A000D3682BB1980703D11B79AC2B3FF46BAF8A
:1084B00008327AE7002A7FF466AFA16821B901B0DB
:1084C000BDE8F04F00F00CB88E0703D10B79922B6A
:1084D0000A46E1D004F10802012166E7994009004B
:1084E0002DE9F04701F1FF3A0546884691464FEAEB
:1084F0000A2700244FF0FF3617F5807F0CD1731C3C
:1085000005D1686A4346302251460BF031FA002407
:1085100044451DD1BDE8F08759F8241071B18A0790
:108520000CD10A79222A09D101360BD1686A47EAAF
:108530000403312251460BF01BFA26460134A7F5FD
:108540008077D9E72846084ABDE8F04707F00AB91E
:1085500059F82410A64208BF896800222846FFF770
:10856000EDFE0134D4E700BF3D39090001F00F03EF
:10857000022B2DE9F04707460C4604D1BDE8F04731
:10858000090906F08DBC00295BD011F0030558D114
:108590000B792C2B3FD1896806F03AFEE568002D57
:1085A0004FD015F003084CD16E68F2B28E2A2B46DC
:1085B00009D1360A05F1040906F1FF3AC24518DC73
:1085C000013655F826301A79312A1AD19968384679
:1085D00006F01EFE7C6A204649F0EDFA204649F07E
:1085E00010FB20465622BDE8F0476FF0020145F02F
:1085F00000BF59F8041F384606F00AFE08F10108CA
:10860000DCE7322A1DD19968786A0222BDE8F0477A
:10861000090949F0DDB92D2B13D18C688CB1636841
:108620001B0A022B01D1E36833B9261D6368B5EB41
:10863000132F0DD3BDE8F0879A07F6D11B79AC2B29
:10864000F3D121463846064ABDE8F04707F08AB81C
:1086500056F8041F3846FFF789FF0135E6E700BFEB
:108660003D40090070B5137803F06003202B5AD108
:108670002E4B90885C7884420ED093F83D4884421B
:1086800051D103F63C0001255478203C032C4AD8F4
:10869000DFE804F005050D3118460025F4E701294F
:1086A00003D10721043037F061FD012070BD01299D
:1086B00002D137F04BFDF8E70329F6D15188847FCA
:1086C000C17001F0010282F001018C4218BF817774
:1086D00052B95B68B3F5966FE7D14FF080434E22F5
:1086E000C3F81C252DF004FF114B124801221A700B
:1086F000F8F75AFAD9E70129DBD00329D5D10E4B77
:108700001B78002BD1D00D4B1B680133CDD0002D31
:10871000CBD15388002BC8D0094B0A4A9A6603F183
:1087200060029A62C1E70020C0E700BF1C10012070
:108730005D6D012018670120146F012020020120C7
:10874000BC620120FC6609002DE9F04741F2780285
:108750000021214848F01FFE1F4B204800211F46E2
:108760004FF0FF094FF4E1380A464FF0080E4FF47E
:10877000806540F63C0C012603F23C441C630CFB74
:1087800001744FF0000A83F80B90C3F804801A724A
:108790005A7283F80AE083F825209D8683F83620F4
:1087A0006287228783F80DA003F13C0AD862C3F8E0
:1087B00018A09D839E776284228400F140045C614E
:1087C0004C1C022C03F63C0300F180004FF0010129
:1087D000D2D1BDE8F08700BF1C1001201C0F012082
:1087E0002DE9F84F4B79022B81468A4615D18B79BA
:1087F000022B12D14D4F97F8266096B1BE7B86B101
:1088000097F8623863B197F84A384BB14FF0E023DC
:10881000D3F8F03DDB0700D500BE0020BDE8F88F9F
:10882000012640F63C037343F91807F803909AF8C1
:1088300002304B709AF800400AEB02085444444559
:10884000627805D223782344984501D3242A18D08E
:10885000052A0CD120463AF07FF80028D6D040F601
:108860003C0303FB0673A2789A7023781C44637858
:10887000042B38D163790A2B35D123464FF0000BF6
:108880002AE01C46DBE743452CD29D18A84529D396
:108890006B78052BBAD1EB7803F00303022BB5D12B
:1088A00028463AF059F80028B0D0AB78DB091ED042
:1088B00040F63C0303FB067383F80C90AA789A7386
:1088C000AA88C2F30A021A8240225A8200225A84DB
:1088D0001A840BF1010B2B4621795FFA8BF291423E
:1088E0001A78D0D89C18A4EB0A0080B296E740F61C
:1088F0003C0C0CFB0673AA8883F82490A97883F8B3
:1089000026107042A98800EA0C00C2F30A02243043
:10891000C1F30A015A85384400225A8719851A87FB
:1089200054F039F80028D4D170E700BF1C100120A2
:1089300000220A4B30B5114614460125987F1C6071
:1089400000B99D77501C022883F8261099734FF0C8
:10895000010203F63C03F1D130BD00BF1C10012021
:108960002DE9F0476F4C984694F8263099420F460F
:108970007AD0A27B8A421BD0A2788A4200D1B9B9B0
:1089800094F862389F4272D094F84A28BA4269D06B
:1089900094F83E28BA4201D1002F63D14FF0E02372
:1089A000D3F8F03DDB0700D500BE0020BDE8F0871E
:1089B00000256E4226F4F86626F0030636059F422F
:1089C0004FEA16563CD140F63C0303FB054306F143
:1089D0002409D96AA14431B106F130001FFA88F2A6
:1089E000204454F0FCF840F63C0101FB0541C87AF4
:1089F000FF281ED00A8F4B8FB1F834E092B29BB2A1
:108A00009A42B6BFC3EB4E0AA2EB030A92441FFA86
:108A10008AFAD6450AD2724540F63C012BD3A2EB26
:108A20000E0301FB05419BB24B87F246BAF1000FE2
:108A300046D14846B9F81430B9F8163053F0ABFFB8
:108A400040F63C0303FB0545AB7BBB4208D10C362B
:108A5000A01954F01CF818B94146A01954F059F85F
:108A60000120A3E70125A4E700263546ABE740F641
:108A70003C060125A7E702EB0E0301FB05419BB273
:108A80004B87F2469E451ED940F63C0101FB05414D
:108A90009A42096B01EB030C19D8AEEB0302AAEB67
:108AA0000E0E73449BB292B29BB1013B0B44002B60
:108AB000BFD04FF0000E013A14E0A2EB0E0292B2CA
:108AC0009645FAD9DEE7A3EB0E039BB2DAE75246EE
:108AD0000021531E6344EAE78B421ED10CEB0203D4
:108AE0000EF1010EC645A4D093F800A08245F3D143
:108AF0000D4B1B6898429CD140F63C0303FB054399
:108B0000002248465A871A8753F045FF074B084A08
